:020000040800F2
:1000000000000220054C00081D850008018500083D
:1000100021850008258500082985000800000000CA
:100020000000000000000000000000005142020833
:100030002B85000800000000C1440208B7450208F3
:10004000554C0008554C0008554C0008554C00080C
:10005000554C0008554C00082D850008554C0008EB
:10006000554C00083385000839850008554C0008B8
:100070003F8500084B850008554C0008554C00088A
:10008000554C0008554C0008554C00085785000891
:10009000638500086F850008554C00087B850008C3
:1000A00081850008554C0008554C0008554C000847
:1000B000554C0008554C0008554C0008554C00089C
:1000C000554C0008554C0008554C0008554C00088C
:1000D000554C00088D850008554C0008554C00080B
:1000E000554C0008554C0008554C0008554C00086C
:1000F000554C0008554C0008554C0008B1850008C7
:10010000554C0008554C0008554C0008554C00084B
:10011000554C0008554C0008BD850008C9850008ED
:10012000D5850008554C0008E1850008ED850008DC
:10013000554C0008554C0008554C0008F98500083E
:100140000586000811860008554C0008C1510008BA
:100150001D860008298600083586000841860008AB
:10016000554C0008554C0008554C0008554C0008EB
:10017000554C0008554C0008554C00080000000084
:08018000554C0008554C000825
:1002000010F8012B11F8013B012A28BF9A42F7D0C0
:10021000D01A704710B488420DD98B1898420AD270
:10022000811832B19A1A13F8014D9A4201F8014D22
:10023000F9D110BC7047002AFBD00A44431E11F8C4
:10024000014B8A4203F8014FF9D110BC70470000FE
:1002500001F0FF01102A2BDB10F0070F08D010F877
:10026000013B013A8B422DD010F0070F42B3F6D17B
:10027000F0B441EA012141EA014122F007047FF094
:1002800000070023F0E80256083C85EA010586EAEB
:10029000010685FA47F5A3FA87F586FA47F6A5FA27
:1002A00087F68EB9EED1F0BC01F0FF0102F0070233
:1002B00032B110F8013B013A83EA010313B1F8D1DE
:1002C0000020704701387047002D06BF35460338BF
:1002D000073815F0010F07D1013015F4807F02BFF8
:1002E000013015F4C03F0130F0BC0138704700BF49
:1002F000034613F8012B002AFBD1181A0138704766
:1003000070B4840746D04C1E002941D0D5B20346B4
:1003100002E0611EE4B30C4603F8015B9907F8D1D3
:10032000032C2ED9D5B245EA05250F2C45EA054503
:1003300019D9264603F11001103E0F2E41F8105C2A
:1003400041F80C5C41F8085C41F8045C01F11001D3
:10035000F2D8A4F1100121F00F0104F00F041031C4
:10036000032C0B440DD91E4621460439032946F8B7
:10037000045BFAD8211F21F0030104310B4404F07F
:1003800003042CB1D2B21C4403F8012BA342FBD1CD
:1003900070BC70470C460346C2E7000081F0004184
:1003A00002E000BF83F0004330B54FEA41044FEA5A
:1003B000430594EA050F08BF90EA020F1FBF54EAF5
:1003C000000C55EA020C7FEA645C7FEA655C00F091
:1003D000E2804FEA5454D4EB5555B8BF6D420CDD62
:1003E0002C4480EA020281EA030382EA000083EAE5
:1003F000010180EA020281EA0303362D88BF30BD85
:1004000011F0004F4FEA01314FF4801C4CEA1131DA
:1004100002D0404261EB410113F0004F4FEA033339
:100420004CEA133302D0524263EB430394EA050FC4
:1004300000F0A780A4F10104D5F1200E0DDB02FA33
:100440000EFC22FA05F2801841F1000103FA0EF2C7
:10045000801843FA05F359410EE0A5F120050EF18D
:10046000200E012A03FA0EFC28BF4CF0020C43FABE
:1004700005F3C01851EBE37101F0004507D54FF0CB
:10048000000EDCF1000C7EEB00006EEB0101B1F51B
:10049000801F1BD3B1F5001F0CD349085FEA300061
:1004A0004FEA3C0C04F101044FEA445212F5800F6C
:1004B00080F09A80BCF1004F08BF5FEA500C50F109
:1004C000000041EB045141EA050130BD5FEA4C0CEC
:1004D000404141EB0101013C28BFB1F5801FE9D249
:1004E00091F0000F04BF01460020B1FA81F308BF6C
:1004F0002033A3F10B03B3F120020CDA0C3208DD38
:1005000002F1140CC2F10C0201FA0CF021FA02F112
:100510000CE002F11402D8BFC2F1200C01FA02F182
:1005200020FA0CFCDCBF41EA0C019040E41AA2BFA7
:1005300001EB0451294330BD6FEA04041F3C1CDA6F
:100540000C340EDC04F11404C4F1200220FA04F08F
:1005500001FA02F340EA030021FA04F345EA030139
:1005600030BDC4F10C04C4F1200220FA02F001FAFB
:1005700004F340EA0300294630BD21FA04F029467D
:1005800030BD94F0000F83F4801306BF81F4801116
:100590000134013D4EE77FEA645C18BF7FEA655C89
:1005A00029D094EA050F08BF90EA020F05D054EA5B
:1005B000000C04BF1946104630BD91EA030F1EBF60
:1005C0000021002030BD5FEA545C05D14000494164
:1005D00028BF41F0004130BD14F580043CBF01F557
:1005E000801130BD01F0004545F0FE4141F470013D
:1005F0004FF0000030BD7FEA645C1ABF1946104618
:100600007FEA655C1CBF0B46024650EA013406BF18
:1006100052EA033591EA030F41F4002130BD00BFD7
:1006200090F0000F04BF0021704730B54FF4806494
:1006300004F132044FF000054FF0000150E700BF15
:1006400090F0000F04BF0021704730B54FF4806474
:1006500004F1320410F0004548BF40424FF0000161
:100660003EE700BF42004FEAE2014FEA31014FEAA4
:1006700002701FBF12F07F4393F07F4F81F06051F3
:10068000704732F07F4208BF704793F07F4F04BF3E
:1006900041F40021704730B54FF4607401F000451B
:1006A00021F000411CE700BF50EA010208BF70477B
:1006B00030B54FF000050AE050EA010208BF70476C
:1006C00030B511F0004502D5404261EB41014FF4D5
:1006D000806404F132045FEA915C3FF4D8AE4FF0DD
:1006E00003025FEADC0C18BF03325FEADC0C18BFC0
:1006F000033202EBDC02C2F1200300FA03FC20FA11
:1007000002F001FA03FE40EA0E0021FA02F114445D
:10071000BDE600BF70B54FF0FF0C4CF4E06C1CEA76
:1007200011541DBF1CEA135594EA0C0F95EA0C0FE7
:1007300000F0DEF82C4481EA030621EA4C5123EA5A
:100740004C5350EA013518BF52EA033541F4801189
:1007500043F4801338D0A0FB02CE4FF00005E1FB3C
:1007600002E506F00042E0FB03E54FF00006E1FB86
:1007700003569CF0000F18BF4EF0010EA4F1FF04C9
:10078000B6F5007F64F5407404D25FEA4E0E6D4109
:1007900046EB060642EAC62141EA55514FEAC5201A
:1007A00040EA5E504FEACE2EB4F1FD0C88BFBCF596
:1007B000E06F1ED8BEF1004F08BF5FEA500E50F147
:1007C000000041EB045170BD06F0004646EA01010D
:1007D00040EA020081EA0301B4EB5C04C2BFD4EB3F
:1007E0000C0541EA045170BD41F480114FF0000E38
:1007F000013C00F3AB8014F1360FDEBF002001F0A6
:10080000004170BDC4F10004203C35DA0C341BDC1F
:1008100004F11404C4F1200500FA05F320FA04F0F1
:1008200001FA05F240EA020001F0004221F0004125
:1008300010EBD37021FA04F642EB06015EEA430E98
:1008400008BF20EAD37070BDC4F10C04C4F12005C8
:1008500000FA04F320FA05F001FA04F240EA02007B
:1008600001F0004110EBD37041F100015EEA430E4C
:1008700008BF20EAD37070BDC4F1200500FA05F26C
:100880004EEA020E20FA04F301FA05F243EA0203EB
:1008900021FA04F001F0004121FA04F220EA0200FA
:1008A00000EBD3705EEA430E08BF20EAD37070BD40
:1008B00094F0000F0FD101F00046400041EB010120
:1008C00011F4801F08BF013CF7D041EA060195F002
:1008D000000F18BF704703F00046520043EB0303BC
:1008E00013F4801F08BF013DF7D043EA06037047A9
:1008F00094EA0C0F0CEA135518BF95EA0C0F0CD0B4
:1009000050EA410618BF52EA4306D1D181EA0301F9
:1009100001F000414FF0000070BD50EA410606BFF3
:100920001046194652EA430619D094EA0C0F02D138
:1009300050EA013613D195EA0C0F05D152EA03367D
:100940001CBF104619460AD181EA030101F000419B
:1009500041F0FE4141F470014FF0000070BD41F0E4
:10096000FE4141F4780170BD70B54FF0FF0C4CF4BE
:10097000E06C1CEA11541DBF1CEA135594EA0C0FDD
:1009800095EA0C0F00F0A7F8A4EB050481EA030E2A
:1009900052EA03354FEA013100F088804FEA033311
:1009A0004FF0805545EA131343EA12634FEA0222DF
:1009B00045EA111545EA10654FEA00260EF00041A0
:1009C0009D4208BF964244F1FD0404F5407402D2F2
:1009D0005B084FEA3202B61A65EB03055B084FEA83
:1009E00032024FF480104FF4002CB6EB020E75EB80
:1009F000030E22BFB61A754640EA0C005B084FEAA8
:100A00003202B6EB020E75EB030E22BFB61A754624
:100A100040EA5C005B084FEA3202B6EB020E75EB6F
:100A2000030E22BFB61A754640EA9C005B084FEAE7
:100A30003202B6EB020E75EB030E22BFB61A7546F4
:100A400040EADC0055EA060E18D04FEA051545EAE3
:100A500016754FEA06164FEAC30343EA52734FEA8C
:100A6000C2025FEA1C1CC0D111F4801F0BD141EA05
:100A700000014FF000004FF0004CB6E711F4801F6A
:100A800004BF01430020B4F1FD0C88BFBCF5E06F4A
:100A90003FF6AFAEB5EB030C04BFB6EB020C5FEA5A
:100AA000500C50F1000041EB045170BD0EF0004EAF
:100AB0004EEA113114EB5C04C2BFD4EB0C0541EAE1
:100AC000045170BD41F480114FF0000E013C90E6DE
:100AD00045EA060E8DE60CEA135594EA0C0F08BFA2
:100AE00095EA0C0F3FF43BAF94EA0C0F0AD150EAA1
:100AF00001347FF434AF95EA0C0F7FF425AF104634
:100B000019462CE795EA0C0F06D152EA03353FF45B
:100B1000FDAE1046194622E750EA410618BF52EAD8
:100B200043067FF4C5AE50EA41047FF40DAF52EAAC
:100B300043057FF4EBAE12E74FF0FF3C06E000BF49
:100B40004FF0010C02E000BF4FF0010C4DF804CD56
:100B50004FEA410C7FEA6C5C4FEA430C18BF7FEA16
:100B60006C5C1BD001B050EA410C0CBF52EA430C44
:100B700091EA030F02BF90EA020F0020704710F1C4
:100B8000000F91EA030F58BF994208BF90422CBF53
:100B9000D8176FEAE37040F0010070474FEA410C4C
:100BA0007FEA6C5C02D150EA013C07D14FEA430C6A
:100BB0007FEA6C5CD6D152EA033CD3D05DF8040BDB
:100BC000704700BF8446104662468C46194663460D
:100BD00000E000BF01B5FFF7B7FF002848BF10F1E4
:100BE000000F01BD4DF808EDFFF7F4FF0CBF012029
:100BF00000205DF808FB00BF4DF808EDFFF7EAFFA5
:100C000034BF012000205DF808FB00BF4DF808ED5F
:100C1000FFF7E0FF94BF012000205DF808FB00BF54
:100C20004DF808EDFFF7CEFF94BF012000205DF8DE
:100C300008FB00BF4DF808EDFFF7C4FF34BF0120EB
:100C400000205DF808FB00BF4FEA410C7FEA6C5CB6
:100C500002D150EA013C0AD14FEA430C7FEA6C5CB6
:100C600002D152EA033C02D14FF0000070474FF02E
:100C7000010070474FEA410212F5001215D211D55A
:100C80006FF47873B3EB625212D94FEAC12343F089
:100C9000004343EA505311F0004F23FA02F018BF0B
:100CA000404270474FF00000704750EA013005D1D4
:100CB00011F0004008BF6FF0004070474FF0000097
:100CC000704700BF4FEA4102B2F1E04324BFB3F5E1
:100CD000001CDCF1FE5C0DD901F0004C4FEAC002B3
:100CE0004CEA5070B2F1004F40EB830008BF20F097
:100CF0000100704711F0804F21D113F13872BCBF51
:100D000001F00040704741F480114FEA5252C2F1A5
:100D10001802C2F1200C10FA0CF320FA02F018BFEE
:100D200040F001004FEAC1234FEAD32303FA0CFC41
:100D300040EA0C0023FA02F34FEA4303CCE77FEAD0
:100D4000625307D150EA01331EBF4FF0FE4040F41A
:100D50004000704701F0004040F0FE4040F40000C9
:100D6000704700BF80F0004002E000BF81F000410A
:100D700042001FBF5FEA410392EA030F7FEA226C41
:100D80007FEA236C6AD04FEA1262D2EB1363C1BFD1
:100D9000D218414048404140B8BF5B42192B88BF40
:100DA000704710F0004F40F4000020F07F4018BF63
:100DB000404211F0004F41F4000121F07F4118BF83
:100DC000494292EA030F3FD0A2F1010241FA03FC2B
:100DD00010EB0C00C3F1200301FA03F100F0004313
:100DE00002D5494260EB4000B0F5000F13D3B0F1DB
:100DF000807F06D340084FEA310102F10102FE2A4A
:100E000051D2B1F1004F40EBC25008BF20F00100B9
:100E100040EA03007047490040EB0000013A28BF58
:100E2000B0F5000FEDD2B0FA80FCACF1080CB2EBDB
:100E30000C0200FA0CF0AABF00EBC2505242184359
:100E4000BCBFD0401843704792F0000F81F40001FE
:100E500006BF80F400000132013BB5E74FEA4103D1
:100E60007FEA226C18BF7FEA236C21D092EA030F3D
:100E700004D092F0000F08BF0846704790EA010FB7
:100E80001CBF0020704712F07F4F04D1400028BFE4
:100E900040F00040704712F100723CBF00F50000C6
:100EA000704700F0004343F0FE4040F400007047FC
:100EB0007FEA226216BF08467FEA236301464202A8
:100EC00006BF5FEA412390EA010F40F480007047BB
:100ED0004FF0000304E000BF10F0004348BF404261
:100EE0005FEA000C08BF704743F0964301464FF09D
:100EF00000001CE050EA010208BF70474FF00003F9
:100F00000AE000BF50EA010208BF704711F0004339
:100F100002D5404261EB41015FEA010C02BF844609
:100F20000146002043F0B64308BFA3F18053A3F568
:100F30000003BCFA8CF2083AA3EBC25310DB01FAAF
:100F400002FC634400FA02FCC2F12002BCF1004F33
:100F500020FA02F243EB020008BF20F001007047C4
:100F600002F1200201FA02FCC2F1200250EA4C0018
:100F700021FA02F243EB020008BF20EADC7070475E
:100F80007BB972B90029BEBF00204FF0004106E0D6
:100F900008BF00281CBF6FF000414FF0FF3000F089
:100FA00057B8ADF1080C6DE904CE002909DB002B20
:100FB0001ADB26F09DFADDF804E0DDE9022304B037
:100FC0007047404261EB4101002B1BDB26F090FA99
:100FD000DDF804E0DDE9022304B0404261EB4101A9
:100FE000524263EB43037047524263EB430326F0E4
:100FF0007FFADDF804E0DDE9022304B0404261EB52
:1010000041017047524263EB430326F071FADDF869
:1010100004E0DDE9022304B0524263EB430370476E
:1010200053B94AB9002908BF00281CBF4FF0FF314F
:101030004FF0FF3000F00CB8ADF1080C6DE904CEB4
:1010400026F056FADDF804E0DDE9022304B070472B
:10105000704700BF4A0011D212F5001211D20DD50F
:101060006FF47873B3EB62520ED44FEAC12343F0AE
:10107000004343EA505323FA02F070474FF0000058
:10108000704750EA013002D14FF0FF3070474FF007
:10109000000070470348044B834202D0034B03B166
:1010A00018477047080300200803002000000000D4
:1010B0000548064B1B1AD90F01EBA301491002D0BA
:1010C000034B03B1184770470803002008030020B2
:1010D0000000000010B5064C237843B9FFF7DAFF93
:1010E000044B13B10448AFF300800123237010BDFB
:1010F00008030020000000008878020808B5054BAE
:101100001BB105490548AFF30080BDE80840FFF773
:10111000CFBF00BF000000000C0300208878020849
:1011200080B56F4686B005900598039003F0D5FD15
:1011300004A800F01BF80246694600204860212000
:10114000086040F22430C2F20000029047F6A0018D
:10115000C0F6020140F24433C2F2000301F091FDF7
:10116000029801F0A5FD039806B080BD81B0009003
:1011700041F27D10C0F6000001B0704780B56F46A7
:1011800084B00390029101920399029A019B00F0AE
:1011900002F804B080BD80B56F4688B00790069114
:1011A00005920493059801280DD1FFE747F6A900A1
:1011B000C0F6020000F0DBF847F6C600C0F60200F9
:1011C00000F0D5F8A5E0059802282FD1FFE7049894
:1011D000416847F6E300C0F60200FFF711F8E8B9EE
:1011E000FFE740F24430C2F200000290002101917A
:1011F000212225F0EEF9029947F6E800C0F6020038
:10120000202203F07FFD0198029981F8200047F623
:10121000EB00C0F6020000F0AAF806E047F6F30083
:10122000C0F6020000F0A3F8FFE771E0059803287C
:101230006DD1FFE70498416847F60410C0F602003C
:10124000FEF7DEFF002858D1FFE704988068FFF71B
:101250004FF8202851D1FFE7012007F8110C00209A
:1012600007F8120CFFE717F8120C1F281FDCFFE726
:101270000498806817F8121C405C24F0C5FF58B130
:10128000FFE70498806817F8122C805C40F2443124
:10129000C2F20001885403E0002007F8110C06E0B8
:1012A000FFE717F8120C013007F8120CDBE717F80C
:1012B000110CC007B8B1FFE747F6E800C0F602001E
:1012C00040F24431C2F200010091202203F01DFDE2
:1012D0000099002081F8200047F6EB00C0F60200DC
:1012E00000F045F808E00498816847F60810C0F659
:1012F000020000F03CF8FFE708E00498816847F638
:101300000810C0F6020000F032F8FFE7FFE7FFE741
:10131000FFE7002008B080BD80B56F4682B0019025
:10132000019820F0ABFB02B080BD80B56F4682B063
:101330000190019820F078FC02B080BD80B56F4626
:1013400040F26830C2F2000000F001F880BD81B0C8
:10135000009000980021016001B0704780B56F4691
:1013600040F26C30C2F20000FFF7F1FF80BD83B0A5
:1013700080B56F4685B03B61FA60B960049007F1B3
:1013800008000390049A03980290029B40F6E050F4
:10139000C2F20000043001904FF4807102F0CEFCE4
:1013A0000198FEF7A5FF0146019803F0BBFE00205F
:1013B00005B0BDE8804003B0704780B56F4690B07F
:1013C0000F900F98079003F0F4FE41F2BD40C0F675
:1013D000000002F0D6F800F0D1FE47F6F131C0F679
:1013E000020141F2D542C0F600020023069300F04C
:1013F00003FD0EA800F0A4F8069B02466846436071
:10140000036040F27030C2F20000039047F62311EF
:10141000C0F6020101F035FC039801F049FC0DA86B
:1014200000F096F8069B024668464360036040F26F
:101430009030C2F20000049047F62D11C0F6020170
:1014400001F01FFC049801F033FC0CA800F088F8B0
:10145000069B024668464360036040F2B030C2F229
:101460000000059047F63311C0F6020101F009FCB7
:10147000059801F01DFC06996A460320106040F2B1
:101480006C30C2F2000047F63812C0F602024FF488
:10149000807300F06DF806996A460420106040F2EF
:1014A0006830C2F2000047F64312C0F602024FF461
:1014B000007300F096F8079810B080BD80B56F46B5
:1014C00082B0019000910198009903F02BFE0098E2
:1014D00002B080BD80B56F4686B00490039103F0E2
:1014E00062FE20B9FFE7072007F8010C21E004980D
:1014F0004068029003F00DFCFFF7FCFC00EE100AC0
:101500009FED0E1A80EE010A10EE100AFFF7AAF8FE
:1015100041EC100B02986946086053EC102B47F61B
:101520004F10C0F6020001F059FB002007F8010C33
:10153000FFE717F8010C06B080BD00BF0024744916
:1015400081B0009041F25560C0F6000001B07047D4
:1015500081B0009041F2AF60C0F6000001B070476A
:1015600081B0009041F29F70C0F6000001B070475A
:1015700080B56F468EB08446B868CDF830C00B9108
:101580000A92099307F8150C0C9804900DA8039083
:1015900000F088F9082020F071FA014603980791BD
:1015A00000F080F901460B9A05A800F083F9DDF8F8
:1015B00010E007990598069A4A600860079B0A9907
:1015C000BDF8242017F8150CEC46CCF804E0CCF854
:1015D000000041F6CB00C0F6000021F027F90EB064
:1015E00080BD80B56F468EB08446B868CDF830C0F7
:1015F0000B910A92099307F8150C0C9804900DA80A
:10160000039000F083F9082020F038FA014603988F
:10161000079100F07BF901460B9A05A800F04AF902
:10162000DDF810E007990598069A4A600860079B64
:101630000A99BDF8242017F8150CEC46CCF804E004
:10164000CCF8000041F6CB00C0F6000021F0EEF827
:101650000EB080BD80B56F4684B0039002910192B8
:101660000399029A019B00F002F804B080BD80B596
:101670006F4686B0059004910392029340F2D030F9
:10168000C2F20000019022F043FB47F65810C0F66A
:101690000200FFF76CFE01984FF4806124F0C6FF52
:1016A0000146019803F03EFD002006B080BD80B5E4
:1016B0006F4684B00390029101920399029A019BB4
:1016C00000F002F804B080BD80B56F4686B004908B
:1016D0000391029201930298012807D1FFE747F690
:1016E0008610C0F60200FFF742FE42E00298022890
:1016F0003ED1FFE70198406847F6B911C0F60201F4
:10170000FEF77EFD28B9FFE70121084603F055FAF0
:101710002DE00198406847F6BF11C0F60201FEF7C0
:101720006FFD18B9FFE703F05AFA1FE0019840680F
:1017300047F6C411C0F60201FEF762FD18B9FFE7D3
:1017400003F04DFA11E00198406847F6CD11C0F65C
:101750000201FEF755FD38B9FFE701200590059815
:1017600080F3138800F008F8FFE7FFE7FFE7FFE7E3
:10177000FFE7002006B080BDBFF34F8F4EF60C513F
:10178000CEF20001086800F4E0600422C0F2FA52D0
:1017900010430860BFF34F8FFFE700BFFDE780B540
:1017A0006F4684B00390029101920399029A019BC3
:1017B00000F002F804B080BD80B56F468AB0099091
:1017C00008910792069303F0A2FA059005984AF64D
:1017D000AB21CAF6AA21A0FB012109094BF2C533AE
:1017E000C9F2A213A1FB0321CA0A44F6D351C1F2E4
:1017F0006201A2FB01C292090492A0FB01129109AD
:1018000044F2075CCCF22E2CA1FB0CEC4FEA1C4CF2
:1018100040F2A32E0CFB0EFCA1EBCC1CACFB03ECAA
:101820004FEADC2CCDF808C0A1FB0331C90A4FF404
:1018300061635943C1EB921148F68902C8F68802E8
:10184000A1FB02214909039100EE100AB8EE400AFB
:10185000DFED130A23F07CF910EE100AFEF702FF09
:1018600041EC100B51EC100B9FED0B0B53EC102BBC
:10187000FFF77AF8029A039B8C4604994CEC100B04
:10188000684680ED000B47F6D410C0F60200FFF763
:101890006EFD00200AB080BD0000000000408F40B7
:1018A00000606A4781B0009041F6E300C0F6000096
:1018B00001B0704783B002900191009202980199A3
:1018C00001600099416003B0704780B56F4682B0F7
:1018D000019001980090009801684068884702B024
:1018E00080BD80B56F4682B00190019900F002F88A
:1018F00002B080BD80B56F4682B001900091FFE7D5
:1019000003F059FC0A2021F06FFAF9E781B000904A
:1019100041F61D10C0F6000001B0704780B56F465B
:1019200082B00190019900F002F802B080BD80B54C
:101930006F4682B001900091FFE7FFE703F033FCB0
:1019400020B9FFE7012000F017F8F7E702F020F8D0
:10195000FFE703F02BFC28B1FFE703F00FFC01F0D9
:10196000E1F9FFE703F01FFC08B9FFE703E00A20F5
:1019700021F03AFAEDE7E0E780B56F4682B00190DA
:10198000019821F031FA02B080BD80B56F46FFF7B3
:10199000D5FCFFF7E3FC80BD80B56F4686B00590AF
:1019A0000598029000F01BF8029808300190FFF7AC
:1019B000CEFC0198029940F2D072C2F2000211608E
:1019C0006A460321116047F6FF12C0F602020021A9
:1019D0004FF4007300F012F8029806B080BD80B595
:1019E0006F4682B0019001980090043000F067F8D3
:1019F000009800F028FE009802B080BD80B56F46C8
:101A00008EB08446B868CDF830C00B910A92099325
:101A100007F8150C0C9804900DA8039000F05DF8E1
:101A2000082020F02BF801460398079100F055F8A4
:101A300001460B9A05A8FFF73DFFDDF810E0079976
:101A40000598069A4A600860079B0A99BDF8242009
:101A500017F8150CEC46CCF804E0CCF8000041F681
:101A6000CB00C0F6000020F0E1FE0EB080BD80B5D6
:101A70006F4684B0029001910298007BC00720B9A4
:101A8000FFE7012007F8010C15E0029948890130B1
:101A90004881029908894989884208DCFFE7029950
:101AA000002048810299086849688847FFE70120BB
:101AB00007F8010CFFE717F8010C04B080BD80B5F2
:101AC0006F4682B0019001980090012020F0B5F996
:101AD00001460098016002B080BD81B0009041F6DF
:101AE000EB20C0F6000001B0704780B56F4682B0B1
:101AF0000190019900F002F802B080BD80B56F46F8
:101B000084B00390029103F002F90190FFE740F2E4
:101B1000D070C2F200000090006841F66F21C0F65C
:101B20000001002200F008F8009800680830012148
:101B300001AA00F030F8EAE780B56F4688B0079058
:101B40000691059207980090043000F032F8009852
:101B50000021049100680490FFE7009904988842EE
:101B600013D0FFE704980290029810380190019872
:101B70000390069A03980599904708B9FFE704E097
:101B8000FFE7049800680490E7E70098043000F04D
:101B90001FF808B080BD80B56F4684B003900291F5
:101BA0000192FFE70198029920F04CFFFFE704B093
:101BB00080BD80B56F4682B00190019800684FF0FB
:101BC000FF3120F0AFFC002818BF012002B080BD1B
:101BD00080B56F4682B001900198006800231946D5
:101BE0001A4620F085F902B080BDB0B502AF0446B8
:101BF00008201FF043FF00210822054624F0E9FCDD
:101C0000281D00F020FD28462C60A565B0BDB0B5AC
:101C100002AF04461C201FF031FF00211C220546A4
:101C200024F0D7FC2846AC61B0BD80B56F4601F109
:101C30001402011D104600F008FD002080BDDDF8F3
:101C400000C002290171036007D0012909D00029D1
:101C50001CBF01207047029904E0C0E9022C00205B
:101C6000704701998260C0F80CC001610020704784
:101C7000F0B503AF2DE9000782B08A465AF8046F29
:101C8000564555D098469146044604E00120D8B305
:101C9000366856454CD056F8140C10B12168814274
:101CA000F4D116F8101C022922D0606801290FD047
:101CB0000029EBD156E9033221689D18A942E5D3EA
:101CC00056F8041C184424F05BFC0028DED10BE01D
:101CD00056F80C1C22680B1D9A42D7D3405856E97F
:101CE0000212401A9042D1D200200028D0D10BE03D
:101CF00056E903012268084482424FF0000038BFD1
:101D000001200028C4D100BF16F8100C022803D20D
:101D10007068D4E9002105E0BAD1616856E9033260
:101D2000706819444B46CDF8008000F0A6FBAFE781
:101D3000002002B0BDE80007F0BD47F6AE610246E4
:101D4000C0F602010020042300F056B800F012BED5
:101D5000F0B503AF2DE9000BD7F8089080461020AE
:101D60001C4615460E461FF089FE47F6117141F6D6
:101D700093520346C0E9004986604573C0F60201EC
:101D8000C0F60002404600F037F80020BDE8000B26
:101D9000F0BDF0B503AF4DF804BD40688D6806682E
:101DA000487B0C46022813D0012802D038B9207B8A
:101DB00028B9AE4203D1D4E9002128469047701BD0
:101DC000B0FA80F04109002021735DF804BBF0BD3A
:101DD000207B002818BFAE42F1D0ECE780B56F46FB
:101DE00082B09C461346019101A90422CDF800C09F
:101DF00000F043FB02B080BD82B0F0B503AF2DE927
:101E0000000782B004460D4607F10800C7E9022327
:101E100001900CB175B9A0E0019A104650F8041F6A
:101E2000019052F8080B019200F014FD0446002DB9
:101E300000F093802878002800F08F8049F2182A5B
:101E400047F60A286E1CC0F6020A4FF00009C0F6D9
:101E5000020804E016F8010B002800F07E800AEB6F
:101E600000014978024601F00301022908BF203A27
:101E7000012908BF0246A2F1410117294FF00000D5
:101E800000F26C80DFE801F01A6A1E0C22306A6AE8
:101E90006A6A3B496A6A6A6A6A6A51596A6A6A6125
:101EA0000198014651F8043F019150F8082B414632
:101EB00001900020009400F059F8CBE7204600F094
:101EC00034FDC7E760681FF0D9FD42E0019A104673
:101ED00050F8041F02F10C030190106892680193FE
:101EE000234600F006FEB5E70198011D0191016847
:101EF000216500F10801406801916065AAE7019A37
:101F0000104650F8041F93680190106802F10C0508
:101F10002246019500F0EDFD9CE70198011D01911D
:101F20000168204600F09DFD94E70198011D019194
:101F30000168204600F076FD8CE70198011D0191B3
:101F40000068214600F08DFD84E70198011D019194
:101F50000068206184F800907CE7204602B0BDE86C
:101F60000007BDE8F04002B07047000082B0F0B555
:101F700003AF4DF8048D82B00D46BA60FB6028B106
:101F80000021044600F03FFD2DB938E0002000F0AC
:101F900028FD04469DB3287807F10801019170B32C
:101FA00049F218260135C0F602064FF0040809E090
:101FB0000198011D01910068214600F033FD15F8DC
:101FC000010BE0B13118497801F00302022A014601
:101FD00008BF2039012A08BF01465429E8D0442906
:101FE0000CD184F800800198011D01910168E16025
:101FF00000F10801406801912061E0E700242046DB
:1020000002B05DF8048BBDE8F04002B070470000FC
:1020100082B0F0B503AF2DE9000784B0C7E9022311
:102020008246806D0D4607F10801039110B95046B4
:10203000FFF7DBFD287800286CD049F218286E1CC9
:10204000C0F602084FF0000923E000BF0398011D0D
:1020500003910068FFF7DBFD039905460B4653F833
:10206000042F01F1140003930B68D1E9034103909D
:10207000CDE9004128460121CDF80890FFF7DFFDAA
:10208000DAF858002946FFF7D0FD16F8010B0028B2
:1020900040D008EB0001497801F00302022A014612
:1020A00008BF2039012A08BF014644291CD0522903
:1020B000CCD04C2936D10398011D03910068FFF75D
:1020C000A6FD039905460B4653F8042F01F11000B5
:1020D00003930B68D1E902410094CDE90210284630
:1020E0000021CDF80490C9E70398011D0391006811
:1020F000FFF78DFD039905460B4653F8042F01F1B8
:102100000C0003930B6889680390CDE900192846F9
:102110000221B1E7002004B0BDE80007BDE8F040AF
:1021200002B070470120F6E7B0B502AF40F2D470BC
:1021300047F60D21C2F20000C0F60201512200F064
:10214000C0FB01200021032201241FF02BFE40F6DA
:102150003005C2F2000500210022002328601FF094
:10216000C7FE28680021002200231FF0C1FE40F6B0
:102170003401C2F2000100200C70B0BD40F2D470F6
:10218000C2F200007047F0B503AF2DE9000F87B031
:10219000914640F63402C2F200021278012A5FD161
:1021A00040F6300AC2F2000A0446DAF800000D4692
:1021B000D7F808B04FF0FF31984620F0B3F948F255
:1021C0002D7105EB4500C0F602010A18085C40F2CB
:1021D0004C01C2F2000151F82030507840F2280141
:1021E000C2F2000151F82000917840F20402C2F2DC
:1021F000000252F8211052688DE8130040F6860460
:1022000040F635060392C2F2000447F61422C2F2E9
:102210000006C0F602022046502186F85050CDF844
:1022200010B002F069FB07F10C0330465021224642
:10223000069301F083FD40F2D470C2F200003146F3
:1022400051224B46CDF8008000F017F9DAF8001063
:10225000044608460021002200231FF049FE00E04A
:102260000724204607B0BDE8000FF0BDF0B503AF6E
:102270002DE9000704460078042828D80E46DFE838
:1022800000F061032A2D3200E0689246806883B333
:102290000021002220F02EFA012832D1D4F80C803F
:1022A000B14659F80C0FD8F80410884209D8D8F86C
:1022B0005020002A53D0D8F85410484690470028A0
:1022C0004DD0E068002180681FF0E8FF3AE001206F
:1022D000BDE80007F0BD0120207333E0E0683169FC
:1022E00000F093F92EE0D4E9032106F10C009047A9
:1022F00028E0BAF1000F08D04FF0FF3120F012F9BA
:1023000008E00320BDE80007F0BD002120F00AF935
:10231000012817D1D4F80C80B14659F80C0FD8F821
:102320000410884207D8D8F850207AB1D8F8541051
:102330004846904750B1E0680021806800220023A1
:102340001FF0D6FD0020BDE80007F0BD404610F8A4
:102350000C1B69B14946082224F021FA11E04046DD
:1023600010F80C1B31B34946082224F018FA2AE071
:10237000D8F81000D6E9032124F011FAF068C8F863
:102380000C00D8F8581029B108F10C00524600236F
:10239000FFF76EFC464656F8485FB542CBD000BF0B
:1023A000281F414652460023FFF760FF2D68B542C3
:1023B000F6D1C0E7D8F81000D6E9032124F0EFF9F0
:1023C000F068C8F80C00D8F8581029B108F10C00D2
:1023D00052460123FFF74CFC464656F8485FB5428B
:1023E0003FF46FAF281F414652460123FFF73EFFDF
:1023F0002D68B542F6D164E7F0B503AF2DE90007CB
:102400000546884608686968884207D892462A6D5A
:1024100099463AB1696D4046904718B10120BDE830
:102420000007F0BD284610F80C1B21B141460822D8
:1024300024F0B5F907E02869D8E9002124F0AFF9C4
:10244000D8F80000E860A96D29B105F10C005246EA
:102450004B46FFF70DFC2C4654F8486FA64208D0B7
:10246000301F294652464B46FFF700FF3668A6420A
:10247000F6D10020BDE80007F0BDF0B503AF2DE9AF
:10248000000B82B0D7F80880044680681E4691464B
:10249000B8F1000F0D4606D00021002220F02AF9E5
:1024A00001280BD01DE026B14FF0FF3120F03AF8A3
:1024B00004E0002120F036F8012812D169462046B8
:1024C00032464346CDE90095FFF796FFA168B8F183
:1024D000000F044608464FF0000104D01FF0DEFE56
:1024E00005E0032403E0002200231FF001FD204645
:1024F00002B0BDE8000BF0BDB0B502AF044600204D
:1025000000F06FFA054600F036FB2046294600F041
:1025100089FA2846B0BDF0B503AF4DF804BD0546B5
:10252000007B60B1A868144680680E464AB100215D
:10253000002220F0DFF8012807D003241AE001244C
:1025400018E04FF0FF311FF0EDFF0020A96828735D
:10255000D1E90321304624F022F9A86800218068DF
:102560001CB100241FF09AFE04E000220023002486
:102570001FF0BEFC20465DF804BBF0BDD0B502AF35
:1025800040F6D60C0020C2F2000C00BF0CF8000090
:102590000130B0F5807FF9D14FF0000E8C2200BFE2
:1025A0001CF80E306FF00700194682EA5303CC077F
:1025B00008BF4B080130F7D30CF80E300EF1010EB6
:1025C000BEF5807F08BFD0BDEAE70000D0B502AFFE
:1025D00048F2203140F6D81C4FF0000ECEF6B8512C
:1025E000C2F2000C0823704681EA5002C40708BFFB
:1025F0004208013B1046F7D14CF82E000EF1010EB7
:10260000BEF5807F08BFD0BDECE7D0B502AF044671
:10261000007A00281CBF0520D0BD2068D4E904231F
:1026200002FB003024F0BBF8D4E90001E268431C4F
:102630000020934228BF03468B42236002BF012043
:1026400020720020D0BD006070470A6802600860F8
:102650007047006800F000B8B0B502AF0D46044600
:102660006CB100BF61682846FDF7CAFD002807D09D
:102670004FF00C0048BF08202458002CF2D1002451
:102680002046B0BDF0B503AF4DF8048D0026C1E97A
:1026900002660E61804600680D460121297060B116
:1026A000064668687168FDF7ABFD00284FF00C0026
:1026B00048BF082030580028F2D140462E6156B15C
:1026C00068687168FDF79CFDB0F1FF3FCCBF06F173
:1026D0000C0006F1080005602A694FF0000C002A82
:1026E00085F800C000F09180012105E02A461546DA
:1026F0001269002A00F089801078002840F0858057
:1027000013699E68B24207D00EB1307860B10126DD
:10271000002EEBD00FE000BFD86808B10678DEB31A
:102720000126002EE2D03EE0317000261D461170D9
:102730001E70002EDAD09668AE4202D010462A46AD
:1027400013E0F06844460028906018BF02611069E9
:102750003061106928B150F80C4F944218BF04380A
:10276000044628462660F2601661DE680170B06893
:1027700083F800C00028D86018BF03611869454677
:102780003061186928B150F8085F9D4218BF0430C5
:1027900005462E60B36036E000261D4601701170BC
:1027A0001E70002EA2D0D668AE4202D010462A4635
:1027B00013E0B06844460028D06018BF0261106979
:1027C0003061106928B150F8084F944218BF0430A6
:1027D000044628462660B26016619E680170F06863
:1027E00083F800C00028986018BF03611869454647
:1027F0003061186928B150F80C5F9D4218BF043849
:1028000005462E60F3601E6171E7D8F800100122C2
:1028100001200A705DF8048BF0BDD0B502AF012035
:10282000002103221FF0BEFA40F6DC54C2F200047D
:1028300000210022002320601FF05AFB20680021A5
:10284000002200231FF054FBFFF7C0FEFFF796FEA7
:102850000020D0BDF0B503AF4DF8048D06465C20D6
:1028600088461FF00BF900215C22044623F0B1FEDC
:1028700004F1140528463146192223F0C4FE012034
:10288000207004F14800A563C4F80480FFF7DBFE64
:1028900004F14C00FFF7D7FE0120002103221FF0B6
:1028A00081FA002100220023A0601FF021FBA06814
:1028B0000021002200231FF01BFB20465DF8048B43
:1028C000F0BDF0B503AF4DF8048D90460E460021E3
:1028D0005C22044623F07DFE04F1140528463146AF
:1028E000192223F090FE0120207004F14800A56316
:1028F000C4F80480FFF7A7FE04F14C00FFF7A3FE25
:102900000120002103221FF04DFA002100220023A4
:10291000A0601FF0EDFAA0680021002200231FF044
:10292000E7FA20465DF8048BF0BDB0B502AF04466F
:102930001430002100F01EF800281CBF0120B0BD9B
:1029400040F6DC55C2F2000528684FF0FF311FF059
:10295000E9FD40F6D85004F13401C2F20000FFF75F
:1029600091FE286800210022002300241FF0C0FAF5
:102970002046B0BDF0B503AF2DE9000B40F6DC59A1
:1029800040F6D8580D460446C2F20009C2F20008CB
:1029900005E000BF012020F027FA013DC5B1D9F8BC
:1029A00000004FF0FF311FF0BDFD40462146FFF70C
:1029B00050FED9F8001006460846002100220023E8
:1029C0001FF096FA46B9002DE4D10025002DE6D17E
:1029D0000020BDE8000BF0BDA6F13400BDE8000BFF
:1029E000F0BDB0B502AF044614201FF047F8002137
:1029F0001422054623F0EDFD002C1EBF0120287097
:102A0000EC602846B0BDB0B502AF0D4600211422DF
:102A1000044623F0DEFD002D1EBF01202070E5607E
:102A20002046B0BDF0B503AF4DF804BD40F6DC560E
:102A3000C2F20006054630680C468D604FF0FF314B
:102A40001FF070FD201D05F14801FFF7FEFD306805
:102A50000021002200231FF04BFA00205DF804BB88
:102A6000F0BDF0B503AF2DE9000B054614208846F4
:102A70001FF004F800211422064623F0AAFD40F6B8
:102A8000DC59B8F1000F1EBF01203070C6F80C8071
:102A9000C2F20009D9F800004FF0FF31B5601FF015
:102AA00041FD301D05F14801FFF7CFFDD9F80000C9
:102AB0000021002200231FF01BFA0C201EF0DEFF75
:102AC00004464660D9F800004FF0FF31A5601FF0C2
:102AD00029FD08F14C012046FFF7B7FDD9F80000A9
:102AE0000021002200231FF003FA0020BDE8000BA4
:102AF000F0BDF0B503AF2DE9000B16460C460021E2
:102B000014229846054623F064FD40F6DC59B8F1DE
:102B1000000F1EBF01202870C5F80C80C2F200090A
:102B2000D9F800004FF0FF31AE601FF0FBFC281D0C
:102B300006F14801FFF789FDD9F8000000210022C5
:102B400000231FF0D5F9D9F800004FF0FF31656080
:102B5000A6601FF0E7FC08F14C012046FFF775FD69
:102B6000D9F800000021002200231FF0C1F9002045
:102B7000BDE8000BF0BD01460220087000220020D5
:102B80000A737047D0B502AFFFF747FE0446FFF760
:102B9000CBFA2044C0B2D0BD83B0B0B502AF81B093
:102BA00040F6E055C2F20005844607F108002C1DEE
:102BB0000EC007F1080320464FF48071624600936F
:102BC00001F0BCF82D682046FDF792FB0146204637
:102BD000A84701B0BDE8B04003B0704783B0F0B57E
:102BE00003AF4DF804BD83B040F6E055C2F20005D6
:102BF000844607F108002C1D0EC007F1080320468B
:102C00004FF480716246029301F098F82A6848F206
:102C10003C70C0F60200062190472E682046FDF762
:102C200067FB01462046B047D5F82C0405F56071D6
:102C3000884212BF066847F6DC26C0F6020647F651
:102C4000BE2047F6522147F6D02247F6D523C0F6DC
:102C50000200C0F60201C0F60202C0F602030096AE
:102C6000FFF79AFF47F6551005F58271C0F602008E
:102C7000FFF792FF03B05DF804BBBDE8F04003B07E
:102C80007047D0B502AFD7E902EC002404770160A9
:102C9000C0E9023E80F810C04261D0BDB0B502AFBD
:102CA0000C46054618300831FFF7CFFC6C60B0BD0C
:102CB000B0B502AF40F6E055C2F200050446183048
:102CC00005F54271FFF7C1FC05F540706060B0BDCD
:102CD00080B56F4682B040F6E051C2F20001D1F8F3
:102CE0002C0401F56071884212BFD0F800C047F68D
:102CF000DC2CC0F6020C47F6BE2047F6522147F600
:102D0000D02247F6D523C0F60200C0F60201C0F675
:102D10000202C0F60203CDF800C0FFF73DFF02B08B
:102D200080BD0000F0B503AF2DE9000F85B00D2880
:102D300002D00A2840F0978040F6E055C2F2000524
:102D4000D5F82004D5F824142A680844C5F82004CE
:102D500047F60110C0F6020003219047D5F8200481
:102D600005F58278002408F80040B5F8DA024FF43F
:102D7000807200F0030105EB81110130A5F8DA0241
:102D800001F5EC704146A5F8D82223F0FBFCB5F81C
:102D9000DA02B5F8DC1200F00300A5F8DA02481CEC
:102DA00081B2D5F82004042928BF0421A5F8DC123B
:102DB00078B100BF0138291891F80421202A08D1E0
:102DC00001F58271C5F820040C70D5F820040028A4
:102DD000F0D105F2031100BF11F8010F2028FBD03C
:102DE000D5F82004002800F0EF8005F5A27B5846B6
:102DF0004022C5F8C4B123F006FC0020291D0022A2
:102E00004FF0000A07E000BF06B35FFA8AF3052B14
:102E100002F101021AD015FA82F393F84461202ED0
:102E2000F2D196B2741994F8454103F5A273202C9F
:102E30001870EAD00AF1010A8B195FFA8AF603F2D8
:102E4000411301EB8606C6F8C031DEE758462F2154
:102E500023F0F8FB10B3814619F8011F00291CBFAD
:102E6000002101701BE040F6E05AC2F2000A9AF815
:102E70002814002900F0D780022900F008810129D8
:102E800040F0CE8249F21822C0F602021044407887
:102E900010F0970F00F0C182481CBFE2D946D94517
:102EA000CDF80C8008D0584600F0EEFD002853D035
:102EB0000024CDF808B008E0D5F82C0405F54071E1
:102EC000441ACDF808B018BF012400F1080BD84609
:102ED00003E000BF0120002857D0D8F80080D84573
:102EE00010D098F804000128F4D0464656F8181D72
:102EF0004846FDF785F90028ECD10020049600280B
:102F0000EBD142E0CCB105F54278464602E000BF85
:102F10000120D0B3366846450FD030790128F7D06C
:102F2000344654F8181D4846FDF76AF90028EFD1D9
:102F3000002004940028EDD127E095F8441147F6CD
:102F40006C3047F65532C0F60200C0F60202002986
:102F500008BF104602990DE095F8441147F6343049
:102F600047F61832C0F60200C0F60202002908BF78
:102F700010465946FFF710FE2A6847F60110C0F6C2
:102F800002000321904700200490049888B1416911
:102F9000DDF80C8081B947F68830C0F60200FFF7F3
:102FA000FBFD2A6847F60110C0F602000321904796
:102FB00001E0DDF80C80002030B14369012151FAB5
:102FC0008AF105F5E2729847D5F82C0405F5607191
:102FD000884212BF066847F6DC26C0F6020647F6AE
:102FE000BE2047F6522147F6D02247F6D523C0F639
:102FF0000200C0F60201C0F60202C0F6020300960B
:10300000FFF7CAFD0023C5F82034C5F82434404634
:103010000021402285F8283405B0BDE8000FBDE846
:10302000F04023F0D6BA1A284BDC032800F0A58024
:10303000092840F077810AF2031100BF11F8010F4F
:103040002028FBD00AF5A275284623F09BFB2846D2
:10305000202123F0F7FA002818BF451C28462F210D
:1030600023F0F0FAAB4630B183461BF8011F00296C
:103070001CBF00210170AB4500F00681284600F01E
:1030800003FD002800F0CC81814601240FE1413886
:10309000032800F2C281DFE800F002A6BCD2BAF930
:1030A000D802BAF8DC2281B2B1F5807F40F0E1802D
:1030B000002A00F0E680BAF8DA02013800F00300D6
:1030C000A5E11B2800F0D3807F2840F02B81DAF89F
:1030D0002004002800F0A48147F69D30C0F60200CD
:1030E000FFF75AFDDAF8200400210138CAF820045D
:1030F000504480F80411DAF82404002800F090818C
:10310000002000BFDAF820144218524492F805213A
:103110005144014481F80421DAF824140130884232
:10312000F0D3DAF820040AF582740844002121540F
:1031300047F6A13048F60F0148F61302C0F6020028
:10314000C0F60201C0F60202FFF726FDDAF82004FD
:10315000DAF80020DAF824142044904747F6551096
:1031600048F61701C0F60200C0F6020105B0BDE83E
:10317000000FBDE8F040FFF70FBDDAF8002047F67A
:103180000110C0F60200032190470020CAF8200475
:10319000CAF82404DAF800208AF8280448F23C70BF
:1031A000C0F6020006219047DAF82C040AF5607197
:1031B000884212BF066847F6DC26C0F6020647F6CC
:1031C000BE2047F6522147F6D02247F6D523C0F657
:1031D0000200C0F60201C0F60202C0F60203009629
:1031E000FFF7DAFC1CE1BAF9D81288B204280DD036
:1031F000BAF8DC32BAF8DA22042BA2F1010240F06C
:10320000BC8002F00302904240F0C3804FF4807013
:10321000C5E0DAF82404002800F0FF80DAF8201472
:1032200001380131CAF82014CAF8240447F65510B1
:1032300048F60701C0F60200C0F6020114E0DAF811
:103240002004002800F0E980DAF824140138CAF8D4
:103250002004481CCAF8240447F6551048F60B0110
:10326000C0F60200C0F60201FFF796FCD5E001208F
:10327000D4E0042A40F08780BAF8DA12884240F09D
:10328000C0804FF48070C2E0DAF82C940AF54070E8
:103290009BF80020A9EB0001B1FA81F1B2FA82F3A8
:1032A00049095B09002A08BF814643EA010447F641
:1032B0001531C0F602015846FCF7A2FF88B347F665
:1032C0001631C0F602015846FCF79AFF48B358463B
:1032D0000494FDF70DF859F8085F80464D454FF00E
:1032E000000429D1DAF808530AF54279A5EB090060
:1032F000B0FA80F00499400908432FD0A0B200280A
:1033000000F08E80012840F08F80DAF830040168E8
:1033100011F80820002A40F0B380007F012840F017
:10332000AF802F2005B0BDE8000FBDE8F04000F0F1
:10333000BDB82D684D45D5D02E4656F8181D5846B7
:10334000424623F04EF90028F3D10134A1B23046B1
:1033500000F07AFCEDE72D684D45CFD02E4656F8AB
:10336000181D5846424623F03CF90028F3D1013499
:10337000A1B2304600F068FCEDE701308A4208BF98
:103380004FF480700BE0481E002908BF4FF4807096
:103390003DE0481C00EB907121F00301401A80B21F
:1033A000B0F5807F37D10020CAF82004CAF8240481
:1033B000DAF800208AF8280448F23C70C0F60200CF
:1033C00006219047DAF82C040AF56071884212BF92
:1033D000066847F6DC26C0F6020647F6BE2047F62A
:1033E000522147F6D02247F6D523C0F60200C0F698
:1033F0000201C0F60202C0F602030096FFF7CCFB02
:103400000BE0033000EB907121F00301401A80B211
:10341000B0F5807F01D000F0C6FB00208AF82804B8
:1034200005B0BDE8000FF0BDDAF8002047F6011046
:10343000BAF83444C0F6020003219047FFF748FC75
:1034400064B3DAF80020DAF820140AF582709047A5
:10345000BAF834041FFA88F18842E1D94FF0FF30FE
:1034600010FA88F4DAF83004006820444078FFF756
:1034700059FCBAF83404A11C01348142F2D3CFE7DD
:1034800011F808000028CBD041444C1EC0B200F017
:103490000DF8A07801340028F8D1C1E747F655109F
:1034A0000AF58271C0F6020060E60000B0B502AF16
:1034B00082B040F6E054C2F20004D4F82024D4F8DC
:1034C000241407F8090C0A443D2A45D861B100BF0D
:1034D000D4F820040A18224492F803212044084416
:1034E000013980F80421F3D12268A7F109000121F4
:1034F0009047D4F8200417F8091C204480F80411E0
:10350000D4F82014D4F824040131C4F8201418B3DA
:10351000084404F582750021295447F6A13048F685
:103520000F0148F61302C0F60200C0F60201C0F611
:103530000202FFF731FBD4F820042268D4F82414E7
:103540002844904747F6551048F61701C0F6020088
:10355000C0F60201FFF720FB02B0B0BD40F6E0521A
:10356000C2F20002136848F23C704FF0000CC0F643
:1035700002000621C2F820C4C2F824C482F828C47C
:103580001847F0B503AF2DE9000F81B040F6E054C5
:10359000C2F2000420604FF48070A4F8D80247F60D
:1035A000DE20C0F6020004F53A754FF0010AC4F8B7
:1035B000E002284684F8FCA204F53876FFF743F8C9
:1035C00047F6E020C0F6020004F54278C4F8000394
:1035D000404684F81CA304F54079FFF734F847F619
:1035E000E420C0F60200C4F8400304F5527084F8E9
:1035F0005CA3FFF728F847F6E820C0F60200C4F8FD
:10360000200304F54A7084F83CA3FFF71CF804F586
:103610005870009047F6EC20C0F6020004F55A7B83
:10362000C4F86003584684F87CA3FFF70CF847F60B
:10363000D020C0F60200C4F8800304F5627084F85C
:103640009CA304F5607AFEF7FEFF04F54670294658
:10365000FEF7FBFF04F54E702946C4F80463FEF73D
:10366000F4FF04F556702946C4F82463FEF7EDFF15
:1036700004F55E702946C4F84463FEF7E6FF04F5DE
:1036800066705946C4F86463FEF7DFFF00980025B2
:10369000C4F8840347F6F120C0F60200C4F8A00382
:1036A00043F26D70C0F60000C4F8B40304F56E7008
:1036B000414684F8BC53C4E9EA5584F8B053FEF798
:1036C000C4FF47F6A600C0F60200C4F8C00343F2E8
:1036D000AD70C0F60000C4F8D40304F5767041461E
:1036E000C4F8A49384F8DC53C4E9F25584F8D053A9
:1036F000FEF7ABFF47F6F520C0F60200C4F8E00382
:1037000043F6E100C0F60000C4F8F40304F57E704F
:103710004146C4F8C49384F8FC53C4E9FA5584F8CC
:10372000F053FEF792FF47F6F820C0F60200C4F807
:10373000000443F66310C0F60000C4F8140404F556
:1037400083604146C4F8E49384F81C54C4F80854D8
:10375000C4F80C5484F81054FEF777FFC4F80494AE
:10376000C4F82CA401B0BDE8000FF0BDD0B502AF85
:1037700040F6E054C2F20004D4F82C0404F5387189
:10378000884202D000F0B8FA06E0226847F6DE2050
:10379000C0F6020001219047226847F60110C0F6EA
:1037A0000200032190470020D0BD0000F0B503AF18
:1037B0002DE9000F83B0022908D0012929D140F654
:1037C000E050C2F20000D0F82C4423E050681546C7
:1037D00000F05AF90446E8B9696847F634300A78C7
:1037E00047F61833C0F60200C0F60203002A08BFED
:1037F0001846FFF7D1F940F6E050C2F20000026827
:1038000047F60110C0F60200032190474FF0FF3049
:1038100062E0002454F8086FA6425CD040F6E058FD
:1038200047F6011947F6014A47F6CE3BC2F20008B7
:10383000C0F60209C0F6020AC0F6020B19E000BF8A
:1038400056E9040256F8183C00284FF0720108BFF0
:103850002D21002A4FF07702504608BF2D22FFF796
:103860009BF9D8F800204846032190473668A642C5
:1038700031D0307950B10228E2D00128F1D156F888
:10388000181C5846FFF788F9EBE700BF56F8040C00
:1038900056F8102C00284FF0780108BF2D218AB16E
:1038A00016F8080C7723002856F8180C56F80C5C0C
:1038B00008BF2D23009047F6DB30C0F602007222CD
:1038C0000195CCE756F8182C56F80C3C47F6F33027
:1038D000C0F60200C3E7002003B0BDE8000FF0BD52
:1038E000D0B502AF02290BD0012916D140F6E05025
:1038F000C2F2000000F56071C0F82C140020D0BDA9
:103900005068144600F0C0F870B140F6E051C2F2C1
:103910000001C1F82C040020D0BD47F6A630C0F647
:103920000200FFF739F90EE0616847F634300A7893
:1039300047F61833C0F60200C0F60203002A08BF9B
:103940001846FFF729F940F6E050C2F2000002687D
:1039500047F60110C0F60200032190474FF0FF30F8
:10396000D0BD80B56F4640F6E050C2F200000021A5
:10397000C0F82014C0F82414026880F8281448F213
:103980004270C0F6020009219047002080BD00006F
:10399000F0B503AF4DF8048D82B040F6E058C2F2A6
:1039A00000080020C8F82004C8F82404D8F8002033
:1039B00088F8280448F24270C0F6020009219047B6
:1039C00048F24B7447F65515C0F602046FF03F06F7
:1039D000C0F6020506E000BF28462146FFF7DCF8E6
:1039E0007C2E0AD240367B2EF6D8D8F8002020460E
:1039F0004021904740347C2EF4D347F60114D8F888
:103A00000020C0F60204204603219047D8F8002089
:103A100047F6FE20C0F6020017219047D8F8002094
:103A2000204603219047D8F82C0408F5607188429D
:103A300012BF066847F6DC26C0F6020647F6BE202F
:103A400047F6522147F6D02247F6D523C0F60200AA
:103A5000C0F60201C0F60202C0F602030096FFF7AC
:103A60009BF802B05DF8048BF0BD40F6E050C2F266
:103A7000000000F54870704740F6E050C2F20000C8
:103A800000F5407070470000F0B503AF2DE9000F5E
:103A900083B00446FCF72CFC054640F6E050C2F229
:103AA0000000D0F82CA4002D78D021782F2907D140
:103AB000013D00F5387A71D00134691C09D16DE0FF
:103AC000691E625C2F2A02BF002262540D46691CE7
:103AD00064D04FF0000B00F538704FF000084FF045
:103AE00000090090019508E0019DF0074FF0000BE0
:103AF00052D0A84508F1010850D014F808002F282A
:103B000001D00028F5D104EB090647F61530C0F6C0
:103B10000200314604F808B0FCF772FB80B347F6A8
:103B20001630C0F602003146FCF76AFB70B30AF1AA
:103B3000080B08F101000026029002E00120002895
:103B4000D2D0DBF800B00AF108008345CCD09BF856
:103B500004000128F2D1ABF11805296804EB090033
:103B6000FCF74EFB0028E9D12F20DDF8089004F87F
:103B7000080001260020AA460028E2D1B4E700BFD1
:103B80000098824514BFDAF804A0824608F10109C2
:103B90002F2004F80800ACE74FF0000A504603B0AD
:103BA000BDE8000FF0BDF0B503AF4DF804BD82B025
:103BB00040F6E0560446C2F200060020C6F8200493
:103BC000C6F82404326886F8280448F23C70C0F62F
:103BD000020006219047D6F82C0406F56071884251
:103BE00012BF056847F6DC25C0F6020547F6BE2081
:103BF00047F6522147F6D02247F6D523C0F60200F9
:103C0000C0F60201C0F60202C0F602030095FEF7FC
:103C1000C3FF06EB8410A6F8D84200F5EC742046EA
:103C2000FCF766FB06F58275C6F820042846214697
:103C300022F0A8FD3268D6F82014284602B05DF8BC
:103C400004BBBDE8F0401047B0B502AF02290446FE
:103C50000BD0012925D140F6E050C2F2000000212E
:103C6000C0F83044A0F83414B0BD40F6E055C2F2BC
:103C700000052A6847F60110C0F6020003219047AC
:103C8000D5F83004016847F65510C0F60200FEF77B
:103C900083FFD5F830040068FCF72AFB0138A5F84B
:103CA0003404206840F6E0520021C2F2000209E02C
:103CB000A2F83414C2F83044B2F83434994201F115
:103CC000010109D2D2F830341B685D5C435C9D422F
:103CD000EED1002BF0D1EBE7126847F60110C0F6E9
:103CE000020003219047216847F65510C0F60200F4
:103CF000BDE8B040FEF750BFD0B502AF044640F675
:103D0000E050C2F2000000F53870844208BFD0BD18
:103D10006068002818BFFFF7EFFF216847F6CA3038
:103D2000C0F60200BDE8D040FEF736BF80B56F4652
:103D300000F091FF07F050FA002080BD80B56F467B
:103D400086B09C460023CDE90133CDE903330593CA
:103D500030B16FF00043994238BF0B460390059392
:103D600001A81146624600F003F806B080BD0000CD
:103D7000F0B503AF2DE9000F81B02DED0C8B9CB099
:103D80009FED218B9FED229B9FED23AB9FED24BBED
:103D90009FED25CB91460E4604464FF0250A354649
:103DA000013603E0A26850540136013516F8010CC3
:103DB000002800F06D8525280CD0D4E903124B1C97
:103DC0009142E360F0D22268002AEBD0616890470C
:103DD000EAE700BF3078002800F05A854FF0000B6A
:103DE0003178A1F12002102A30D80120DFE802F05A
:103DF000252E2E272E2E2E2E2E2E2E292E2B2E2EFB
:103E0000200000BF00BF00BFFFFFFFFFFFFFEFFF6D
:103E1000FFFFFFFFFFFFEF7F0000000065CDCD41FA
:103E20000000000065CDCDC1000000000000E03FB3
:103E30004BEA000B01360135D2E70820F8E71020E5
:103E4000F6E70420F4E70220F2E700BFA1F130001A
:103E5000092811D84FF0000815F8010F08EB880168
:103E60006A7800EB4100A2F130010A29A0F1300884
:103E7000F2D36E1C18E000BF2A2913D159F8040BA5
:103E80000028804648BFC0F10008002816F8010F3E
:103E900048BF4BF0020B38B9002000287FF47FAFF9
:103EA00000F0F6BC4FF0000830782E281CD13146C7
:103EB00011F8010F002858D0A0F13002092A4BF464
:103EC000006B2ED8701E0025827805EB8501C37823
:103ED00002EB4101A1F13005A3F130010A2900F103
:103EE0000100F1D3861C00E00025307868384FEAE5
:103EF0007000092850D8DFE800F00521294F4F4F06
:103F00003F4F4F48314611F8010F70B3682840F019
:103F10002A8116F8020F002800F045824BF0C00BF2
:103F20003AE02A2840F0BB8016F8021F59F8040B2B
:103F3000002900F0D98120EAE075D6E716F8010FD4
:103F4000002800F006814BF4806B25E0314611F823
:103F5000010F50B16C2840F00A8116F8020F0028BA
:103F600000F026824BF4C06B16E000200E460028BD
:103F70007FF415AF00F08CBC16F8010F50B900208B
:103F800000287FF40CAF00F083BC16F8010F002866
:103F900000F0E4804BF4007B3078A0F12501532938
:103FA00000F2F880DFE811F0E700F600F600F60016
:103FB000F600F600F600F600F600F600F600F60051
:103FC000F600F600F600F600F600F600F600F60041
:103FD000F600F600F600F600F600F600F600F60031
:103FE000F600F600F600F600F6005400F600F600C3
:103FF000F600F600F600F600F600F600F600F60011
:10400000F600F600F600F600F600F600F600800076
:10401000F600F600F600F600F600F600F600F600F0
:10402000F60080004C017E00F6005400F600F60019
:104030007E00F600F600F600F600F60080000401AF
:10404000F600F6001801F6008000F600F600800089
:10405000462809F1070020F0070090ED00DB1090E2
:104060005AEC1D9B484651464A46534608BF4BF002
:10407000200BFCF7E9FD002840F0038453EC182BDB
:1040800048465146FCF7B8FD002800F0F78047F697
:1040900021412046C0F60201042200F0D7BB0025D2
:1040A0000E4622E74BF4804BA0F15801202915D889
:1040B0001023DFE801F01813131313131313131352
:1040C00011131313131313131313131313171313BE
:1040D0001313131313131800022304E02BF0100B17
:1040E0000A2300E00823582808BF4BF0200B5FEAA2
:1040F0000B5048BF2BF0010B5FEA4B4006F1010665
:1041000014D45FEA4B5000F1DB815FEA8B502BF057
:104110000C0C00F1DF805FEA4B6000F12681D9F8DA
:1041200000105FEA0B6048BF89B220E15FEA4B50A4
:1041300000F1C6815FEA8B5000F1CF805FEA4B60EF
:1041400000F12081D9F800005FEA0B6148BF00B29E
:104150001AE1002000287FF422AE99E30020002815
:104160007FF41DAE94E34BF0800B0E4614E74BF446
:10417000007B0E4610E7D4E90301421C8842E2604E
:1041800080F09D812268002A00F03F81616825202F
:10419000904794E1D4E903124B1C9142E36080F014
:1041A0008E812268002A00F034816168904786E1A0
:1041B00059F8041B42F2010000294BEA000C00F000
:1041C000FC8000952046002210230A25CDF808C067
:1041D000019500F0B1FB72E159F8041B002900F0D1
:1041E000F68008784FF0000C002808468E460FD065
:1041F0002846002D08BF6FF000404142704600BFC6
:1042000010F8013F01314CF100020BB1002AF7D048
:10421000A0EB0E000BF40062A842294638BF01460D
:10422000002A08BF01461BF00200119040F01981DE
:10423000414580F01081F346A8EB010A10923CE062
:104240001BF0020A55D1B8F1020FC0F0CC80A8F1E2
:10425000010506E0A16820220A5400BF013D00F0DC
:10426000C480D4E90301421C8842E260F6D222688D
:10427000002AEFD0616820209047EFE7484653ECD2
:10428000192B5146FCF7D6FCA8B31BF0040047F6E7
:104290002641C0F6020147F62B404FF00402C0F65B
:1042A000020008BF014608BF0322CEE2A168202217
:1042B0000A54BAF1010A00F0D080D4E90301421C8B
:1042C0008842E260F5D22268002AEFD0616820209F
:1042D0009047EEE759F8041B4BE059F8040B0146F0
:1042E000002848BF414255E0002000287FF457AD28
:1042F000CEE201257BE053EC1A2B48465146FCF7F1
:1043000099FC002840F0A78253EC1B2B48465146ED
:10431000FCF772FC002840F09E825FEA0B50CDF85B
:1043200030A058BF0625122DC0F0EF80A5F1120E67
:10433000BEF11F0F28BF4FF01F0E0EF101014FF00D
:10434000000A302314A852460AF1010A5145835449
:10435000F9D16FEA0E000544AAF101001F284FF0C1
:10436000000038BF01200990D3E099F8001009F14E
:10437000040920460022CDE90058CDF808C000F01D
:10438000DBFA9DE099F900000146002848BF414250
:1043900009F10409C20F2046CDE90058CDF808B054
:1043A00000F0CAFA8CE0002000287FF4F8AC6FE23D
:1043B000002000287FF4F3AC6AE247F6174120465C
:1043C000C0F6020105220A23CDF800C008E047F636
:1043D00010412046C0F6020106224346CDF800B047
:1043E00000F08AFB6BE0022501E008F10105D4E949
:1043F000031259F8040B4B1C9142E3600ED2226861
:1044000052B16168C0B2904708E0A16801F800A00D
:1044100055E0A268505452E0A2685054BAF1000F1F
:104420004FF0250A4BD0454549D2A8EB050505E0DC
:10443000A16820220A5400BF013D40D0D4E9030105
:10444000421C8842E260F7D22268002AF0D06168FC
:1044500020209047F0E7013103E0109A08F10101B4
:10446000DE469EF800001091002D294618BF01215C
:1044700000281EBFB2FA82F24FEA521B51EA0B012A
:1044800023D111984FF0250A0028109817D04045E5
:1044900015D2A8EB000505E0A16820220A5400BF50
:1044A000013D0CD0D4E90301421C8842E260F7D2FE
:1044B0002268002AF0D0616820209047F0E701369A
:1044C000012000287FF46BACE2E10EF1010A013D0E
:1044D0000EE0A268505400BF1AF8010B013D4FF0E6
:1044E000000141F10001002818BF51EA0B01C8D0BA
:1044F000D4E903124B1C9142E360EDD22268002AFA
:10450000E7D06168C0B29047E6E7012009904FF01C
:10451000000A8DED12DB9DF84F0080F080008DF8D1
:104520004F000C9ADDE91201002A4CBF814611466A
:1045300048460B9122F0A6FFCDE90D01FCF7BCF82F
:104540000B460B9902464846CDF81090FBF72AFF20
:1045500048F62002C0F6020202EBC50292ED000B03
:1045600053EC102BCDE90723FCF7D4F881460A91D0
:1045700022F088FF11900F91FCF79EF80B460A99E4
:1045800002464846FBF70EFF53EC1C9B4A46CDE91A
:1045900005100A93FCF74EFBCDF80C9090B11198E2
:1045A0000F99013041F1000111908946FCF784F820
:1045B00002460B46DDE90701FCF728FBD0B9DDF820
:1045C00038C024E0DDE905100A9B4A46FCF70AFBE7
:1045D000D8B1DDF83C90119BDDF838C043EA090002
:1045E000B0FA80F04009184300F001001B1849F1AF
:1045F00000090DE00D98DDF838C001300D904CF148
:10460000000C00234FF0000902E0DDE90EC9119B08
:10461000F5B90D986146CDF83C90CDF838C0994673
:10462000FCF74AF802460B4604980B99FBF7BAFED2
:10463000039A0A9BFCF7E0FAB0FA80F00D99400962
:104640004B46DDE90EC9084009184CF1000C0D91EC
:10465000C5B35FEACB4028D55FEACB6025D4581EAE
:1046600079F1000021DB0135CDF838C011931846EF
:1046700049460A220023FCF783FC0A22A0FB02C35E
:1046800001EB810203EB4202119B013DB3EB0C03F2
:1046900069EB02021A43119B04BF89460346002AB4
:1046A000E4D008BF013DDDF838C041F2100000EA57
:1046B0000B00B0F5805F59D1581E79F1000055DA32
:1046C0000D9D11E00BF01000012181EA10100999F5
:1046D0000D9D81F0010108430DF1500904D12E20F8
:1046E00009F80A000AF1010ABAF11F0F23D8284677
:1046F00061460A220023E146FCF742FC00EB8002FF
:10470000A5EB42020A3D6FF0120369F1000EED1AAB
:104710004FF0FF357EEB050302F1300C0AF1010288
:1047200014AB03F80AC007D2BAF11F0F05468C4636
:104730009246DCD300E052460BF00300012813D16F
:10474000B8F1000F4FF0300314A93FD00C980028A7
:104750004FF0000048BF01201BF00C0518BF0125D9
:104760002843A8EB000833E014A93AE00998CDF8F3
:1047700038C0002844D01846CDF83C9049460A225B
:1047800099460023013DFCF7FBFB00EB8002A9EBFF
:1047900042020F9B3032B9F10A0C119263F1000210
:1047A0006FF01203BCEB03034FF0FF3372EB030314
:1047B000119A0AF1010E14AB03F80A2021D2BAF1C2
:1047C0001F0FF24603468946D5D31AE04FF0000882
:1047D0001F2A06D8424504D28B541E2A02F1010238
:1047E000F8D91F2A31D80C98002807D45FEA4B70FB
:1047F00028D45FEA0B7028D5202024E02D2022E069
:10480000D646BEF1200F4FF0000038BF0120BEF1A8
:104810001F0F2BD8DDF838C00DF150095DB3694288
:104820000D9D3023BEF11F0F4FF0000009F80E3030
:1048300038BF0120BEF11E0F0EF1010E1CD8013150
:10484000F0D119E02B208854013220464346CDF8A0
:1048500000B000F051F91098013600F1080901206C
:104860004FF0250A00287FF49AAA11E0DDE90D5CDB
:104870000DF1500900E00D9D0028F2467FF42FAFA6
:1048800032E747F61D412046C0F602010322DDE76C
:10489000206838B1E0681CB0BDEC0C8B01B0BDE8FD
:1048A000000FF0BD20690028F4D0A1680029F1D0E4
:1048B000E268824228BF421E00208854EAE782B0A4
:1048C00080B56F4686B0C7E9022307F108020023CE
:1048D0000092CDE90133CDE90333002805931EBFD3
:1048E00003906FF00040059001A8FFF741FA06B071
:1048F000BDE8804002B0704781B080B56F4687B098
:104900009446BB6007F1080200230192CDE902330F
:10491000CDE90433069330B16FF00043994238BFBC
:104920000B460490069302A86146FFF721FA07B0F0
:10493000BDE8804001B07047F0B503AF2DE9000736
:104940008AB0D7F810809C46E1B108F0200383F0CC
:10495000610303F1F60A00250DF1080EB1FBFCF628
:10496000534606FB1C1405F101090A2C38BF3023FD
:10497000234461450EF8053016D31F2D4D463146B0
:10498000ECD311E05FEA085107D430218DF808100C
:1049900028F010084FF0010906E04FF00009BCF1C3
:1049A000100F08BF28F01008D7E902135FEA8876D5
:1049B00023D463B15FEAC87605D018F00C0618BF9F
:1049C000012616439B1B5FEAC87604D115E000233D
:1049D0005FEAC87611D099450FD2B9F11F0F0CD8F4
:1049E00002AD30264C4600BF04F1010E9E452E5507
:1049F00004D21F2C7446F7D300E0CE468E450ED26B
:104A0000BEF11F0F0BD802AD302600BF05F80E60B7
:104A1000BEF11E0F0EF1010E98BF8E45F6D3CE45A6
:104A2000464688BF26F01006BCF1080F42F210047B
:104A300018BF4646264244D0340517D4BEF1000FB5
:104A400014D08E4518BF9E4510D1CE4588BFAEF11B
:104A5000010EBEF1000F1AD0BCF1100F02D0BCF154
:104A6000020F03D1CE4588BFAEF1010EBCF1100F8D
:104A700012D116F0200104D1BEF1200F01D278210D
:104A800011E049B1BEF1200F06D258210BE04FF0E2
:104A9000000EBCF1100FECD0BCF1020F08D1BEF13A
:104AA0001F0F05D8622102AD05F80E100EF1010EA0
:104AB000BEF11F0F05D802A9302501F80E500EF1E6
:104AC000010EBEF11F0F0ED80AB12D2106E07107AD
:104AD00003D4310707D5202100E02B2102AA02F8D8
:104AE0000E100EF1010E02A97246009600F004F8B5
:104AF0000AB0BDE80007F0BDF0B503AF2DE9000F27
:104B000081B00546B868D5F80C909B4616468007DC
:104B1000884618D15E4516D2ABEB06044FF0200A4A
:104B200004E0A96801F800A0013C0CD0D5E903011C
:104B3000421C8842EA60F7D22A68002AF1D06968EC
:104B400020209047F0E7B86800F0020A9EB1A8F173
:104B5000010403E0AA685054013E0CD0D5E90312C9
:104B6000A05D4B1C9142EB60F6D22A68002AF1D07E
:104B700069689047F0E7BAF1000F1AD0E868A0EB37
:104B80000901594515D2202407E0A9680C5400BF3B
:104B9000E868A0EB090159450BD22969421C8842FB
:104BA000EA60F5D22A68002AEFD069682020904791
:104BB000EEE701B0BDE8000FF0BD4EF61050CEF2AA
:104BC00000000268032922F00402026005D00129D6
:104BD00001D130BF704740BF20BF20BF704747F2B0
:104BE0000000C4F20000016841F0020101604EF6CD
:104BF0001050CEF20000016841F00401016030BFA6
:104C000070470000DFF834D003F032FD0C480D4946
:104C10000D4A002302E0D458C4501B1DC4188C4216
:104C2000F9D30A4A0A4C002301E01360121DA24284
:104C3000FBD321F067FDFFF779F8704700000220F1
:104C4000000000200803002034930208080300201D
:104C5000E0310020FEE780B56F4640F27000C2F2FE
:104C600000000021016000F0BDFA01F077FE02F0C3
:104C70001FFC02F0B6FB01F0D1FE01F009FF01F0CC
:104C800041FF01F063FF01F085FF01F0FDFF02F03D
:104C900037F902F09BF902F047FB02F03DFA01F010
:104CA000DFFF01F099FF01F0B9FF02F017F802F001
:104CB000C1F802F0D5FA02F019FB02F059FB02F03C
:104CC00003FA02F073FB42F25C00C2F2000000F053
:104CD00048FCBDE8804000F08CB980B56F4618F004
:104CE000D6F8002818BF012080BD80B56F4682B07D
:104CF0000021019101AB0021002218F051F9019827
:104D000002B080BD002318F04BB918F02BBA1EF08A
:104D100084BAF0B503AF4DF804BD1EF07EFA4EF232
:104D20001805CEF200052E6804461EF076FA2968B2
:104D3000844208BF314655F8043C4FF47A7251431F
:104D40000133B1FBF3F15043401A00F57A700021B2
:104D50005DF804BBF0BD006844F60001C4F2000138
:104D6000884210D041F20041C4F2010188420DD0C6
:104D700041F20001C4F20101884219BF042001215F
:104D80000120002104E00021002001E00220002198
:104D9000002918BF704741F2182100EBC000C2F291
:104DA000000101EBC00050F8081F09B14068084736
:104DB0007047006844F60001C4F20001884210D038
:104DC00041F20041C4F2010188420DD041F20001DC
:104DD000C4F20101884219BF0420012101200021F1
:104DE00004E00021002001E002200021002918BF7A
:104DF000704741F2182200EBC000C2F2000252F8E4
:104E0000301019B102EBC0004068084770470068D5
:104E100044F60001C4F20001884210D041F2004182
:104E2000C4F2010188420DD041F20001C4F2010137
:104E3000884219BF042001210120002104E0002143
:104E4000002001E002200021002918BF704741F234
:104E5000182100EBC000C2F2000101EBC00050F8C5
:104E6000181F09B1406808477047006844F6000100
:104E7000C4F20001884210D041F20041C4F20101A5
:104E800088420DD041F20001C4F20101884219BFED
:104E9000042001210120002104E00021002001E084
:104EA00002200021002918BF704741F2182100EBB1
:104EB000C000C2F2000101EBC00050F8101F09B1A0
:104EC000406808477047006844F60001C4F20001DA
:104ED000884210D041F20041C4F2010188420DD055
:104EE00041F20001C4F20101884219BF04200121EE
:104EF0000120002104E00021002001E00220002127
:104F0000002918BF704741F2182100EBC000C2F21F
:104F1000000101EBC00050F8201F09B140680847AC
:104F20007047006844F60001C4F20001884210D0C6
:104F300041F20041C4F2010188420DD041F200016A
:104F4000C4F20101884219BF04200121012000217F
:104F500004E00021002001E002200021002918BF08
:104F6000704741F2182100EBC000C2F2000101EBD2
:104F7000C00050F8381F09B140680847704781B039
:104F800001680868C00632D5002000900A680092C7
:104F90004A680092009A44F60002C4F2000291426C
:104FA00011D041F20040C4F2010081420ED041F222
:104FB0000000C4F20100814219BF04210120012137
:104FC000002030B113E0002118B110E002210020D0
:104FD00068B901EBC10041F21821C2F2000101EBF6
:104FE000C00050F8401F11B1406801B0084701B03F
:104FF000704780B56F4644F67F70C0F6000003F03E
:1050000031FB41F23870C2F200000068C16841F023
:105010001001C16080BD00EBC00C41F21820C2F24B
:10502000000000EBCC0000EBC10C40F83120002068
:10503000CCF804307047D0B502AF0446022807D838
:1050400048F6BC0160B2C0F6020151F8200000E051
:10505000002001F0C7F9022C84BF0120D0BD48F622
:10506000B00160B2C0F6020151F8200001680020D2
:105070004860D0BD80B56F464BB1022811D848F6C4
:10508000BC0340B2C0F6020353F820000AE0022835
:105090000DD848F6BC0340B2C0F6020353F8200016
:1050A00006E0002092B20A2300F042FF03E0002055
:1050B00092B201F067F8002818BF012080BD80B5CA
:1050C0006F464BB1022811D848F6BC0340B2C0F677
:1050D000020353F820000AE002280DD848F6BC036A
:1050E00040B2C0F6020353F8200006E0002092B25E
:1050F0000A2300F095FF03E0002092B201F003F9CB
:10510000002818BF012080BD48F6BC0140B2C0F69F
:10511000020151F82000C16B808D09684968401A6E
:1051200070470000F0B503AF4DF8048D0C46804683
:1051300010E000BF00204146324619F0B9FD0020C2
:1051400019F0D6FD0120B044A51B1DF04DFEB44260
:105150002C460FD3002019F012FE06468442E9D2F5
:1051600000204146224619F0A3FD002019F0C0FDA1
:105170002546ECE700205DF8048BF0BDD0B502AF0A
:1051800082B00024A7F109010020012207F8094C90
:1051900019F054FDC0B217F8091C012818BF2146A8
:1051A000C8B202B0D0BD002019F023BD002019F014
:1051B00037BD1CF078BB4FF0FF3000211AF084BBE4
:1051C00000201BF081BF022808BF704741F2F02287
:1051D000C2F2000252F8301019B102EBC000406870
:1051E0000847704780B56F4643F60040C4F202009E
:1051F000016841F400710160016841F4806101605F
:10520000016841F480710160032000F02FF8002054
:1052100003F0CEF802F072FA002080BD40F2740074
:1052200041F2F821C2F20000C2F2000100780A68DF
:1052300010440860704741F2F820C2F20000006894
:1052400070470000B0B502AF0446FFF7F4FF054613
:1052500040F27400C2F200000078611C18BF0444E0
:10526000FFF7E9FF401BA042FAD3B0BD4EF60C5148
:10527000CEF200010A684FF6FF031A4060F30A22DB
:1052800042F0806040F0FD7008607047D0B502AF1A
:105290004EF60C5CCEF2000CDCF80030C3F3022EAC
:1052A0008EF00704042C28BF0424BEF103034FF042
:1052B000FF3E0EFA04F438BF0023A14399400EFAD2
:1052C00003F39A43114300F1604200F00F03090118
:1052D00002F56442043B6344002848BF03F10C021A
:1052E0001170D0BD002848BF704700F01F01012297
:1052F00002FA01F14EF200124009CEF2000242F829
:1053000020107047002848BF704700F01F0101229D
:1053100002FA01F14EF280124009CEF2000242F888
:105320002010BFF34F8FBFF36F8F7047002804BF6B
:1053300001207047D0B502AF044690F83D0028B96F
:10534000002084F83C00204602F0AFFC022084F8E4
:105350003D002068211D00F017F8012084F8460068
:1053600084F83E0084F83F0084F8400084F841004F
:1053700084F8420084F8430084F8440084F845002F
:1053800084F83D000020D0BDD0B502AF40F6FF3E0E
:105390000368C4F2000E40F2004C7045C4F2010CE8
:1053A0000FDCB0F1804F19D040F20042C4F200028D
:1053B000904213D040F60002C4F2000290420DD099
:1053C00010E040F60042C4F20002904206D0604570
:1053D00004D00022C4F20102904203D14A6823F0B3
:1053E0007003134341F6FF72C4F2000290420DDCD9
:1053F00070451FDCB0F1804F41D040F20042C4F252
:10540000000290423BD040F6000221E043F6FF72DA
:10541000C4F20102904220DC42F20002C4F2000217
:1054200090422CD00022C4F20102904227D0604565
:1054300025D028E040F60042C4F2000290421ED07F
:1054400041F60002C4F20002904218D041F6004238
:10545000C4F20002904212D015E044F20002C4F2FD
:10546000010290420BD044F60002C4F201029042C5
:1054700005D044F20042C4F20102904203D1CA684E
:1054800023F44073134323F080024B69D1F800E00A
:105490008C681A430260C46240F48062C0F828E05D
:1054A000624504BF09690163012141610169C907BE
:1054B00008BFD0BD016921F001010161D0BD90F8A4
:1054C0003D1001291CBF01207047022180F83D10CA
:1054D000006841F2FF72C168C4F20002904241F0DC
:1054E0000101C1600DDC40F2FF71C4F2000188428D
:1054F00015DCB0F1804F29D040F20041C4F2000128
:1055000022E040F2FF31C4F20101884212DC41F690
:105510000001C4F20001884218D0002112E040F6D8
:105520000001C4F20001884210D040F60041C4F2EC
:10553000000109E044F20001C4F20101884205D0F3
:1055400040F20041C4F20101884204D1816801F0B7
:105550000701062903D0016841F001010160002024
:1055600070470146006841F21113C26822F001023F
:10557000C260026A1A4208D1026A40F244431A42E7
:1055800003D1026822F0010202600122002081F8AA
:105590003D207047002804BF01207047D0B502AFFE
:1055A000044690F83D0028B9002084F83C002046CD
:1055B00000F01EF8022084F83D002068211DFFF74E
:1055C000E3FE012084F8460084F83E0084F83F00A2
:1055D00084F8400084F8410084F8420084F84300D5
:1055E00084F8440084F8450084F83D000020D0BDD4
:1055F000704741B1082909D0042914BF00F14102C4
:1056000000F13F0204E000F13E0201E000F140023F
:105610001278012A1CBF01207047022241B10829DB
:1056200009D0042914BF80F8412080F83F2004E00D
:1056300080F83E2001E080F84020006801F01F0162
:105640000122036A02FA01F123EA01020262026AFC
:105650000A4341F2FF71C4F20001884202620BDC8E
:1056600040F2FF71C4F20001884213DCB0F1804FB8
:1056700045D040F2004115E040F2FF32C4F2010291
:10568000904214DC41F60003C4F20003984236D085
:10569000002314E040F60001C4F2000188422ED03D
:1056A00040F60041C4F20001884228D02CE044F2C8
:1056B0000003C4F20103984221D040F20043C4F237
:1056C0000103984220D1436C884243F40043436471
:1056D000C6DD904207DC41F60001C4F200018842B9
:1056E0000DD0002107E044F20001C4F2010188421C
:1056F00005D040F20041C4F20101884204D1816822
:1057000001F00701062903D0016841F001010160A1
:1057100000207047D0B502AF026801F01F0E4FF0B5
:10572000010C146A0CFA0EF324EA0303136240F22C
:105730000043D2F820C042F48064C4F201039C42CA
:10574000C2F820C00DD1136A41F21114234208D1CE
:10575000136A40F24444234203D1536C23F40043C0
:105760005364136A41F21114234204D1136A40F2C4
:105770004444234212D0082916D0042909D0002914
:105780004FF0010114BF80F8411080F83E10002056
:10579000D0BD012180F83F100020D0BD136823F058
:1057A000010313600829E8D1012180F8401000208E
:1057B000D0BDF0B503AF4DF804BD04460068C56820
:1057C0000669B10716D515F0020113D06FF002017A
:1057D0000161012121778069800703D0204600F014
:1057E00093F805E0204600F090F8204600F08EF88F
:1057F00000202077700718D515F0040015D0206818
:105800006FF00401016102212177806910F4407F6B
:1058100003D0204600F078F805E0204600F075F847
:10582000204600F073F800202077300717D515F0D8
:10583000080014D020686FF008010161042121776D
:10584000C069800703D0204600F05EF805E02046DE
:1058500000F05BF8204600F059F800202077F006B1
:1058600018D515F0100015D020686FF010010161F7
:1058700008212177C06910F4407F03D0204600F052
:1058800043F805E0204600F040F8204600F03EF8DE
:1058900000202077F00718BF15F0010002D1300674
:1058A00009D412E020686FF001010161204601F087
:1058B0000DFF300609D515F0800006D020686FF086
:1058C00080010161204600F08CFA700609D515F0C0
:1058D000400006D020686FF040010161204600F0D2
:1058E00016F8B0060DD515F020000AD021686FF02B
:1058F000200220460A615DF804BBBDE8F04000F0DC
:105900006FBA5DF804BBF0BD7047704770477047D1
:10591000F0B503AF2DE9000B90F83C30012B01D11D
:10592000022306E14FEAB2020123032A80F83C3049
:1059300000F2FC80DFE802F0024081C3036840F21D
:1059400000481C6A1A6A24F0020422F001021A625A
:105950001A46D3F804E052F818CF8E6843F48065F5
:10596000C4F20108454544EA060405D1CE6824F096
:105970000C0426F004063443D1F80090454507D1C5
:10598000D1E905562EF4407E45EA0E0545EA060E9D
:105990002CF0730646EA0906C3F804E09E614E68DF
:1059A00009695E631C629E6946F008069E619E69F5
:1059B00026F004069E61B5E0036840F200481C6AC8
:1059C0001A6A24F0200422F010021A621A46D3F850
:1059D00004C052F818EF8E6843F48065C4F20108E1
:1059E000454544EA061408D1CE6824F0C0096FF09A
:1059F000400404EA061444EA0904D1F8009045453D
:105A000007D1D1E905862CF4406546EA080645EA47
:105A1000860C2EF4E64646EA0926C3F804C09E61C9
:105A20004E6809699E631C629E6946F400669E6129
:105A30009E6926F480669E6173E0036840F2004828
:105A40001C6A1A6A24F4007422F480721A621A46DC
:105A5000D3F804C052F81CEF8E6843F48065C4F29A
:105A60000108454544EA062409D1CE6824F440697A
:105A7000360240F2FF4426EA040444EA0904D1F85D
:105A80000090454507D1D1E905862CF4405546EAFA
:105A9000080645EA061C2EF0730646EA0906C3F816
:105AA00004C0DE614E680969DE631C62DE6946F08F
:105AB0000806DE61DE6926F00406DE6132E0036876
:105AC00040F20046D3F820C01A6A43F4806522F4FD
:105AD00080521A621A465C6852F81CEFD1F80080B6
:105AE000D1F80890C4F20106B54204D14D6924F4FE
:105AF000804444EA85142EF4E64545EA08255C60B6
:105B0000DD612CF400564D6846EA093609691D64CA
:105B10001E62DE6946F40066DE61DE6926F4806698
:105B2000DE6109021368194300231160002180F827
:105B30003C101846BDE8000BF0BD80B56F4690F8EC
:105B40003C20012A4FF0020200F0C280012380F8BD
:105B50003C3080F83D20D0F800C04FF67772DCF87A
:105B6000083023EA0202CCF808200B684F2B28DC0F
:105B70001F2B43DD202B44D0302B42D0402B40F054
:105B8000A980D1F804E0C968DCF82030DCF82020D6
:105B900022F00102CCF82020DCF8182022F0F002DC
:105BA00042EA011123F00A0242EA0E02CCF8181070
:105BB000CCF82020DCF8081041F0470121F030013A
:105BC0007DE06F2B25DDB3F5005F46D0B3F5805F38
:105BD00077D0702B7ED1D1E901E3C968DCF80820C9
:105BE00043EA0E0322F47F4243EA01211143CCF839
:105BF0000810DCF8081041F0770160E00BB1102BC1
:105C000068D1DCF8081021F07001194341F0070158
:105C100055E0502B34D0602B5CD1D1F804E0C9683A
:105C2000DCF82030DCF8202022F01002CCF8202014
:105C3000DCF8182022F4704242EA013123F0A0027D
:105C400042EA0E12CCF81810CCF82020DCF808102C
:105C500041F0670121F0100131E0D1E901E3C968A9
:105C6000DCF8082043EA0E0322F47F4243EA0121D4
:105C70001143CCF80810DCF8081041F480411EE014
:105C8000D1F804E0C968DCF82030DCF8202022F0EC
:105C90000102CCF82020DCF8182022F0F00242EAC1
:105CA000011123F00A0242EA0E02CCF81810CCF8D7
:105CB0002020DCF8081041F0570121F02001CCF839
:105CC00008100022012180F83D10002180F83C10CE
:105CD000104680BD0122F5E7D0B502AF90F83C2018
:105CE000012A4FF0020252D0012380F83C3080F8A4
:105CF0003D200268D2F804E0D2F808C00C682EF00B
:105D00007003234341F2FF74C4F20004A2425360C3
:105D10000DDC40F2FF73C4F200039A4215DCB2F1CD
:105D2000804F29D040F20043C4F2000322E040F249
:105D3000FF33C4F201039A4212DC41F60003C4F2BD
:105D400000039A4218D0002312E040F60003C4F288
:105D500000039A4210D040F60043C4F2000309E069
:105D600044F20003C4F201039A4205D040F200431A
:105D7000C4F201039A4204D149682CF0800319430C
:105D800091600121002280F83D1080F83C201046EF
:105D9000D0BDB0B502AF90F83C20012A04BF02206C
:105DA000B0BD01F108053CCDD1E900CE23F47C5310
:105DB00022F470521A432EF4F0431A432CF4E043B9
:105DC0001A4324F4C0431A432A43C96922F4804287
:105DD000036811435964002180F83C100846B0BDA7
:105DE00070477047002804BF01207047D0B502AF4C
:105DF000044690F8410028B9002084F8400020466D
:105E000002F023F9242084F841002068C16821F4BD
:105E10000051C160204600F016F82068016921F4A5
:105E200090410161416921F02A014161C16841F459
:105E30000051C16000202021606484F8411084F882
:105E400042106063D0BDD0B502AF04460068D4E90B
:105E500002C22369016921F4405111430161626961
:105E600043EA0C01E3691143C268194349F20C6328
:105E70009A431143C1604169A26921F4407141F222
:105E80000043114340F48062C4F201039A4241612D
:105E900002D103F07BFF01E003F065FFE169636875
:105EA0001922B1F5004FA0FB020120D15A00DB0FEF
:105EB000FBF7B6F848F21F51C5F2EB11A0FB012326
:105EC0005A094FF69C73C0F6FF7303F1805302FB2F
:105ED0000300322303EBC000A0FB01014FF4F87074
:105EE00000EA111000EB0210C1F342111CE09A000D
:105EF0009B0FFBF795F848F21F51C5F2EB11A0FB81
:105F000001235A094FF69C73C0F6FF7302FB03008E
:105F1000322303EB0010A0FB0101F02000EA511036
:105F200000EB0210C1F34311084421688860D0BD22
:105F3000F0B503AF2DE90007044690F84100202892
:105F40001CD1884600294FF0010066D01646002A71
:105F500063D00020606421201D4684F84100FFF7D3
:105F60006AF9A684E684A1688246B1F5805F01D112
:105F7000206938B1C1464FF0000805E00220BDE8B5
:105F80000007F0BD4FF00009E08C48B36E1C0BE039
:105F9000B9F1000F1BD019F8010B21684860E08CA3
:105FA0000138E084E08CD8B1206800680006EFD4A6
:105FB000002EF9D0FFF73FF901464FF003004DB333
:105FC000A1EB0A01A94225D82068C068ECE738F89F
:105FD000020B21686FF35F2048604FF00009DEE795
:105FE00020680068400614D46E1C03E02068006836
:105FF00040060ED4002EF9D0FFF71DF901464FF0F0
:1060000003003DB1A1EB0A01A94203D82068C06892
:10601000ECE70020202184F84110BDE80007F0BD26
:10602000F0B503AF2DE9000782B0044690F84200B6
:10603000202861D1884600294FF0010000F09D80A2
:106040001646002A00F09980002022211D46606437
:1060500084F842102063FFF7EEF8A685E685A16874
:106060008246B1F5805F02D12069002846D0C14642
:106070004FF00008E08DE8B36E1C00BF2068006898
:10608000800615D4002EF9D0FFF7D5F80146002D73
:106090004FF003006ED0A1EB0A01A9426AD8206834
:1060A000C168490744BF01685FEA0171E6D528E08D
:1060B000B9F1000F0BD0A068B0F5805F10D008B91F
:1060C000206968B12068406800F07F000AE020681D
:1060D0004FF0000940686FF35F2028F8020B03E0DF
:1060E0002068406809F8010BE08D0138E085E08DFB
:1060F0000028C3D100203DE002203EE04FF000091F
:10610000B8E7002101910168019140680190019870
:1061100020680C3050E8000F216820F490700C319A
:1061200041E80002002AF3D12068143050E8000F43
:10613000216820F00100143141E80002002AF3D167
:10614000206B01280CD100BF20680C3050E8000FF4
:10615000216820F010000C3141E80002002AF3D140
:10616000202084F84200002008212063616484F824
:1061700040000320202184F8421002B0BDE800074F
:10618000F0BD0000B0B502AF044690F841002028F1
:106190001CBF0220B0BD4FF00100A1B3002A13467E
:1061A00008BFB0BD4FF0000C21202162A384E3841E
:1061B000C4F844C084F84100A06B46F2092E46F2B0
:1061C0004F252268C0F6000EC0F60005C0E90FE5B5
:1061D00046F25525C0F600050432C0E9135C02F012
:1061E0008CFF20686FF04001016000BF2068143010
:1061F00050E8000F216840F08000143141E80002AF
:10620000002AF3D10020B0BD0168806B0968C90580
:1062100048BFFEF7A0BD0021C18400BF0168143152
:1062200051E8001F026821F08001143242E8001397
:10623000002BF3D101680C3151E8001F026841F0D6
:1062400040010C3242E80013002BF3D17047806B01
:10625000FEF7AFBD806B0168496990F84120212AA3
:1062600013D111F0800110D00021C18401680C31DC
:1062700051E8001F026821F0C0010C3242E800130F
:10628000002BF3D1202180F841100168496990F872
:106290004220222A31D111F040012ED00021C185A7
:1062A00001680C3151E8001F026821F490710C3232
:1062B00042E80013002BF3D10168143151E8001FAC
:1062C000026821F00101143242E80013002BF3D1DF
:1062D000016B01290CD100BF01680C3151E8001F8E
:1062E000026821F010010C3242E80013002BF3D1B8
:1062F000202180F8421000210163416C41F010011F
:106300004164FEF7E0BDD0B502AF90F84230202BDB
:106310001CBF0220D0BD00294FF0010418BF002A85
:1063200001D12046D0BD0024046300F003F82046CC
:10633000D0BD0000F0B503AF4DF804BD82B01346E8
:1063400000260446816283854664222084F8420048
:106350000A462168E06B46F6B50C46F6451E46F245
:106360005525C0F6000CC0F6000EC0F6000504313D
:10637000C0E90FCEC0E9135602F0BFFE01962068B7
:1063800001680191406801900198206960B100BFE7
:1063900020680C3050E8000F216840F480700C3108
:1063A00041E80002002AF3D12068143050E8000FC1
:1063B000216840F00100143141E80002002AF3D1C5
:1063C0002068143050E8000F216840F0400014317C
:1063D00041E80002002AF3D1002002B05DF804BBBE
:1063E000F0BD0000D0B502AF044600BF20680C30FD
:1063F00050E8000F216820F490700C3141E8000251
:10640000002AF3D12068143050E8000F216820F0F2
:106410000100143141E80002002AF3D1206B012869
:106420000CD100BF20680C3050E8000F216820F02C
:1064300010000C3141E80002002AF3D120684069C5
:1064400040061AD52068143050E8000F216820F06B
:106450004000143141E80002002AF3D1E06B60B142
:1064600046F29141C0F60001016502F0DFFE68B11D
:10647000E06B016D88470020D0BD00202021E08521
:1064800084F8421020632046FEF74BFD0020D0BD6B
:10649000806B00212022C18580F842200163FEF735
:1064A00040BD0000B0B502AF82B00446006801688C
:1064B000C368426901F02F05202D03F0200506D1A5
:1064C0002DB1204602B0BDE8B04000F089B95FEAC6
:1064D000017C1EBF02F0010E03F4907212EB0E025B
:1064E00053D1226B012A05D111F0100218BF13F00D
:1064F000100236D10A0622D513F080021FD094F87C
:10650000411021293FD1A168B1F5805F03D12169F4
:10651000002900F05C81216A4A1C226209784160EE
:10652000E18C01390A04E1842DD1C16821F0800198
:10653000C160C16841F04001C16002B0B0BD490610
:1065400021D513F040011ED0C16821F04001C16087
:106550002021204684F8411002B0BDE8B040FEF78B
:10656000FABB0021019101680191416801910199F3
:106570004069400611D4A08DE18DE28D002A18BF3C
:10658000884240F0F08002B0B0BDC80718BF13F4D5
:10659000807052D1480756D45CE0E06B01684968CE
:1065A0008AB2002AEFD0A38D9A42ECD2E185C0696D
:1065B000B0F5807F39D000BF20680C3050E8000F64
:1065C000216820F480700C3141E80002002AF3D1E8
:1065D0002068143050E8000F216820F001001431C9
:1065E00041E80002002AF3D12068143050E8000F7F
:1065F000216820F04000143141E80002002AF3D164
:10660000202084F842000020206300BF20680C3066
:1066100050E8000F216820F010000C3141E8000222
:10662000002AF3D1E06B02F0BDFD02206063A08D73
:10663000E18D401A81B22046C4E0606C40F0010058
:106640006064480706D5BEF1000F03D0606C40F0CF
:1066500002006064880706D5BEF1000F03D0606CAD
:1066600040F004006064BCF1000F09D545EA0E005B
:10667000B0FA80F0400903D1606C40F0080060641B
:10668000606C00283FF47FAF11F0200018BF002D90
:1066900002D0204600F0A4F820684069616C00F048
:1066A000400001F00801401850D000BF20680C30B5
:1066B00050E8000F216820F490700C3141E800028E
:1066C000002AF3D12068143050E8000F216820F030
:1066D0000100143141E80002002AF3D1206B0128A7
:1066E0000CD100BF20680C3050E8000F216820F06A
:1066F00010000C3141E80002002AF3D1202084F878
:1067000042000020206320684069400625D500BF74
:106710002068143050E8000F216820F04000143148
:1067200041E80002002AF3D1E06BB0B146F6A701C0
:10673000C0F60001016502F079FD00283FF423AFA7
:10674000E06B016D02B0BDE8B04008472046FEF79F
:10675000BAFB0020606402B0B0BD204602B0BDE8C4
:10676000B040FEF7B0BB401A21680C3151E8001F61
:10677000226821F490710C3242E80013002BF3D10F
:106780002168143151E8001F226821F00101143200
:1067900042E80013002BF3D1202184F8421000219D
:1067A000216300BF21680C3151E8001F226821F0ED
:1067B00010010C3242E80013002BF3D1022281B207
:1067C0002046626302B0BDE8B04000F072B8216AB2
:1067D00031F8022B6FF35F2242602162A0E60000D5
:1067E00081B090F8421022291DD18268B2F5805FF5
:1067F00002D1016900294AD0816AB2F5805F07D0D1
:106800000AB9026922B10268526802F07F0201E00F
:10681000026852680A70816A01318162C18D013952
:106820000A04C18501D001B070470168CA6822F02E
:106830002002CA60CA6822F48072CA604A6922F0E3
:1068400001024A61202180F8421000214163026B5D
:10685000012A25D1016300BF01680C3151E8001FF6
:10686000026821F010010C3242E80013002BF3D132
:1068700001680A68D20606D5002200920A680092D2
:10688000496800910099818D01B000F012B801684B
:10689000826A49686FF35F2122F8021B8262BDE7BA
:1068A00001B0FEF7B4BA806B0021C185C184FEF748
:1068B0000ABB70470168806B0968C90538D400219C
:1068C000C18500BF01680C3151E8001F026821F446
:1068D00080710C3242E80013002BF3D101681431AF
:1068E00051E8001F026821F00101143242E8001350
:1068F000002BF3D10168143151E8001F026821F028
:106900004001143242E80013002BF3D1202180F81B
:106910004210016B01290BD101680C3151E8001FB5
:10692000026821F010010C3242E80013002BF3D171
:1069300000214163016B012918BFFEF768BA818D00
:10694000FFF7B7BF806B01214163016B012918BFBD
:10695000FEF78BBA818D4908FFF7ABBFF0B503AFE7
:106960004DF804BD92B006AC204630211FF014FF54
:10697000002543F640000595CDE90355CDE90155C5
:106980000095C4F202000168022641F080510160C6
:10699000006800F080500090009847F200000095D9
:1069A000C4F20000016841F480410160006800F415
:1069B000804000900098092006904FF480300790A6
:1069C00001200B904FF480000D9006200E90A8201F
:1069D000CDE90F060720119020460C9602F02CFFFF
:1069E00008B172B6FEE70F20CDE901064FF4A050C2
:1069F00004904FF48050059001A80521039503F001
:106A0000D1F810B172B600BFFEE712B05DF804BB5A
:106A1000F0BD000072B600BFFEE70000B0B502AFE7
:106A200084B041F2FC2042F2000101230024C2F2B2
:106A30000000C4F20101C0F600730125CDE9024453
:106A4000CDE900444FF40032047680F82040C0E9DC
:106A50000A34C56180F8304080E81600C0E903447C
:106A6000456101F00EFE10B172B600BFFEE71020C6
:106A7000CDE9000541F2FC20C2F200006946029413
:106A800001F0A6FE08B172B6FEE704B0B0BD00008A
:106A9000B0B502AF84B041F2443042F2002101238C
:106AA0000024C2F20000C4F20101C0F60073012507
:106AB000CDE90244CDE900444FF40032047680F879
:106AC0002040C0E90A34C56180F8304080E81600F3
:106AD000C0E90344456101F0D4FD10B172B600BFB6
:106AE000FEE70820CDE9000541F24430C2F2000083
:106AF0006946029401F06CFE08B172B6FEE704B07C
:106B0000B0BD0000D0B502AF41F28C3046F200417A
:106B1000C2F20000C4F2000140F20014032200237C
:106B2000C0F2011480E80E0000F10C014FF4A02C1B
:106B30004FF4C00E81E808508461838301F0D2FED7
:106B4000002808BFD0BD72B6FEE70000D0B502AF86
:106B500041F2B43046F60001C2F20000C4F2000176
:106B600040F2001403220023C0F2011480E80E005A
:106B700000F10C014FF4A02C4FF4C00E81E8085036
:106B80008461838301F0AEFE002808BFD0BD72B6D9
:106B9000FEE7000080B56F4641F2DC3045F200416F
:106BA000C2F20000C4F2000141F6802200234FF43B
:106BB000804CC0F2060280E80E00C0E9033CC0E948
:106BC0000533C0E9073302F0F9FC002808BF80BD97
:106BD00072B600BFFEE7000080B56F4641F230405C
:106BE00045F60001C2F20000C4F2000141F6802225
:106BF00000234FF4804CC0F2060280E80E00C0E98A
:106C0000033CC0E90533C0E9073302F0D7FC002894
:106C100008BF80BD72B600BFFEE7000080B56F46BA
:106C200041F2844045F60041C2F20000C4F2000186
:106C300041F6802200234FF4804CC0F2060280E827
:106C40000E00C0E9033CC0E90533C0E9073302F098
:106C5000B5FC002808BF80BD72B600BFFEE700008B
:106C600080B56F4641F2D84040F60001C2F2000004
:106C7000C5F20601016003F0BBF8002808BF80BD23
:106C800072B600BFFEE70000B0B502AF41F2E840C7
:106C900043F20001C2F20000C4F201014FF482721B
:106CA000002380E80E0000F10C014FF0020C4FF0C1
:106CB000010E4FF40074182581E808500A21C0E93C
:106CC0000645C0E90833C0E90A3103F0ABF80028F3
:106CD00008BFB0BD72B600BFFEE70000D0B502AF7E
:106CE00096B041F2405000220021C2F20000C4F2EE
:106CF0000102A72344F61F641591CDE91311CDE9D4
:106D00001111CDE90F11CDE90D11CDE90B11CDE92F
:106D10000911CDE90711CDE90511CDE90311CDE93F
:106D20000111C0E90023C0E90214C0E90411816126
:106D3000FEF7FCFA08B172B6FEE74FF480501290ED
:106D400041F24050C2F2000012A9FEF7F6FE10B167
:106D500072B600BFFEE741F24050C2F20000FEF7FB
:106D600019FC10B172B600BFFEE741F2405000249A
:106D7000C2F2000010A9CDE91044FEF7ADFF10B13A
:106D800072B600BFFEE76020CDE9090441F2405031
:106D9000C2F2000009A90022CDE90B44CDE90D445F
:106DA0000F94FEF7B5FD10B172B600BFFEE741F2D9
:106DB0004050C2F2000009A90422FEF7A9FD10B15B
:106DC00072B600BFFEE741F24050C2F2000009A9CE
:106DD0000822FEF79DFD10B172B600BFFEE74FF42A
:106DE0007A700A9041F24050C2F2000009A90C22C8
:106DF000FEF78EFD08B172B6FEE70020CDE9010076
:106E0000CDE9030005904FF40051089041F2405045
:106E10000691C2F2000001A9FEF7BBFF08B172B6ED
:106E2000FEE741F24050C2F2000000F0F1FF16B060
:106E3000D0BD0000D0B502AF8EB041F2885040F214
:106E400000420021C2F20000C4F20002A7234FF664
:106E5000FF740D91CDE90B11CDE90911CDE90711B1
:106E6000CDE90511CDE90311CDE90111C0E90023F8
:106E7000C0E9021401618161FEF758FA08B172B6E7
:106E8000FEE74FF480500A9041F28850C2F20000B1
:106E90000AA9FEF752FE10B172B600BFFEE741F23A
:106EA0008850C2F20000FEF775FB10B172B600BF49
:106EB000FEE741F288500024C2F2000008A9CDE9A3
:106EC0000844FEF709FF10B172B600BFFEE760206C
:106ED000CDE9010441F28850C2F2000001A9082264
:106EE00003940594FEF714FD08B172B6FEE741F273
:106EF0008850C2F2000000F08BFF0EB0D0BD000041
:106F0000D0B502AF8EB041F2D05040F60002002161
:106F1000C2F20000C4F20002A7234FF6FF740D91E5
:106F2000CDE90B11CDE90911CDE90711CDE9051125
:106F3000CDE90311CDE90111C0E90023C0E9021434
:106F400001618161FEF7F2F908B172B6FEE74FF414
:106F500080500A9041F2D050C2F200000AA9FEF718
:106F6000ECFD10B172B600BFFEE741F2D050C2F2A4
:106F70000000FEF70FFB10B172B600BFFEE741F252
:106F8000D0500024C2F2000008A9CDE90844FEF761
:106F9000A3FE10B172B600BFFEE76020CDE9010488
:106FA00041F2D050C2F2000001A9082203940594D6
:106FB000FEF7AEFC08B172B6FEE741F2D050C2F265
:106FC000000000F025FF0EB0D0BD0000D0B502AF2C
:106FD0008EB041F2186040F600420021C2F200007B
:106FE000C4F20002A7234FF6FF740D91CDE90B11F7
:106FF000CDE90911CDE90711CDE90511CDE903115D
:10700000CDE90111C0E90023C0E9021401618161E9
:10701000FEF78CF908B172B6FEE74FF480500A9083
:1070200041F21860C2F200000AA9FEF786FD10B115
:1070300072B600BFFEE741F21860C2F20000FEF730
:10704000A9FA10B172B600BFFEE741F21860002441
:10705000C2F2000008A9CDE90844FEF73DFE10B1D8
:1070600072B600BFFEE76020CDE9010441F218606E
:10707000C2F2000001A9002203940594FEF748FC27
:1070800008B172B6FEE741F21860C2F2000001A931
:107090000422FEF73DFC10B172B600BFFEE741F2DC
:1070A0001860C2F2000001A90822FEF731FC10B1FD
:1070B00072B600BFFEE741F21860C2F2000000F0B5
:1070C000A7FE0EB0D0BD0000D0B502AF82B041F235
:1070D000606041F200410024C2F20000C4F20001ED
:1070E0000923CDE90044A72280E81600C36084612B
:1070F000FEF71CF908B172B6FEE741F26060C2F219
:1071000000006946CDE90044FEF7E6FD08B172B61D
:10711000FEE702B0D0BD0000D0B502AF96B041F29C
:10712000A86040F200420021C2F20000C4F2010255
:10713000A72344F61F641591CDE91311CDE9111170
:10714000CDE90F11CDE90D11CDE90B11CDE90911F3
:10715000CDE90711CDE90511CDE90311CDE9011103
:10716000C0E90023C0E90214C0E904118161FEF7FF
:10717000DDF810B172B600BFFEE74FF480501290F8
:1071800041F2A860C2F2000012A9FEF7D6FC10B1CD
:1071900072B600BFFEE741F2A860C2F20000FEF73F
:1071A000F9F910B172B600BFFEE741F2A860002401
:1071B000C2F2000010A9CDE91044FEF78DFD10B118
:1071C00072B600BFFEE7602009904FF47A70CDE9F7
:1071D0000A0441F2A860C2F2000009A90022CDE928
:1071E0000C44CDE90E44FEF793FB10B172B600BF1C
:1071F000FEE741F2A860C2F2000009A90422FEF7EE
:1072000087FB10B172B600BFFEE741F2A860002410
:10721000C2F2000009A908220A94FEF779FB10B116
:1072200072B600BFFEE74FF40050069041F2A8602E
:10723000C2F2000001A9CDE90144CDE9034405945F
:107240000894FEF7A6FD10B172B600BFFEE741F24A
:10725000A860C2F2000000F0DBFD16B0D0BD000057
:1072600080B56F4688B041F2F06044F200420021E0
:10727000C2F20000C4F20102A72341F2873C079149
:10728000CDE90511CDE90311CDE90111C0E90023D4
:10729000C0E9021C01618161FEF748F808B172B6CD
:1072A000FEE741F2F060C2F20000FEF773F910B1A0
:1072B00072B600BFFEE7602001900020CDE9020019
:1072C000059041F2F060C2F2000001A90022FEF731
:1072D0001FFB10B172B600BFFEE741F2F060C2F2D0
:1072E000000000F095FD08B080BD000080B56F463D
:1072F00041F2387041F20001C2F20000C4F2010113
:1073000000234FF00C0C4FF4E13280E80E00C0E98E
:107310000333C0E905C3C361FEF764FD002808BF5D
:1073200080BD72B6FEE70000D0B502AF41F28070BA
:1073300044F6000C48F2A062C2F20000C4F2000C55
:10734000C0F201024FF4805300214FF4806E0424F8
:10735000C0E900C2C0E90231C0E904E4C0E9061195
:10736000FEF740FD002808BFD0BD72B6FEE7000062
:1073700080B56F4641F2C87041F20041C2F2000090
:10738000C4F2010100234FF00C0C4FF4E12280E81D
:107390000E00C0E90333C0E905C3C361FEF722FD57
:1073A000002808BF80BD72B6FEE7000080B56F46BA
:1073B00041F61000C2F200004FF0A041016004212C
:1073C00001714FF40071C18002214172002141819D
:1073D0000173C18102F0C4F9002808BF80BD72B6F4
:1073E000FEE780B56F4682B0002043F63001019081
:1073F000C4F202010A6842F480020A600A6802F4D8
:1074000080020192019A00900868002240F4001066
:1074100008600868052100F40010009000980C2016
:10742000FDF734FF0C20FDF75DFF0D200521002244
:10743000FDF72CFF0D20FDF755FF2F200521002221
:10744000FDF724FF2F20FDF74DFF382005210022F6
:10745000FDF71CFF3820FDF745FF3A2005210022EB
:10746000FDF714FF3A20FDF73DFF3B2005210022E8
:10747000FDF70CFF3B20FDF735FF442005210022DE
:10748000FDF704FF4420FDF72DFF452005210022D4
:10749000FDF7FCFE4520FDF725FF462005210022D3
:1074A000FDF7F4FE462002B0BDE88040FDF71ABFAC
:1074B000F0B503AF2DE9000F87B0002643F630008A
:1074C0000696CDE90466CDE902660196C4F2020093
:1074D000016840F2004841F0020101600168C4F215
:1074E000020801F00201019101990196016808F575
:1074F000A05441F0400101600168002201F0400108
:1075000001910199019601684FF0400A41F0010193
:107510000160016801F00101019101990196016882
:1075200041F008010160016801F008010191019931
:107530000196016841F004010160016801F0040155
:10754000019101990196016841F48071016001681F
:1075500001F48071019101990196016841F02001C7
:107560000160016801F02001019101990196016813
:1075700041F080010160016801F0800101910199F1
:107580000196016841F0100101600068402100F09F
:10759000100001900198204602F000F8A8F58069DB
:1075A000484610210122012501F0F8FF40464FF422
:1075B0008051002201F0F2FF40460121012201F03A
:1075C000EDFFCDE902A50DF1080A20465146CDE9AF
:1075D000045501F00BFF082002904FF4041B2046D5
:1075E0005146CDE903B501F001FF072008F580649D
:1075F000CDE9020620465146049601F0F7FE4846C2
:107600005146CDE9025B049501F0F0FE1020CDE972
:10761000020548465146CDE9045501F0E7FE302009
:10762000CDE9020B20465146049501F0DFFE4FF4F0
:10763000805002A961C140465146059601F0D6FE30
:1076400040465146CDE90255CDE9045501F0CEFE44
:107650004FF4404002900220CDE90305032005903D
:10766000052006904046514601F0C0FE0620052147
:107670000022FDF70BFE0620FDF734FE0920052150
:107680000022FDF703FE0920FDF72CFE0A2005214C
:107690000022FDF7FBFD0A20FDF724FE172005213F
:1076A0000022FDF7F3FD1720FDF71CFE07B0BDE833
:1076B000000FF0BD41F6F44141F26060C2F20001FA
:1076C0000022C2F200000A60FDF7F9BE006841F234
:1076D0000001C4F2000188420ED041F20041C4F220
:1076E0000001884218BF704741F6F440C2F2000022
:1076F0000168013101607047FDF790BD82B0002044
:1077000043F640010190C4F202014A6842F480420B
:107710004A604A6802F480420192019A0090086827
:10772000002240F08050086008680F2100F080506F
:10773000009000986FF0010002B0FDF7A7BD80B582
:107740006F4686B0006842F20022C4F201020021B6
:107750009042CDE90411CDE90211019116D042F217
:107760000001C4F20101884238D10020009043F6A4
:107770004400C4F20200016841F4807101600068B5
:1077800000F480700090009806B080BD43F644007D
:107790000091C4F20200026842F480620260026852
:1077A00002F480620092009A009150F8142C42F08A
:1077B000200240F8142C50F8140C00F02000009027
:1077C00000984FF4806001900320CDE9020141F25E
:1077D0000040C4F2020001A901F008FE06B080BD1D
:1077E000F0B503AF4DF804BD86B0006846F6000260
:1077F000C4F2000200219042CDE90411CDE902114A
:10780000019136D046F20041C4F20001884240F0B6
:107810008B8042F25801C2F200010A6843F6400030
:10782000C4F20200531C0B6052B9002100910168A0
:1078300041F000710160016801F000710091009950
:107840000021009150F8101C152441F0080140F867
:10785000101C50F8100C142500F00800009000983F
:1078600040F20040C4F2020000F50060132603213C
:1078700036E043F64000C4F202000091016841F096
:1078800080610160016801F080610091009942F21D
:107890005801C2F200010A68531C0B6052B9002162
:1078A0000091016841F000710160016801F0007110
:1078B000009100990021009150F8101C412441F0E2
:1078C000020140F8101C50F8100C402500F0020096
:1078D0000090009840F200403F266021C4F2020070
:1078E00001910221029100210391032104910921B8
:1078F000059101A901F07AFD304605210022FDF72E
:10790000C5FC3046FDF7EEFC284605210022FDF7B8
:10791000BDFC2846FDF7E6FC204605210022FDF7C8
:10792000B5FC2046FDF7DEFC06B05DF804BBF0BDFB
:10793000F0B503AF2DE9000F87B00446006845F6A7
:107940000041C4F2000100268842CDE90566CDE978
:10795000036602963AD045F60001C4F2000188425F
:1079600000F09B8045F20041C4F20001884240F0E3
:10797000DF80002543F630040195C4F2020420683C
:1079800002A940F002002060206800F0020001908F
:1079900001984FF44070029012200390012004904F
:1079A00003200590042006900020C4F2020000F598
:1079B000806001F01BFD0195206940F400102061FA
:1079C000206900F4001001900198B1E043F6300501
:1079D0000196C4F20205286840F2000840F0040055
:1079E00028602868C4F2020800F0040001900198A1
:1079F000019628680DF1080940F001002860286808
:107A00004FF0030A00F00100019001984FF400705C
:107A1000029012200390012004904FF0040B08F50F
:107A200000604946CDF814A0CDF818B001F0DEFC96
:107A30004FF48070029012200390012004A981E885
:107A4000010C4046494601F0D1FC019628694FF0EF
:107A5000C06140F400002861286941F6585500F4DF
:107A600000000190019846F24000C2F20005C4F205
:107A700002004FF4806285E843002846C5E90362AE
:107A8000C5E90566C5E907666E6201F091FA00284E
:107A900018BFFEF7BFFFA56349E0002643F6300597
:107AA0000196C4F202052868122140F020002860E7
:107AB000286800F020000190019803200391012123
:107AC0000290CDE90410042006900020C4F20200C8
:107AD00000F5A05002A901F089FC019628694FF039
:107AE000606140F480002861286941F6F84500F49F
:107AF00080000190019846F24000C4F20200783004
:107B0000C2F20005402285E847004FF400304FF4F0
:107B10008063C5E908062846C5E90436C5E9066656
:107B200001F046FA002818BFFEF774FF6563AC63E6
:107B300007B0BDE8000FF0BD81B0006840F600015D
:107B4000C5F20601884201D001B0704700200090C4
:107B500043F63400C4F20200016841F040010160C4
:107B6000006800F040000090009801B07047F0B548
:107B700003AF2DE9000F87B0044643F2000500680B
:107B8000C4F201050026A8420696CDE904660396D4
:107B9000029640F0868043F630000196C4F202005F
:107BA00041690DF1080941F48051416141694FF08B
:107BB000010B01F4805101910199019601684FF088
:107BC000030841F00201016001684FF0050A01F06D
:107BD0000201019101990196016841F001010160E2
:107BE0000068494600F001000190019818200290B9
:107BF0000220039005F55440CDF810B0CDF8148064
:107C0000CDF818A001F0F2FB802002900220CDE90F
:107C1000030BCDF8148046F2104805F55040494654
:107C2000C4F20208CDF818A001F0E0FB41F6B85507
:107C3000C2F200054FF440304FF0C06A4FF4806943
:107C4000C5E908062846C5E9008AC5E90266C5E90E
:107C50000496C5E9066601F0ABF9002818BFFEF7E7
:107C6000D9FEE564AC6341F6186508F14800C2F23C
:107C700000054021C5E9000A05F10800002280E85E
:107C800006024FF40030C5E908022846C5E905227E
:107C9000EA6101F08DF9002818BFFEF7BBFEA5646C
:107CA000AC6307B0BDE8000FF0BD80B56F4682B091
:107CB000006841F2FF31C4F20001884227DD40F242
:107CC000FF31C4F20101884241DC41F20041C4F2BB
:107CD0000001884255D00021C4F20101884240F0E1
:107CE00095800020019043F64000C4F202004168F4
:107CF000002241F0010141604068052100F00100CF
:107D0000019001981820FDF7C1FA18204EE040F2CA
:107D10000041C4F2000188424DD040F60001C4F297
:107D20000001884263D040F60041C4F2000188425D
:107D30006CD10020019043F64000C4F202000168BB
:107D400041F008010160006800F008005CE040F2CA
:107D50000041C4F2010188423BD044F20041C4F228
:107D60000101884252D10020019043F64000C4F244
:107D70000200416841F400314160406800F4003085
:107D800042E00020019043F64000C4F20200016886
:107D9000002241F0200101600068052100F0200070
:107DA000019001983720FDF771FA372002B0BDE845
:107DB0008040FDF797BA0020019043F64000C4F2DE
:107DC0000200016841F002010160006800F0020059
:107DD0001AE00020019043F64000C4F2020041681E
:107DE00041F002014160406800F002000CE0002018
:107DF000019043F64000C4F20200016841F0040122
:107E00000160006800F004000190019802B080BD9C
:107E1000F0B503AF2DE9000F87B000684FF6FF7192
:107E2000C4F2000188424FF000010691CDE904112F
:107E3000CDE9021131DC40F20041C4F20001884278
:107E40005DD040F60001C4F20001884274D040F6D3
:107E50000041C4F20001884240F0F380002001900C
:107E600043F63000C4F20200016841F08001016075
:107E70000068012100F08000019001984FF4E0506B
:107E8000029002200390CDE90410069040F6000015
:107E9000C4F2020000F5A054CFE044F20041C4F265
:107EA0000101884268D040F20041C4F201018842D9
:107EB00000F080800021C4F20101884240F0C180BE
:107EC0000020019043F63000C4F20200016841F046
:107ED000100101600068012100F01000019001987C
:107EE0004FF4D440029002200390CDE9041040F6F4
:107EF0000000C4F20200069100F500649DE000203D
:107F0000019043F63000C4F20200016840F600041C
:107F100041F0040101600068012100F004000190BB
:107F200001984FF48070029002200390CDE9041074
:107F30000690C4F2020480E00020019043F6300075
:107F4000C4F20200016841F00801016000680121EB
:107F500000F00800019001984FF480400290022048
:107F6000049103210390CDE9051040F60000C4F20E
:107F7000020000F5806460E00020019043F63000CC
:107F8000C4F20200016841F020010160006800F0C5
:107F9000200001900198402002900220CDE90300CA
:107FA00005900320069040F60000C4F2020000F5A0
:107FB000406442E0002043F630010190C4F2020127
:107FC0000A6840F6000442F480720A600A68C4F24B
:107FD000020402F480720192019A01900A6802265A
:107FE00042F004020A60096804F5C05501F004017A
:107FF0000191019980210DF108080291CDE90360FA
:1080000005904FF0030928464146CDF8189001F03D
:10801000EDF94FF0400A4FF0010B28464146CDE9FB
:1080200002A6CDE904B6CDF8189001F0DFF9CDE94C
:1080300002A6CDE904B6CDF8189002A9204601F0B9
:10804000D5F907B0BDE8000FF0BDF0B503AF2DE9DD
:10805000000F87B00446006844F60001C4F2000136
:1080600000268842CDE90566CDE90366029600F058
:108070009A8041F20041C4F20101884200F0DE80A2
:1080800041F20001C4F20101884240F0488100261B
:1080900043F630000196C4F20200416940F2000844
:1080A00041F0100141614169C4F2020801F0100180
:1080B000019101990196016802AD41F00201016050
:1080C00001684FF0020A01F0020101910199019645
:1080D00001684FF0030B41F00101016000684FF0AF
:1080E000070900F00100019001988020029008F536
:1080F00080602946CDE903A6CDF814B0CDF81890DC
:1081000001F074F94FF40070CDE9020ACDF818902F
:1081100046F2280940462946CDE9046BC4F202091B
:1081200001F064F941F6786509F59260C2F2000544
:108130004FF0006A4021C5E9000A05F108004FF43C
:10814000806880E842014FF4803B2846C5E9056617
:10815000EE61C5E908B600F02BFF002818BFFEF756
:1081600059FCA563AC6341F6D86509F58C60C2F291
:108170000005C5E9000A2846C5E90266C5E9048686
:10818000C5E90666C5E908B600F012FF002818BF69
:10819000FEF740FC252005210022E563AC63FDF7D6
:1081A00075F82520B9E043F630000196C4F20200CC
:1081B000016941F480210161016901F4802101918B
:1081C00001990196016841F004010160006802A96B
:1081D00000F00400019001984FF4406002900220EA
:1081E000CDE9030603200590072006900020C4F285
:1081F000020000F5006001F0F9F841F6387546F22A
:108200002800C2F20005C4F202004FF0006185E8C8
:1082100043004FF400304FF48062C5E90806284659
:10822000C5E90362C5E90566EE6100F0C1FE0028FC
:1082300018BFFEF7EFFBE563AC6370E0002643F682
:1082400030000196C4F20200416946F2280841F06C
:10825000200141614169C4F2020801F0200101914D
:1082600001990196016841F040010160006802A98E
:1082700000F04000019001984FF4844002900220E9
:10828000CDE9030603200590082006900020C4F2E3
:10829000020000F5C05001F0A9F841F6987508F504
:1082A0008360C2F200054FF0206A4FF48069C5E98F
:1082B000000A4FF4803B2846C5E90266C5E90496EA
:1082C000C5E90666C5E908B600F072FE002818BFC9
:1082D000FEF7A0FBE563AC6341F6F87508F58F6027
:1082E000C2F200054021C5E9000A05F1080080E856
:1082F00042022846C5E90566C5E9076B6E6200F0D3
:1083000057FE002818BFFEF785FB472005210022F5
:10831000A563AC63FCF7BAFF4720FCF7E3FF07B0A7
:10832000BDE8000FF0BDB0B502AF86B00068002414
:10833000B0F1A04F0594CDE903440294019401D01B
:1083400006B0B0BD43F630050094C4F202052868BB
:1083500001A940F001002860286800F001000090A9
:1083600000984FF4C05001900220CDE90204032090
:1083700004900A2005900020C4F2020001F036F8B3
:108380006868052140F080006860009468690022F8
:1083900040F480406861686900F480400090009873
:1083A0004320FCF773FF4320FCF79CFF06B0B0BDF1
:1083B000F0B503AF4DF804BD86B0002543F640018B
:1083C0000195C4F202010A68044642F010020A60F4
:1083D000096801A801F0100101910199694601F0B5
:1083E000E8FC049E002E18BF012601F0BCFC4DF6EF
:1083F0008361B040C4F21B31A0FB01014FF0FF309C
:1084000000EB914142F25C0041F20002C2F2000036
:10841000C4F2000240F2E733C0E90021C0E9025390
:1084200005618561FCF782FF0546C0B942F25C0038
:10843000C2F20000FDF743F8054680B93620FCF78C
:1084400051FF0F2C0AD8362021460022FCF71EFFD0
:1084500040F27000C2F20000046000E001252846EE
:1084600006B05DF804BBF0BD88B090E80E50D0E9CE
:108470000545C069079106920593CDF810C0CDF867
:108480000CE002940195009000BFFDE700000000A1
:1084900000000000000000000000000000000000DC
:1084A00000000000000000000000000000000000CC
:1084B00000000000000000000000000000000000BC
:1084C00000000000000000000000000000000000AC
:1084D000000000000000000000000000000000009C
:1084E000000000000000000000000000000000008C
:1084F000000000000000000000000000000000007C
:108500001EF0040F0CBFEFF30880EFF309808169C0
:10851000004A10476984000870470000FEE7000029
:10852000FEE70000FEE70000FEE77047012001F0D3
:108530003AB8082001F037B8102001F034B841F6FD
:108540003870C2F2000000F083BE41F65850C2F20B
:10855000000000F07DBE41F28C30C2F2000000F05D
:10856000D7BB41F28C30C2F2000000F0D1BB41F227
:108570008C30C2F2000000F0CBBB202001F013B819
:1085800041F24050C2F20000FDF713B9D0B502AF7E
:1085900041F23874C2F200042046FDF783FF42F234
:1085A000A400C2F2000001682046BDE8D0400847A0
:1085B00041F6F840C2F2000000F04ABE42F25C0010
:1085C000C2F20000FDF7F5B841F26060C2F20000AF
:1085D000FDF7EFB841F6B850C2F2000000F038BE27
:1085E00041F69870C2F2000000F032BE41F6186009
:1085F000C2F2000000F02CBE41F2B430C2F2000022
:1086000000F086BB41F2B430C2F2000000F080BB43
:1086100041F2B430C2F2000000F07ABB41F6D860FB
:10862000C2F2000000F014BE41F6F870C2F2000081
:1086300000F00EBE41F67860C2F2000000F008BE05
:10864000D0B502AF41F2C874C2F200042046FDF773
:1086500029FF42F2A400C2F2000001682046BDE8F2
:10866000D040084742F2A401C2F2000108607047FE
:108670004EF68850CEF20000016841F470010160AE
:108680007047002804BF01207047D0B502AF0446F0
:10869000006C30B92046FFF752F80020606484F87F
:1086A0003C00206CC0063AD4206C41F20211884391
:1086B000023042F204312064C4F20101086820F45F
:1086C000403008600A6894E809101A43D4F810E0B2
:1086D0000A604168012321F4807141604168C0F65D
:1086E000007341EA0E214160416821F04071416010
:1086F000416841EA0C014160816821F400618160B8
:10870000E168826811438160A16A8268994222F01F
:1087100070628260826804D122F040510AE0012038
:1087200052E011438160816821F040518160E16A2B
:10873000826811438160816821F002018160816853
:10874000227E94F8203041EA42018160416883B181
:1087500041F40061416041684EF2000221F4604141
:108760004160616ACFF6FF72436802EB4131194301
:1087700001E021F400614160C16A40F2000C21F483
:108780007001C162E2696169CFF6F07CC36A0CEBEB
:1087900002521A43C262826822F40072826094F824
:1087A0003020836843EA42228260826822F4806239
:1087B0008260826842EA8121816000206064216CCD
:1087C000012262F301012164002184F83C10D0BD34
:1087D000F0B503AF4DF804BD81B00022009290F8CF
:1087E0003C20012A01D1022177E00E6801221FFA04
:1087F00086FC80F83C204FEA4C0212FA86F30268AD
:108800000A2E32BF10321E3B0C324FF0070E156895
:108810000EFA03F4A54315608D68146805FA03F396
:10882000234313604968062906D8026801EB8101D9
:10883000053902F134030AE00C2901EB81010268D9
:1088400087BF413902F12C03233902F130031F2283
:108850001C688A4024EA02021A601A680CFA01F1C4
:10886000114342F2043E1960C4F2010E0168AEF5F4
:108870004172914208BF122E02D0914208D029E0E5
:10888000DEF8003043F48003CEF80030914221D16D
:1088900026F0010110291DD1DEF80010102E41F440
:1088A0000001CEF8001015D140F27801C2F20001AB
:1088B00009684DF68362C4F21B32A1FB0212910CCF
:1088C00001EB8101490000BF0091009911B10099AD
:1088D0000139F9E7002180F83C10084601B05DF845
:1088E00004BBF0BDB0B502AFC0B1044690F82000A3
:1088F00010B92046FEF774FF2068016841F00101BD
:108900000160FCF798FC054620684168C90707D15B
:10891000FCF791FC401B0B28F6D312E00120B0BD00
:10892000016821F002010160FCF785FC054600BFEB
:108930002068416889070DD5FCF77DFC401B0B289A
:10894000F6D3606A052140F400306062012084F8AB
:108950002010B0BD217E0268012922F0800208BFEC
:1089600080320260617E0268012922F0400208BF65
:1089700040320260A17E0268012922F0200208BF75
:1089800020320260E17E0268012922F0100218BF45
:1089900010320260217F0268012922F0080208BF1C
:1089A00008320260617F0268012922F0040208BFD8
:1089B00004320260D4E901C2D4E9033561691A4383
:1089C0002A431143ACF101021143C161002001218E
:1089D000606284F82010B0BDB0B502AF90F82020DE
:1089E000013A012A2FD846F20060C4F20000026862
:1089F00042F001020260026822F47C520260D1F867
:108A000014E0CC694A6A0368012C43EA022202603E
:108A10000EF01F024FF0010303FA02F2C3696FEA7E
:108A2000020C23EA0203C36113D02CBBC36803EA20
:108A30000C03C360CB688C8844EA034300EBCE048C
:108A400023640B4611E0416A41F480214162012018
:108A5000B0BDC3681343C3600B688C8844EA03430A
:108A600000EBCE04236401F10C038C681B8843EAFD
:108A7000044300EBCE04636443688D6943EA020457
:108A8000D1F810E0096A002D08BF03EA0C04446025
:108A90004369BEF1000F43EA020408BF03EA0C0475
:108AA0000129446102D1C1691143C161016821F00A
:108AB000010101600020B0BDB0B502AF044690F8DE
:108AC000200001281CD1022084F8200020680168C1
:108AD00021F001010160FCF7AEFB0546206840680B
:108AE000C00713D0FCF7A7FB401B0B28F6D3606A26
:108AF00040F400306062052084F820000120B0BD01
:108B0000606A40F4002060620120B0BD0020606215
:108B1000B0BDD0B502AF90F820E0D0F800C0AEF103
:108B2000010EBEF1010FDCF808E00ED81EF0E05F88
:108B300011D0CEF3016E012000FA0EF018608B68A0
:108B40007BB1486843EAC0030DE000F12401012035
:108B50004FF4802238E000F1240101204FF400128C
:108B600032E008684305D1E9030403430CEB0E101F
:108B7000C0F88031C0F88441097D012905D100F594
:108B8000C2710B6843F480730B609479D179537987
:108B9000240492F804C044EA016141EA032101EB94
:108BA0000C03C0F88C31937892F800C05478D278D6
:108BB0001B0443EA026242EA0422624400F5C071E7
:108BC000C0F88821002001220B681A430A60D0BD3A
:108BD000D0B502AF90F82040013C012C75D8046854
:108BE00000290CBFE4682469A40774D0046804EB6E
:108BF000011CDCF8B0410CF5D87E14F0040494603C
:108C0000DCF8B04119BFE4085460640D1460DEF86C
:108C100000400CF5DA7E04F00204D460DCF8B441C4
:108C200024075ABFDEF8004004F00F040824146142
:108C3000DEF800400029C4F307249461DEF8004008
:108C40004FEA14445461DCF8B8211A70026802EB50
:108C50000112D2F8B8214FEA12225A70026802EBD0
:108C60000112D2F8B8214FEA12429A70026802EB60
:108C70000112D2F8B8214FEA1262DA70026802EBF0
:108C80000112D2F8BC211A71026802EB0112D2F86B
:108C9000BC214FEA12225A71026802EB0112D2F88B
:108CA000BC214FEA12429A71026802EB0112D2F81B
:108CB000BC214FEA1262DA7100680CBF00F10C01AE
:108CC00000F11001002020220AE000F1240101201F
:108CD0004FF4802204E000F1240101204FF400123F
:108CE0000B681A430A60D0BD90F82020013A012A8F
:108CF00004D8006800F11402002004E000F124020E
:108D000001204FF48021136819431160704700005F
:108D1000F0B503AF2DE9000F81B004460068466945
:108D2000D0F80490D0F80880D0F80CB0D0F810A09B
:108D300081690091F10703D10025300722D429E091
:108D40005FEAC87113D001215FEA887281600BD499
:108D50005FEA487000F1B3805FEA087000F1B98003
:108D6000204600F00DF902E0204613F055FD0025E5
:108D70005FEAC85000F186805FEAC83000F1B28037
:108D8000300707D51BF0100004D0206845F40075AB
:108D90001021C160700708D51BF0080005D02068BD
:108DA0000821C160204600F0EEF8B00706D5206823
:108DB000C068800702D0204613F028FE700607D551
:108DC0001AF0100004D0206845F48065102101617C
:108DD000B00608D51AF0080005D020680821016106
:108DE000204600F0D1F8F00606D52068006980071B
:108DF00002D0204613F067FEB00308D519F010002A
:108E000005D0206810214160204600F0BEF8F00334
:108E100008D519F0080005D02068082141602046D7
:108E200000F0B4F8300440F19A805FEA497040F1F4
:108E30009380009B06F4807003EA10202843990772
:108E4000014648BF41F00201B20558BF014658072C
:108E50000D4648BF45F00405700558BF0D46300566
:108E600040F17A8013F0700000F07680103800092D
:108E700005286CD8DFE800F0035D6063666945F0A3
:108E8000080564E020684FF480715FEA88528160D1
:108E90000DD45FEA485015D45FEA08501CD4204630
:108EA00000F06FF85FEAC8307FF56AAF1AE020463D
:108EB00013F0DCFC5FEAC8307FF562AF12E04FF4DC
:108EC000006555E705F500555FEAC8307FF558AFF6
:108ED00008E04FF480554BE705F580455FEAC83060
:108EE0007FF54EAF20684FF480315FEA88328160B1
:108EF0000CD45FEA483010D45FEA083013D420461F
:108F000000F040F830073FF53DAF43E7204613F04F
:108F1000D7FC30073FF536AF3CE705F50045300795
:108F20003FF530AF36E705F5803530073FF52AAF1E
:108F300030E745F010050AE045F0200507E045F070
:108F4000400504E045F0800501E045F480752068A7
:108F5000816921F0700181612068042141605DB167
:108F6000606A40EA05012046616201B0BDE8000F79
:108F7000BDE8F04013F0CEBC01B0BDE8000FF0BD7D
:108F80007047704770477047704770477047014699
:108F900090F820000138022803D2002200204A6203
:108FA0007047486A40F4802201204A6270470000FE
:108FB000F0B503AF2DE9000B0446FCF73CF9C4B152
:108FC0000546022084F835000020216884F834002A
:108FD000086820F00100086020680168C9070CD00B
:108FE000FCF729F9401B0528F6D90321202203208C
:108FF0007DE00120BDE8000BF0BD016848F23F02B2
:10900000CFF21002D4E9013501EA020ED4E90321BE
:1090100043EA0E032B43D4E9056C1A431143D4E908
:109020000789314341EA0C02616A42EA08020429D5
:1090300042EA090304D1D4E90B261A4342EA0603A3
:1090400003604269042922F0070241EA02012DD19E
:10905000D4E90A5341EA050143B3BCF5005F08D0E7
:10906000BCF1000F12D1022D16D0012D07D09DB1F9
:1090700019E0032D17D8DFE805F00B0F0B02A3F161
:10908000C072B2FA82F252094AB90FE0032D02D23D
:10909000012222B90AE006D1C3F3006232B10121F4
:1090A0004022012023E00022002AF8D16FF00F02B5
:1090B0004AF6AB2352FA80F2CAF6AA23A2FB033681
:1090C00048F6E00341613109C0F60203595C40F201
:1090D000FF3398435F2A4FF03F0288BF0430C4E952
:1090E000160102FA01F1816000220121002062656F
:1090F00084F83510BDE8000BF0BDF0B503AF4DF8B6
:1091000004BD90F834C0BCF1010F47D04FF0010C02
:1091100080F834C0D0F858E090F835C0BCF1010FA9
:1091200039D14FF0020C80F835C04FF0000CC0F878
:1091300054C0D0F800C08468056CC06DDCF80060D5
:10914000402C26F48026CCF80060CCF804300B4686
:1091500004BF13460A463F2101FA00F0CCF808305C
:10916000CCF80C20CEF80800DCF8000040F0160027
:10917000CCF800002DB1DCF8000040F00800CCF87D
:109180000000DCF8000040F00100CCF800000020F6
:109190005DF804BBF0BD002180F8341002205DF8BA
:1091A00004BBF0BDF0B503AF4DF804BD866D0446B9
:1091B000FCF741F894F83510022924D105462068BF
:1091C000216C026822F016020260426922F08002DD
:1091D000426109B9A16C19B1016821F0080101606F
:1091E000016821F00101016020680068C0070ED00D
:1091F000FCF721F8401B0628F6D3202060650320E9
:1092000084F835000CE080206065012008E0E06D06
:109210003F2101FA00F0B060012084F83500002001
:10922000002184F834105DF804BBF0BD90F83510CF
:10923000022909D1052180F835100068016821F064
:1092400001010160002070478021416501207047C5
:10925000F0B503AF4DF8048D82B0044600200190B4
:1092600040F27800C2F200000268D4E9166048F2C9
:10927000B51335680821C1F64E3381402942A2FB5F
:1092800003280CD0226813685B0708D5136823F005
:1092900004031360B160616D41F00101616501215A
:1092A0008140294208D022685269120604D5B16073
:1092B000616D41F00201616504218140294208D0BD
:1092C00022681268920704D5B160616D41F0040113
:1092D000616510218140294215D02068026812077B
:1092E00011D5B16002680168520306D4C90506D4DD
:1092F000016821F00801016001E008033ED4216CFF
:1093000009B120468847E16D202000FA01F22A4287
:1093100040D020680368DB063CD5B26094F8353055
:109320000268052B1AD122F016020260426922F06F
:1093300080024261226C0AB9A26C1AB1026822F062
:10934000080202603F208840B060012084F83500A8
:10935000216D002084F83400E1BB42E00168520333
:1093600010D4C90512D4016821F010010160012058
:1093700084F83500002084F8340007E0A16C00294F
:10938000BFD1C0E7080301D4616C00E0E16B09B113
:1093900020468847606D20B3606DC00718D0052057
:1093A00084F8350020684FEA9821026822F0010213
:1093B000026000BF019A01328A42019202D802681B
:1093C000D207F7D1012084F83500002084F834005A
:1093D000E16C31B1204602B05DF8048BBDE8F0408D
:1093E000084702B05DF8048BF0BD0000F0B503AF94
:1093F0002DE9000F82B000F13E4241F6004402F137
:10940000FF76C4F2020408224FEAB625A04208BF44
:10941000072200244FF0000A4FF00008072D38BF44
:109420004FEAB622009209E008F101080AF1020AA7
:10943000B8F1100F04F1040400F0A7800A680123BA
:1094400003FA08FB12EA0B09EED0D1F804E00EF0A3
:10945000030CACF10102012A12D882680323CD6803
:1094600003FA0AF6B24305FA0AF52A438260426813
:10947000CEF3001622EA0B0206FA08F632434260E7
:10948000BCF1030F1DD0C26803238D6803FA0AF6EE
:10949000B24305FA0AF63243BCF1020FC26010D1A2
:1094A0006FF0030202EA58020244D2F820C004F02E
:1094B0001C050F230E69AB402CEA0303AE40334377
:1094C0001362026803234E6803FA0AF39A4306F014
:1094D000030303FA0AF31A4316F4403F0260A3D0D1
:1094E000002243F644030192C4F202031A6843F6D1
:1094F000004E42F480421A601A68C4F2010E02F46F
:1095000080420192019A28F003024FF6084C7244FF
:10951000CFF6FF7C52F80C3004F00C060F25B54056
:10952000AB43009D05FA06F6334342F80C30DEF8F3
:1095300008204B6842EA090643F60C4CDD0258BF8E
:1095400022EA0906CEF80860C4F2010CDCF800201B
:109550009D0242EA090658BF22EA0906CCF80060DB
:10956000DEF804209D0342EA090658BF22EA0906F4
:10957000CEF80460DEF80020DB0342EA090358BF9E
:1095800022EA0903CEF800304EE702B0BDE8000F32
:10959000F0BD0069084018BF01207047002A08BFCD
:1095A00009048161704743F61441C4F201010A685D
:1095B000024214BF0860704713F0F8BAF0B503AF69
:1095C0004DF8048DB0B3044690F83D0028B9002052
:1095D00084F83C002046FEF7ABF9242084F83D00D7
:1095E0002068016821F001010160016841F4004137
:1095F0000160016821F40041016000F0B4FB48F211
:109600008041C0F21E0140F60012656888424FF0AA
:109610000001C0F23D0248F2A16C4FF0000338BFD8
:1096200001219042C0F2010C38BF0123654538BFCB
:109630000B461BB101205DF8048BF0BD4DF6836134
:10964000C4F21B31A0FB011221684FEA924E4B6815
:109650004FF4967623F03F0343EA92434B6044F67F
:10966000D3530EFB06F6C1F26203D1F82080A6FBAD
:109670000336B60928F03F03654538BF960C721CC7
:109680001A430A62CA6948F2A0664CF6FF73C0F238
:109690000106B54222EA030C0AD801386A00B0FB81
:1096A000F2F001306FF31F30042898BF04202BE044
:1096B000A368A0F1010E9BB119206843BEFBF0F036
:1096C0000422013062F31F30000512D09BB1192033
:1096D0006843BEFBF0F00422013062F31F3011E05A
:1096E00005EB4500BEFBF0F001306FF31F300005C5
:1096F000ECD1012008E005EB4500BEFBF0F00130A5
:109700006FF31F3040F4004040EA0C00C861086865
:10971000D4E9072320F0C00010431843086088688C
:1097200048F2FF3204F10C0690434CCE184310432C
:10973000A5698860C86820F0FF0030432843C860EE
:10974000086840F00100086000202021206484F8AF
:109750003D10206384F83E005DF8048BF0BD0000EE
:10976000B0B502AF82B0002858D00446056890F822
:10977000950428B9002084F894042046FEF7D3FD10
:109780000320B5F1A04F84F8950404BF0020A07118
:10979000206801F058F994E80F00257C009501F04D
:1097A000CFF8C0BB2068002101F054F998BB2079A4
:1097B00050B300EBC000800000214FF0010C0023EB
:1097C000002500BFE21824331575D585984205F1B0
:1097D000010582F815C01176C2E907115162F1D175
:1097E00000210022002300BFA518243285F854323E
:1097F000904203F1010385F8551285F85812C5E926
:109800009711C5F86412EFD194E80F00257C0095FC
:1098100001F054F930B1022084F89504012528465E
:1098200002B0B0BD00250120657484F8950420685D
:1098300001F040FAF3E70000F0B503AF2DE9000BAB
:1098400082B0002800F0AE808146007843F6000622
:10985000C007C4F2020646D0B06800F00C0004282D
:1098600006D1306880033ED5D9F80400D8BB99E012
:10987000B06800F00C00082802D170684002F0D4F3
:10988000D9F80450B5F5A02F0AD0B5F5803F0BD01C
:10989000306820F480303060306820F4802006E0AA
:1098A000306840F480203060306840F480303060B0
:1098B000FBF7C1FC002D054612D000BF30688003C5
:1098C00011D4FBF7B8FC401B6428F7D92EE100BF88
:1098D000FBF7B1FC401B64284FF0030000F2278126
:1098E00030688003F4D499F8000080071CD5B06874
:1098F00010F00C0F09D0B06800F00C00082840F000
:1099000090807068400200F18C803068800703D539
:10991000D9F80C00012845D13068D9F8101020F092
:10992000F80040EAC100306099F8000000073BD41D
:1099300099F8000040074ED4D9F8184084B3B068B5
:1099400000F00C00082840F0A180012C2AD070689B
:10995000D9F81C1000F480028A4223D1D9F82010D3
:1099600000F03F028A421DD147F6C071D9F8242089
:109970000140B1EB821F15D1D9F828200023CFF682
:10998000FF7303EBC23200F440316FF30F029142D8
:1099900008D1D9F82C1000F07060B0EB016F01D144
:1099A0000020C4E00120C2E0D9F81400002840F2F1
:1099B0000000C4F2472059D00121C0F8801EFBF7F7
:1099C0003AFC0546706F8007B2D4FBF734FC401BAD
:1099D0000228F7D9AAE0306C10F080580AD1002094
:1099E0000190306C40F080503064306C00F080505A
:1099F0000190019847F20004C4F200042068C005F9
:109A000026D4206840F480702060FBF714FC0546E3
:109A10002068C0051CD4FBF70EFC401B0228F7D9B8
:109A200084E0D9F80C00002854D00020C4F247206C
:109A300001210160FBF7FFFB054600BF306880078E
:109A40003FF56AAFFBF7F7FB401B0228F6D96DE044
:109A5000D9F80850052D51D0012D53D0306F20F08A
:109A600001003067306F20F004004EE00021C0F8A4
:109A7000801EFBF7E0FB0546706F80077FF558AF4F
:109A8000FBF7D9FB401B0228F6D94FE040F2000853
:109A9000C4F247280020C8F86000FBF7CCFB022C7A
:109AA00005460BD13068800159D5FBF7C4FB401B3C
:109AB00002284FF00300F5D939E000BF306880017B
:109AC0007FF56EAFFBF7B7FB401B02284FF003009A
:109AD000F4D92CE00020C4F2472000210160FBF7FC
:109AE000AAFB0546306880077FF51EAFFBF7A3FB96
:109AF000401B02284FF00300F4D918E0306F40F00B
:109B000004003067306F40F001003067FBF793FBD3
:109B1000002D054641F2883415D000BF306F800714
:109B200014D4FBF788FB401BA042F7D9032002B0F6
:109B3000BDE8000BF0BD00BFFBF77DFB401BA04262
:109B40004FF00300F3D8306F8007F5D4B8F1000F61
:109B50007FF4F2AE306C20F080503064ECE609F116
:109B60001C052FCD08430021CFF6FF7140EA82107B
:109B700001EBC3316FF30F0140EA056008437060E9
:109B80000120C8F86000FBF756FB044630688001EE
:109B90003FF506AFFBF74FFB001B02284FF0030019
:109BA000F4D9C4E7F0B503AF2DE9000B002879D054
:109BB00043F60808C4F202080446D8F8F8038946B8
:109BC00000F00700884207D288F8F893D8F8F80325
:109BD00000F00700484565D12068810717D5410787
:109BE00005D5D8F8001041F4E051C8F8001001077D
:109BF00005D5D8F8001041F46041C8F80010D8F835
:109C00000010A26821F0F0011143C8F80010C0074D
:109C100040D1D8F8F80300F00700484507D988F884
:109C2000F893D8F8F80300F0070048453AD12068C7
:109C3000410707D5D8F80010E26821F4E05111433C
:109C4000C8F80010000708D5D8F80000216920F4F2
:109C5000604040EAC100C8F8000000F04FF8D8F8B2
:109C6000001048F6C802C1F30311C0F60202515CAD
:109C700040F2780220FA01F140F27000C2F20000D6
:109C80000068C2F200021160FEF792FB0020BDE8FE
:109C9000000BF0BD6068811E022907D258F8081C2D
:109CA000890109D40120BDE8000BF0BD012820D1B5
:109CB00058F8081C8903F5D5D8F8001021F00301E5
:109CC0000843C8F80000FBF7B6FA064641F28835AB
:109CD000D8F80000616800F00C00B0EB810F98D05C
:109CE000FBF7A9FA801BA842F2D90320BDE8000BBC
:109CF000F0BD58F8081C8907D4D5DDE7D0B502AF10
:109D000043F60404C4F20204606800F00C00082862
:109D10000AD0042819BF42F20040C0F2F40041F614
:109D20000030C0F2B700D0BD206821682368490226
:109D300041F60031C0F2B70100F03F02C3F38810D2
:109D40005CBF42F20041C0F2F401A1FB000100231C
:109D5000F7F766F921680222C1F3014102EB4101E4
:109D6000B0FBF1F0D0BD40F2780043F60801C2F23A
:109D70000000C4F202010068096848F6D802C1F385
:109D80008221C0F60202515CC840704740F2780060
:109D900043F60801C2F20000C4F20201006809683B
:109DA00048F6D802C1F34231C0F60202515CC84005
:109DB00070470F22026043F60802C4F202021368E1
:109DC00003F003034360136803F0F0038360136838
:109DD00003F4E053C360D2F800C04FF4E05303EA49
:109DE000DC030361D2F8F80300F007000860704755
:109DF000002804BF01207047D0B502AF0446407967
:109E000020B9002020712046FDF796FE02206071E7
:109E10002068016841F004010160012060710020A8
:109E2000A060D0BDF0B503AF4DF804BD38B1044615
:109E3000406A30B10020206104F1140007E00126DF
:109E40004BE06068B0F5827F03D004F11C00002174
:109E500001600026A66294F8510020B9204684F8DB
:109E60005060FDF784FE022084F8510094E80F0052
:109E700001F48271056802F4044225F04005056092
:109E8000114403F400622369114403F00202636980
:109E9000114403F00102A369E569114403F400725F
:109EA000114405F03802256A114405F08002A56AC4
:109EB000114305F4005211430160626A042101EA72
:109EC000134102F0100211444160C16921F40061A4
:109ED000C1610120666584F8510030465DF804BB1D
:109EE000F0BD0000F0B503AF2DE9000B84B00446CF
:109EF00090F85000012801D102206CE00120994621
:109F000015460E4684F85000FBF795F994F8511069
:109F100001295CD18046002E4FF0010018BF002DB2
:109F200056D0032084F85100002060652663A58682
:109F3000E586A063A087E087A168C4E91000B1F5B9
:109F4000004F08D12068016821F0400101600168DC
:109F500041F48041016020680168490603D401682A
:109F600041F04001016061686B1EE268B1FA81F165
:109F7000B3FA83F349095B09B2F5006F41EA0301C3
:109F80002DD131B136F8021BC1602663E08E013855
:109F9000E086E08E00284AD009F101050AE000BF02
:109FA000216B31F8022BC2602163E08E0138E0861C
:109FB000E08EE0B3206881688907F1D4FBF73BF9B4
:109FC000002DF5D0A0EB08004845F1D32DE002208C
:109FD000002184F8501004B0BDE8000BF0BD39B189
:109FE00031780173206B01302063E08E0138E08608
:109FF000E08EE0B109F101050BE000BF216B0978AB
:10A000000173206B01302063E08E0138E086E08E22
:10A0100068B1206881688907F0D4FBF70CF9002D3E
:10A02000F5D0A0EB08004845F1D303204BE02046D3
:10A03000022101224B46CDF8008000F00FFC28B130
:10A04000606D032540F02000606529E040F2780053
:10A05000C2F20000006849F68171C1F25E61A0FBA6
:10A060000101480D4FF47A71484303906068B0F5E0
:10A07000827F0BD12046802100224B46CDF8008004
:10A08000002500F0EBFB0028DAD109E0039830B19D
:10A09000039801380390206880680006F6D40025F4
:10A0A000002D1CBF20206065A06838B900200290F8
:10A0B0002068C1680291806802900298606D08B1C2
:10A0C000012085E70020012184F8511080E700007D
:10A0D000F0B503AF2DE9000782B0044690F85100B7
:10A0E00001280ED16068994692460D46B0F5827FF0
:10A0F00001D1A068C8B194F85000012803D102260C
:10A100000EE0022609E0012684F85060FBF793F880
:10A11000002D18BFBAF1000F13D1002084F85000B1
:10A12000304602B0BDE80007F0BD042084F85100BD
:10A13000204629462A465346CDF8009000F074F890
:10A14000EFE78046042084F8510000206065A56395
:10A15000A4F83CA0A4F83EA02063A086E086A168F5
:10A160002064B1F5004F606408D12068016821F0D7
:10A1700040010160016821F48041016020680168AC
:10A18000490603D4016841F040010160E168E08FB5
:10A19000D9B1B8B309F101050AE000BFC068A16BED
:10A1A00021F8020BA163E08F0138E087E08F48B30C
:10A1B00020688168C907F1D1FBF73DF8002DF5D083
:10A1C000A0EB08004845F1D31AE0D8B109F1010528
:10A1D0000AE0007BA16B0870A06B0130A063E08FE8
:10A1E0000138E087E08F68B120688168C907F0D145
:10A1F000FBF721F8002DF5D0A0EB08004845F1D37E
:10A2000003260DE020464946424600F039F9002871
:10A210001CBF20206065606D08B101267DE7002627
:10A22000012084F8510078E7F0B503AF2DE900076D
:10A2300084B0044690F85000012801D10220CAE001
:10A2400001201D4616468A4684F85000FAF7F3FFAF
:10A2500094F85110814601296DD1BAF1000F4FF0E9
:10A26000010018BF002E00F0B380002D00F0B08078
:10A2700094F85100002104281CBF052084F85100E7
:10A280006165A663E587A587C4F830A0E5862068E8
:10A29000A586216461640168490603D4016841F020
:10A2A0004001016061686B1EE268B1FA81F1B3FAA6
:10A2B00083F3D7F8088049095B09B2F5006F41EADA
:10A2C000030146D139B13AF8021BC160C4F830A08D
:10A2D000E08E0138E086012608F10105E08E10B914
:10A2E000E08F00287BD02068816889070CD5E18E3B
:10A2F00051B1012E08D1216B002631F8022BC2602A
:10A300002163E18E0139E1868168C9070AD0E18FB6
:10A3100041B1C068A16B012621F8020BA163E08F57
:10A320000138E087FAF787FF002DD7D0A0EB0900AE
:10A330004045D3D348E06068B0F5827F07D1A0687C
:10A3400000284FF0020008BF042941D185E7022010
:10A350003EE041B19AF800100173206B0130206398
:10A36000E08E0138E086012608F10105E08E08B98B
:10A37000E08FA0B32068816889070DD5E18E59B1BF
:10A38000012E09D1216B002609780173206B013061
:10A390002063E08E0138E08620688168C9070BD011
:10A3A000E18F49B1C068A16B01260870A06B013034
:10A3B000A063E08F0138E087FAF73DFF002DD5D08C
:10A3C000A0EB09004045D1D3012084F851000320BF
:10A3D000002184F8501004B0BDE80007F0BD20460D
:10A3E000022101224346CDF8009000F037FA48B12F
:10A3F000606D032540F02000606575B32020606526
:10A400000120E5E740F27800C2F20000006849F65A
:10A410008171C1F25E61A0FB0101480D4FF47A71B8
:10A42000484303906068B0F5827F0BD120468021BD
:10A4300000224346CDF80090002500F00FFA0028D6
:10A44000D6D1DAE7039830B1039801380390206839
:10A4500080680006F6D40025CFE7A06838B9002050
:10A4600002902068C1680291806802900298606D35
:10A4700000284FF0010004BF84F851000020A7E736
:10A48000B0B502AF82B0044640680B46B0F5827F9B
:10A4900012D1A168B1F5004F02D0B1F5806F04D19F
:10A4A00021680D6825F040050D60B0F5827F03D16D
:10A4B000A068B0F5806F0FD12046012100920022E4
:10A4C000002500F0CBF920B1606D032540F020009D
:10A4D0006065284602B0B0BD009220468021EEE7BC
:10A4E000806B01684A6822F003024A60416D41F0C6
:10A4F00010014165012180F8511000F0ABB9B0B5F1
:10A5000002AF044690F85100012810D113460A46C4
:10A51000A16871B96068B0F5827F0AD10425204630
:10A52000114684F85150BDE8B04000F05FB80220F9
:10A5300058E094F85000012804BF0220B0BD01206B
:10A54000002A84F8500018BF002B4BD004204FF095
:10A55000000C254684F8510045F854CFB1F5004F62
:10A5600045F81C2C25F8183C25F8163C45E905CC87
:10A5700025F820CC25F81ECC08D12068016821F0F0
:10A5800040010160016821F480410160E06C4AF201
:10A590000D7E4AF21373C0F6000EC0F60003C0E948
:10A5A0000F3E4AF2E143C0F600032168C0E9133CC4
:10A5B000E38F0C31FEF7A1FD10B1012010210EE058
:10A5C00025682868400603D4286840F040002860C9
:10A5D00055F8040F012140F02000286000202A686F
:10A5E00011432960002184F85010B0BDF0B503AFCD
:10A5F0004DF8048D044690F85000012803D1022044
:10A600005DF8048BF0BD012084F8500094F851608F
:10A61000012E58D100294FF0010018BF002A5FD049
:10A62000002B5DD094F851004FF000082546042817
:10A630001CBF052084F8510045F8548F2163A38680
:10A64000E386A263A387E387C4E9108894F85100E6
:10A650004AF20D714AF28173C0F60001C0F60003A0
:10A66000042808BF0B464AF213704AF28971C0F6FB
:10A670000000C0F6000108BF0146E06C2668C0E992
:10A680000F134AF2E141C0F60001C0E91318E38F4D
:10A6900006F10C01FEF731FD78B92268216BA06C40
:10A6A000536843F001035360C0E90F88C0E9138881
:10A6B000E38E0C32FEF721FDC0B1012010212A6883
:10A6C000114329600CE06068B0F5827F07D1A06873
:10A6D00000284FF0020008BF042E01D19AE70220A3
:10A6E000002184F850105DF8048BF0BD25682868BF
:10A6F000400603D4286840F04000286055F8040F55
:10A70000022140F0200028600020D8E7806B00F094
:10A71000A3B8B0B502AF846B0546FAF78CFD296883
:10A720000968C90527D402462068A168436823F058
:10A730002003436031B96168B1F5827F02D16FF0C7
:10A74000030101E06FF001014368194041602046B8
:10A750006421FFF795FE00281CBF202060650020C3
:10A76000E087012084F85100606D20B12046BDE8EB
:10A77000B04000F06FB82046BDE8B04012F01FBBFB
:10A78000806B00F06AB80000B0B502AF82B0846B95
:10A790000546FAF750FD29680968C90554D40546ED
:10A7A000206801224168642321F020014160204695
:10A7B0000221009500F052F828B1606D032540F0A9
:10A7C0002000606528E040F27800C2F200000068D6
:10A7D00049F68171C1F25E61A0FB0101480D4FF4A1
:10A7E0007A71484301906068B0F5827F0AD12046B3
:10A7F0008021002264230095002500F02FF8002816
:10A80000DBD109E0019830B101980138019020684E
:10A8100080680006F6D400251DB1606D40F0200070
:10A8200060652068416821F0030141600020E086F6
:10A83000E087012084F85100606D28B1204602B005
:10A84000BDE8B04000F006B8204602B0BDE8B04018
:10A8500000F001B87047704770477047F0B503AF1C
:10A860002DE9000F81B0BC68994693460E4680469C
:10A87000FAF7E1FC201A00EB0904FAF7DCFC40F2DD
:10A880007801C2F200010968C1F3CB316143009144
:10A89000D8F8001089683140891BB1FA81F1490963
:10A8A000594501D1002046E0824609F1010509E041
:10A8B000D8F8000080683040801BB0FA80F0400972
:10A8C0005845EFD0002DF3D0FAF7B5FCA0EB0A0005
:10A8D000A04207D200980099002808BF0446481EED
:10A8E0000090E5E7D8E900014268B1F5827F22F0E7
:10A8F000E00242600BD1D8F80810B1F5004F02D049
:10A90000B1F5806F03D1016821F040010160D8F8F2
:10A910002810B1F5005F07D1016821F400510160F2
:10A92000016841F400510160012088F851000020C5
:10A9300088F85000032001B0BDE8000FF0BD000012
:10A9400082B002F47F42B2F5807F38D1826B4FF63D
:10A95000BF7322F480328263C268CFF6BD731A409F
:10A96000C260029BC268DBB222F44012012BC260BB
:10A9700003D1C26842F48012C2600022009200BF7C
:10A98000009A01320092009AB2F1706F3DD80269CC
:10A99000B2F1FF3FF4DC00220092026942F00102B2
:10A9A000026100BF009A01320092009AB2F1706F0A
:10A9B0002BD80269D207F5D14FF0000C33E0C26802
:10A9C00042F04002C2600022019200BF019A0132AF
:10A9D0000192019AB2F1706F1AD80269B2F1FF3F89
:10A9E000F4DC00220192026942F00102026100BF20
:10A9F000019A01320192019AB2F1706F08D802698E
:10AA0000D207F5D14FF0000C04E04FF0030C0AE040
:10AA10004FF0030C826B13F47F4F14BF22F480328B
:10AA200042F48032826301F47F01B1F5803F07D1A7
:10AA3000816841F006018160816841F020018160F8
:10AA4000604602B070470146806820F00102002095
:10AA50008A607047B0B502AF0446C06820F0C040BD
:10AA6000E06099B1012927D1E068002540F000504D
:10AA7000E06000BF0A20FAF7E5FB6069C00705F156
:10AA80000A0014D1BE2D0546F4D310E0E06800257D
:10AA900040F08040E06000BF0A20FAF7D3FB606915
:10AAA000C00705F10A0002D0BE2D0546F4D3C83810
:10AAB000B0FA80F04009B0BD0120B0BDF0B503AFE1
:10AAC0002DE9000F84B01B0C00F580760F250024C3
:10AAD000013D46F8044FFBD1DDB23DB1836B23F459
:10AAE00000138363836B43F4002310E0D0F8043831
:10AAF00043F00203C0F80438836B43F4001383630C
:10AB0000836B23F400238363836B23F4802302F499
:10AB10007F4683630023B6F5807FC0F8003E07D1EF
:10AB2000D0F80068B3EB116F07D1C0F8006808E0F7
:10AB3000D0F8003843F0030301E046F00103C0F809
:10AB400000380023029300BF029B01330293029B53
:10AB5000B3F1706F18D80369B3F1FF3FF4DC002341
:10AB600002934FF484630361029B4FF0000E0133A4
:10AB70000293029BB3F1706F88BF4FF0010E05D8AE
:10AB800003699B06F0D401E04FF0010E002303930C
:10AB9000CDE90052039B01330393039BB3F1706F24
:10ABA00018D80369B3F1FF3FF4DC002303931023AB
:10ABB000036100BF039B4FF0000B01330393039B22
:10ABC000B3F1706F88BF4FF0010B05D80469E4063C
:10ABD000F0D401E04FF0010BCCB24FF00008C0F808
:10ABE0001088C0F81488C0F81C889CB300F5106663
:10ABF0004FEA441C4FF67F39002400BF35594FF00F
:10AC00009042002C08BF4FF0006202EAE57233194F
:10AC100032512034A445C3F81080C3F80890EDD118
:10AC200000F530664FF000094FF67F3A002400BF70
:10AC300033594FF09045002C08BF4FF0006505EAEE
:10AC4000E373321933512034A445C2F81090C2F88E
:10AC500008A0EDD1D0F8102811F47F0F22F48072F3
:10AC6000C0F810286FF08042C0F81880426103D10C
:10AC7000816941F010018161816943F60002C8F2E7
:10AC80003C021143019A816112F47F0F009A03D0B4
:10AC9000816941F008018161012A05D1816941F092
:10ACA000804141F0040181614EEA0B0004B0BDE82F
:10ACB000000FF0BD0146D0F8000E20F00300C1F8EF
:10ACC000000ED1F8040840F002020020C1F8042868
:10ACD0007047F0B503AF2DE9000BD2B042F2A800E7
:10ACE000C2F200000D9040F24F21C3F60651016000
:10ACF0004EF61A31C3F26A4141604AF66A01C4F263
:10AD00009421816047F68811C3F6F371C160002277
:10AD10000A9202744FF07C51019141614FF07E51D3
:10AD200003918161C2610262416281620021CBF6BE
:10AD300080710291C1620121069180F8301048F6BD
:10AD4000E803C0F602033BA90A46B3E87051A2E843
:10AD5000705193E8705182E8705147910621049137
:10AD600048913AAB0C934993499951914799489A24
:10AD7000343000F0E6F90D98403040F27C01C2F228
:10AD80000001A0221BF006FD0D98E03040F21C11DE
:10AD9000C2F20001B1E83C50A0E83C5091E83C50C0
:10ADA00080E83C5039A800F0E9F9019B029A069925
:10ADB000DDF828C0DDF80CE004460D98C0F810411D
:10ADC0004DF27D04C3F63354C0F8144148F2340404
:10ADD000CBF6B754C0F818414BF22D24C3F69D545E
:10ADE000C0F81C414CF6CD44C3F6CC54C0F8204109
:10ADF0004CF6CD44CBF64C64C0F824414AF24C6486
:10AE0000C3F68A54C0F8284144F26744C3F6296463
:10AE1000C0F82C4140F23B14C3F6AD64C0F8304199
:10AE200047F2A404C3F6BD64C0F8344147F6E124F8
:10AE3000C3F69464C0F838414CF28F24C3F67564AD
:10AE4000C0F83C41C0F840E1C0F84431C0F848C106
:10AE50004CF6CD44C3F64C74C0F84C41C0F850E1F8
:10AE6000C0F8542180F858C10023C4F22013C0F860
:10AE70005C31C0F860E1C0F864C1C0F868C1C0F8D6
:10AE80006CC1C0F87031C0F8742180F87811C0F836
:10AE90007C21C0F8802149F69A15C3F61975C0F8CF
:10AEA00084514FF07F55C0F88851C0F88CC1C0F86C
:10AEB00090C1C0F89441C0F898E1C0F89C2180F896
:10AEC000A0C140F2000EC4F2400EC0F8A4E140F26E
:10AED000000EC4F2A00ECDF814E0C0F8A8E140F2D4
:10AEE000000EC4F2200EC0F8ACE1C0F8B0C1C0F84A
:10AEF000B4C1C0F8B831C0F8BC2180F8C011C0F8A6
:10AF0000C421C0F8C82140F20922C0F8CC2140F287
:10AF1000FF23C0F8D031032280F8D42180F8D5C1B6
:10AF200080F8D6C140F20A2CC0F8D8C1C0F8DC3194
:10AF300080F8E02180F8E11180F8E21140F2474109
:10AF4000C4F21301389100F5F27038A900F01EF92F
:10AF50000D984CF2D641C4F22701379100F5F470F8
:10AF600037A900F013F90D980A99369100F5F6709B
:10AF700036A900F00BF90D984EF63311C4F23001EA
:10AF8000359100F5F87035A900F000F90D984AF6F2
:10AF90009841C3F6E871349100F5FA7034A900F0D5
:10AFA000F5F80D980A99339100F5FC7033A900F07B
:10AFB000EDF80D980A99329100F5FE7032A900F073
:10AFC000E5F80D98049948F6181CC0F6020C24AA5E
:10AFD0001346BCE87043A3E870439CE8704383E8E1
:10AFE00070433092319123AB0B934A934A9950911D
:10AFF0003099319A00F5007000F0A3F80D98059A89
:10B000000699C0F80C224AF22C02C4F29912C0F838
:10B0100010224CF28F22C3F6F542C0F814224FF0F2
:10B020007852C0F8182249F69A12C3F69952C0F81D
:10B030001C2280F820124FF08341C0F824124FF4F4
:10B040004871C0F8281200F50B7040F24C11C2F2A2
:10B050000001482207921BF09DFB0D9800F51D7022
:10B0600040F29411C2F2000178221BF093FB069982
:10B07000079A0A9B0D984FF4027CC0F8ECC240F28C
:10B08000FF1CC0F8F0C24FF0020C80F8F4C280F848
:10B09000F53280F8F61200F53E7040F20C21C2F253
:10B0A0000001B1E81850A0E8185091E8385080E845
:10B0B000385048F64811C0F602010FA808901BF05E
:10B0C00069FB08990D982191092122910EAB0993F2
:10B0D0004B934B994F912199229A00F5477000F0BC
:10B0E00030F809980A990D9A02F54A7340F2302C0B
:10B0F000C2F2000CBCE87040A3E870409CE87041CC
:10B1000083E8704182F84C134C904C9800F016FA8A
:10B110000B984D904D9800F011FA0C984E904E9867
:10B1200000F00CFA0D994BF2AF10C0F6000040F29F
:10B130000002C2F200021BF017FB52B0BDE8000B88
:10B14000F0BD80B56F468AB00992089107900693CA
:10B1500007980390069900F08BFC08A8019000F076
:10B16000D1FC01460198029100F0D2FC02990246FE
:10B17000039800F08AFC03980AB080BD81B000906B
:10B180004BF2D320C0F6000001B0704780B56F4687
:10B1900084B00390029103980190029890ED000A08
:10B1A00000F010F9019880ED000A04B080BD80B570
:10B1B0006F4682B001900198009000F5037000F096
:10B1C00025F9009800F58A7000F02DF9009800F03C
:10B1D00036F9009802B080BD80B56F46ADF5567D5A
:10B1E00042F2A801C2F2000102A8019000F045F865
:10B1F00001989FED050A00F009F80198FFF7D7FFC5
:10B200000DF5567D80BD00BF0000FA4380B56F4646
:10B21000ADF5627D02908DEDE10A1020F6F77CF825
:10B22000029A049009A80390E0A9E1AB00F03FFD69
:10B230000399049800F056FD039800F080FD0498EF
:10B24000DF9007A80590F6F782F80598DF996B461E
:10B2500004221A6047F66042C0F602024FF400630F
:10B2600000F079FD18F004FC012803D1FFE717F086
:10B2700075FEFFE70DF5627D80BDB0B502AF84B00D
:10B280000390029103980190029900F05CF90198F3
:10B2900000F58A70029901F58A7100F078F9019839
:10B2A00000F50370029901F5037100F090F901981F
:10B2B00000F54A72029901F54A71B1E81850A2E806
:10B2C0001850B1E83850A2E838500978117004B02D
:10B2D000B0BD80B56F4682B08DED010A9DED010ACB
:10B2E00000F002F802B080BD83B002908DED010A3B
:10B2F000002000909DED010A9FED2D1AB4EE410A49
:10B30000F1EE10FA06D8FFE74EF20000C4F2AB509F
:10B31000009049E09DED010A9FED261AB4EE410A26
:10B32000F1EE10FA06D8FFE74EF20000C4F2AB507F
:10B33000009038E09DED010A9FED1F1AB4EE410A1E
:10B34000F1EE10FA06D8FFE74EF20000C4F2AB505F
:10B35000009027E09DED010A9FED181AB4EE410A16
:10B36000F1EE10FA06D8FFE74CF20000C4F2C1502B
:10B37000009016E09DED010A9FED111AB4EE410A0E
:10B38000F1EE10FA06D8FFE74CF20000C4F2DA50F2
:10B39000009005E046F20000C4F2EA500090FFE79A
:10B3A000FFE7FFE7FFE7FFE79DED000A03B0704707
:10B3B000000048420000704200008C420000A042A1
:10B3C0000000C84280B56F4682B08DED010A9DED48
:10B3D000010ADFED0D0A19F0BBFB8DED010A9DEDB1
:10B3E000010AB5EE400AF1EE10FA09D5FFE79DED2E
:10B3F000010A9FED051A30EE010A8DED010AFFE703
:10B400009DED010A02B080BDDB0FC94080B56F46DB
:10B4100082B001900198009000F5887000F01BF850
:10B42000009802B080BD80B56F4682B0019001984F
:10B430000090EC3000F00FF8009802B080BD80B5AD
:10B440006F4682B0019001980090343000F003F80C
:10B45000009802B080BD80B56F4688B00490049813
:10B460000390016801914168029100F00FF8019A80
:10B4700002990792069105900798069900F01DF829
:10B48000039800F008F8039808B080BD81B00090E0
:10B49000009801B0704780B56F4682B00190019866
:10B4A000009001688268521AD21000F016F80098D5
:10B4B00000F02CF8009802B080BD80B56F4682B0D5
:10B4C000019000910198009900F002F802B080BD4F
:10B4D00082B00190009102B0704780B56F4688B08D
:10B4E00004900391029204980190039860B1FFE7E1
:10B4F000019A039902980792069105900798069978
:10B50000059A00F010F8FFE708B080BD80B56F46DF
:10B5100084B00290029801900390039800F00EF816
:10B52000019804B080BD80B56F4684B0039002914D
:10B5300001920298F5F7F9FE04B080BD81B0009049
:10B54000009801B07047B0B502AF84B0039002918B
:10B5500003980190029A0146B2E81850A1E81850E9
:10B56000B2E81850A1E8185092E8385081E83850F5
:10B5700034300299343100F041F80198403002999A
:10B580004031D4221BF006F9019804B0B0BD80B55B
:10B590006F4684B003900291039801900299D022E3
:10B5A0001BF0F8F80198D0300299D03100F0EDF995
:10B5B0000198DC300299DC3100F000FA0198EC309F
:10B5C0000299EC3100F01AF8019804B080BD80B502
:10B5D0006F4684B0039002910398019002994FF452
:10B5E00088721BF0D7F8019800F58870029901F570
:10B5F000887100F003F8019804B080BD80B56F46F3
:10B6000092B00890079108980390079800F037F8D7
:10B610000090079800F03CF800990346039806AAAA
:10B6200001920B920A930A9B0D920C930C9B0F9222
:10B630000E93DDF83CC00E9BCDF844C0109300F093
:10B640002CF8019809900998FFF778FF079800F007
:10B6500048F80590079800F04FF8014603980491C8
:10B6600001680291FFF712FF029A034605980499B8
:10B6700000F025F801460398416012B080BD81B00A
:10B680000090009801684068401AC01001B07047EF
:10B6900081B00090009801B0704780B56F4684B0CB
:10B6A00003900291019203980090019900F030F804
:10B6B0000098029900F03FF8009804B080BD80B572
:10B6C0006F4686B00590049103920293059801900D
:10B6D00004980090039A0198009900F081F806B050
:10B6E00080BD80B56F4682B00090009901A800F03F
:10B6F00043F9019802B080BD80B56F4682B00090DA
:10B700000098011D01A800F037F9019802B080BD32
:10B7100080B56F4688B0039002910398019002991A
:10B7200005900491059A04990792069100F018F883
:10B73000019808B080BD80B56F4684B00390029137
:10B7400003980190029900F014F8019908600868C4
:10B7500048600868029A00EBC200886004B080BDAF
:10B7600081B000900098002101604160816001B0CB
:10B77000704780B56F4686B00390029103980190A0
:10B78000029858B1FFE70199029805910490059835
:10B790000499002200F008F8009002E000200090D8
:10B7A000FFE7009806B080BD80B56F4684B0029078
:10B7B00001910092029901980391B0F1805F09D341
:10B7C000FFE70198B0F1005F02D3FFE718F055FFE3
:10B7D00018F050FF0198C000F5F79EFD04B080BD41
:10B7E00080B56F4686B0059004910392012007F85A
:10B7F0000D0C07F80E0C0598019004980090039A20
:10B800000198009900F002F806B080BD80B56F463F
:10B8100086B00590049103920598029004980190D7
:10B82000039A0298019900F002F806B080BD80B535
:10B830006F4688B007900691059207980390039889
:10B8400000F02EF8049006980190019800F028F876
:10B850000290059A0498029900F002F808B080BDA1
:10B8600080B56F4688B007900691059207980490BE
:10B87000049800F02FF8029006980390039800F0C7
:10B8800029F80190059800F02FF8019902460298D6
:10B8900000F013F8014605A800F009F808B080BDD3
:10B8A00082B0009000980190019802B0704782B079
:10B8B00001900091009802B0704780B56F4684B047
:10B8C00003900291019203980299019A00F011F8F5
:10B8D00004B080BD80B56F4682B0019001A800F031
:10B8E00046F8006802B080BD81B00090009801B0B9
:10B8F000704780B56F4684B003900291019203981F
:10B900000299019A00F002F804B080BD80B56F463C
:10B9100084B003900291019202980399401AC010DA
:10B9200000900098022807DBFFE701980399009A2E
:10B93000D200F4F76FFC09E00098012805D1FFE779
:10B940000198039900F008F8FFE7FFE701980099D4
:10B9500000EBC10004B080BD82B001900091009A5C
:10B960000199106852684A60086002B0704781B05F
:10B970000090009801B0704782B00190009101984A
:10B9800000990968016002B0704780B56F4684B0C5
:10B990000390029103980190029900F02FF801980A
:10B9A00004300299043100F029F801980830029916
:10B9B000083100F023F8019804B080BD80B56F46CF
:10B9C00084B00390029103980190029900F016F858
:10B9D000019804300299043100F010F80198083001
:10B9E0000299083100F00AF801980C3002990C31E4
:10B9F00000F004F8019804B080BD000084B002900B
:10BA00000191029900910391019800680860FFE795
:10BA1000009890ED000A9FED141AB4EE410AF1EE81
:10BA200010FA0ADBFFE7009890ED000A9FED0F1A6D
:10BA300030EE010A80ED000AEAE7FFE7009890ED9A
:10BA4000000AB5EE400AF1EE10FA0AD5FFE70098B9
:10BA500090ED000A9FED041A30EE010A80ED000A15
:10BA6000ECE7039804B07047DB0FC940DB0FC9C097
:10BA700080B56F4684B003900291039801900299BB
:10BA8000FFF746FE019804B080BD80B56F4690B0C8
:10BA900009900891079209980590089A07990C92C5
:10BAA0000B910C9A0B990CAB0F930E920D910D9973
:10BAB0000E9A891AC910069106990191FFF7E6FCC2
:10BAC0000146019800F037F801460598FFF751FE4E
:10BAD0000146059801600168069A01EBC201816088
:10BAE000089904910799029101680391FFF7CEFC30
:10BAF0000299039A0346049800F044F805994860B7
:10BB000010B080BD81B000900098006801B070470F
:10BB100080B56F4684B0039003980190FFF7F2FF61
:10BB200001460198029100F0BCF80146029800EB32
:10BB3000C10004B080BD80B56F468CB00690059101
:10BB400006980290059904A8019009900891099A15
:10BB500008990B920A9100F023F80146019803918D
:10BB600007900798FFF7EAFC02980399884206D9E4
:10BB7000FFE747F62F40C0F6020018F087FD069851
:10BB80000CB080BD80B56F4684B0039002910192E5
:10BB9000009303980299019A00F02AF804B080BD3E
:10BBA00080B56F4686B002906FF0704001900299A8
:10BBB00003910399049104990591009001A86946A5
:10BBC00000F003F8006806B080BD83B001900091DA
:10BBD0000098006801990968884203D2FFE700983D
:10BBE000029002E001980290FFE7029803B07047CC
:10BBF00080B56F4684B0039002910192012007F84E
:10BC00000D0C07F80E0C03980299019A00F002F847
:10BC100004B080BD80B56F4684B00390029101925C
:10BC200003980299019A00F002F804B080BD80B533
:10BC30006F4684B0039002910192039800F027F8B8
:10BC40000090029800F023F801460098019A00F055
:10BC500002F804B080BD80B56F4686B005900491AF
:10BC60000392059800F018F80290049800F014F878
:10BC700001900398FFF738FE019902460298FFF7FA
:10BC80001CFE014603A8FFF712FE06B080BD81B07E
:10BC90000090009801B0704781B00090009801B00A
:10BCA000704781B000900098406801B0704780B53F
:10BCB0006F4688B00390079006910592049306980A
:10BCC00000F082F80190059800F083F80290049843
:10BCD00000F084F80199029A0346039800F083F873
:10BCE00008B080BD80B56F4686B00490039104987B
:10BCF000029005900021019181604160016000F097
:10BD0000F1F801980299C860039800F0F3F898B12F
:10BD1000FFE7039800F003F90146029800F0EFF8FE
:10BD200002994BF62970C0F60000C8604BF63F70D0
:10BD3000C0F600008860FFE7059806B080BD80B5BA
:10BD40006F4682B0019001980090043000F0A3FC8F
:10BD5000009802B080BD80B56F468EB08446B8684A
:10BD6000CDF830C00B910A92099307F8150C0C9886
:10BD700004900DA8039000F0B0FC082015F07EFEA2
:10BD800001460398079100F0A8FC01460B9A05A80C
:10BD900000F0ABFCDDF810E007990598069A4A60C0
:10BDA0000860079B0A99BDF8242017F8150CEC468B
:10BDB000CCF804E0CCF800004CF20170C0F60000B2
:10BDC00016F034FD0EB080BD81B00090009801B037
:10BDD000704781B00090009801B0704781B000902A
:10BDE000009801B0704780B56F4688B00790069103
:10BDF0000592049307980390043002900598FFF78A
:10BE0000E8FF01900498FFF7E9FF019902460298C4
:10BE100000F003F8039808B080BD80B56F4686B087
:10BE2000059004910392059802900498FFF7D1FFC2
:10BE300001900398FFF7D2FF01990246029800F0A3
:10BE400003F8029806B080BD80B56F4686B00590B5
:10BE500004910392059802900398FFF7BFFF0146F3
:10BE6000029800F00DF80298043001900498FFF752
:10BE7000B0FF0146019800F014F8029806B080BDAA
:10BE800080B56F4684B003900291039801900298A8
:10BE9000FFF7A4FF0146019800F014F8019804B0E0
:10BEA00080BD80B56F4684B00390029103980190E5
:10BEB0000298FFF78EFF01460198FFF7DEF901981F
:10BEC00004B080BD80B56F4684B0039002910398A2
:10BED00001900298FFF782FF01460198096801600E
:10BEE00004B080BD81B000900098002101608160A5
:10BEF00001B0704781B00090012001B0704780B55B
:10BF00006F4684B00390029103980090029800F06D
:10BF100006F80146009800F033F804B080BD81B007
:10BF20000090009801B0704780B56F4682B00190D4
:10BF3000019800F05BF900F04EF902B080BD80B5C9
:10BF40006F4684B00390029107F8092C17F8090C8A
:10BF500001280BD1FFE7029800F048F90090039800
:10BF600000F036F801460098086006E00398029950
:10BF700017F8092C00F0D4FAFFE7002004B080BDC8
:10BF800080B56F4684B0029001914FF45670F5F77A
:10BF9000C3F900900198FFF7C2FF0146009800F036
:10BFA00008F8029800F014F801460098086004B000
:10BFB00080BD80B56F4684B00390029103980190D4
:10BFC00002990430043100F00CF8019804B080BDEF
:10BFD00080B56F4682B00190019800F0F7F802B08A
:10BFE00080BD80B56F4684B00390029103980190A4
:10BFF000029900F003F8019804B080BD80B56F4647
:10C0000084B00390029103980190029900F009F81E
:10C01000019804300299043100F00CF8019804B042
:10C0200080BD82B00190009101980099096801607B
:10C0300002B0704780B56F4684B0039002910398B8
:10C040000190029900F003F8019804B080BDB0B5EA
:10C0500002AF84B00390029103980190029900F01E
:10C0600022F8019800F58A70029901F58A7100F0B2
:10C070003EF8019800F50370029901F5037100F094
:10C0800056F8019800F54A72029901F54A71B1E833
:10C090001850A2E81850B1E83850A2E83850097892
:10C0A000117004B0B0BDB0B502AF84B0039002917E
:10C0B00003980190029A0146B2E81850A1E818507E
:10C0C000B2E81850A1E8185092E8385081E838508A
:10C0D000343002993431FFF791FA019840300299D7
:10C0E0004031D4221AF056FB019804B0B0BD80B59F
:10C0F0006F4684B003900291039801900299D02278
:10C100001AF048FB0198D0300299D03100F026F89F
:10C110000198DC300299DC3100F039F80198EC30FC
:10C120000299EC31FFF76AFA019804B080BD80B53E
:10C130006F4684B0039002910398019002994FF4E6
:10C1400088721AF027FB019800F58870029901F5B2
:10C150008871FFF753FA019804B080BD80B56F462F
:10C1600084B003900291039801900299FFF746FC76
:10C170000198043002990431FFF740FC019808301F
:10C1800002990831FFF73AFC019804B080BD80B5F0
:10C190006F4684B003900291039801900299FFF7D3
:10C1A0002DFC0198043002990431FFF727FC019817
:10C1B000083002990831FFF721FC01980C300299F0
:10C1C0000C31FFF71BFC019804B080BD81B00090DA
:10C1D000009801B0704780B56F4682B00190019819
:10C1E00000F019F800F00CF802B080BD80B56F4681
:10C1F00082B00190019800F085F9006802B080BD1E
:10C2000080B56F4682B00090009800F004F800F00E
:10C2100007F802B080BD81B00090009801B070476F
:10C2200080B56F4686B005900598019000F027F81C
:10C23000019804A900F002F806B080BD80B56F46F1
:10C2400088B006900591069802900430009000F0A6
:10C250003AF80146059A04A800F02AF80146009829
:10C26000019100F044F80146059A03A800F034F863
:10C2700001990246029800F003F808B080BD7047AB
:10C2800080B56F4686B00590049103920598FFF73C
:10C290009BFD01900498FFF79CFD00900398FFF729
:10C2A0009DFD00990246019800F02AF806B080BD75
:10C2B00080B56F4684B00390029101920298FFF717
:10C2C00088FD04B080BD80B56F4682B001900198B2
:10C2D00000F0E9F802B080BD80B56F4684B00390ED
:10C2E000029101920298FFF779FD04B080BD80B5FC
:10C2F0006F4682B00190019800F0EDF802B080BD69
:10C3000080B56F46ADF55A7DD890D791D692D89822
:10C31000FFF75AFD0090D798FFF75BFD014602A892
:10C320000190FEF7AAFFD698FFF758FD0199024643
:10C33000009892ED000A00F006F80198FEF737FF2A
:10C340000DF55A7D80BD80B56F468AB00291099087
:10C350008DED080A0120039015F090FB07900798D7
:10C3600000F03AF8039815F089FB06900698F5F767
:10C3700024F8039815F082FB05900598F4F7D0FE99
:10C380000C2015F07BFB04900498F5F705FB42F2B6
:10C39000FC30C2F200000078C007B8B9FFE741F6F0
:10C3A0001800F4F7B9FF029901909DED080A00F01A
:10C3B0001EF8019842F2F831C2F20001086042F220
:10C3C000FC31C2F2000101200870FFE7FFE74FF0E7
:10C3D000FF30F5F7D1FAFAE780B56F4682B00190E9
:10C3E00001980090F6F7CEFB009802B080BD80B5B2
:10C3F0006F4686B0059004918DED030A0598029072
:10C40000002101910DF06EFD02980199F83006F0BF
:10C410002EF9029800F5896004F0EBFF029800F510
:10C420009A60049901F54A7107F0E4FD029800F260
:10C430004C5008F0AAFE029800F5AA600CF054FADD
:10C44000029800F51960049901F5537109F091F80B
:10C45000029800F522600AF080F9029800F6B420F4
:10C4600001210BF046FC029800F6B82004999DEDDE
:10C47000030A00F083F9029800F57360049901F54E
:10C480008A719DED030A01F0AEFE029841F2E83197
:10C490000844049901F503719DED030A02F0FDFFC4
:10C4A000029806B080BD80B56F4682B001900198B9
:10C4B00000F002F802B080BD80B56F4682B00190F6
:10C4C0000198043000F002F802B080BD81B0009005
:10C4D000009801B0704780B56F4682B00190019816
:10C4E00000F002F802B080BD80B56F4682B00190C6
:10C4F000019800F002F802B080BD81B00090009871
:10C5000001B0704780B56F4682B00190019800F08D
:10C5100002F802B080BD81B00090009801B0704771
:10C5200080B56F4686B00590049107F8092C17F87E
:10C53000090C01460291032824D80299DFE801F092
:10C540000209141E059800F020F80146002008603A
:10C5500018E00498FFF74AFE01900598FFF738FDB0
:10C560000146019808600DE0059800900498FFF7D7
:10C570003DFE0146009800F011F803E0059800F038
:10C580001DF8FFE7002006B080BD80B56F4682B081
:10C5900001900198FFF71AFE02B080BD80B56F468A
:10C5A00084B00390029103980090029800F033F851
:10C5B0000146009800F016F804B080BD80B56F46C3
:10C5C00084B002900298FFF703FD0068019038B133
:10C5D000FFE70198FFF7B3FB0198F4F7A6FEFFE72A
:10C5E00004B080BD80B56F4684B0029001914FF4D5
:10C5F0005670F4F791FE0090019800F00CF8014697
:10C60000009800F00DF80298FFF7E2FC0146009850
:10C61000086004B080BD81B00090009801B0704700
:10C6200080B56F4684B003900291039801900299FF
:10C630000430043100F003F8019804B080BD80B5E7
:10C640006F4684B00390029103980190029900F024
:10C6500003F8019804B080BD80B56F4684B00390A4
:10C660000291039801900299096840F8041B02990D
:10C67000043100F003F8019804B080BD80B56F4626
:10C6800084B003900291039801900299FEF7F5FDA2
:10C69000019804B080BD80B56F4682B001900198CA
:10C6A000009000F003F8009802B080BD80B56F469E
:10C6B00082B0019001980090043000F003F80098D7
:10C6C00002B080BD80B56F4682B0019001980090A5
:10C6D000FEF76DFD009802B080BD81B000904CF275
:10C6E0001970C0F6000001B0704783B0029001914C
:10C6F00000920298019901600099416003B070476F
:10C7000080B56F4682B00190019800900098016852
:10C710004068884702B080BD80B56F4682B0019006
:10C72000019900F002F802B080BD80B56F4682B07A
:10C7300001900091009800F002F802B080BD80B531
:10C740006F4682B001900198009000F009F810B196
:10C75000FFE717F0A5FF0098C168884702B080BDC9
:10C7600081B0009000988068B0FA80F0400901B074
:10C77000704780B56F46FEF7ACFA80BD80B56F4656
:10C78000A8B0239022918DED210A2398089024903F
:10C790002299FEF7D8FE089800210991C0F81411DB
:10C7A000C0F81811C0F82411C0F82011C0F82C11DD
:10C7B000C0F8281180F8401100F5C2702299097C58
:10C7C0000EF08AF9089800F5DE70229914319DED7B
:10C7D000210A0EF05CFB089800F50470F4F7B7FD31
:10C7E000089800F50570012100F0B8F8089809993B
:10C7F00000F21C400C2219F0ECFE099807F81D0C01
:10C80000FFE7089917F81D0C91F88511884265DA41
:10C81000FFE79420F4F780FD01902298403017F84C
:10C820001D1C00F0ACF8014601989DED210A0DF0A9
:10C830004DFA089800F5B27017F81D1C00F0BAF810
:10C840000146019808607820F4F766FD039022986D
:10C85000E03017F81D1C00F0C6F8029013AA0792EA
:10C8600025922598279047F66F41C0F6020114A83B
:10C87000069000F01EF917F81D1C0DA8059000F099
:10C8800040F9059A06991AA8049000F0C7F8049890
:10C8900018F01AF90299024603980BF05FFB08980A
:10C8A00000F5BA7017F81D1C00F072F903990246E2
:10C8B0000498116017F0ABFF059817F0A8FF0698D1
:10C8C00017F0A5FF07982690269801F0C3F9FFE717
:10C8D00017F81D0C013007F81D0C92E7089890F826
:10C8E0008501800000F06DF901460898C0F89811A4
:10C8F000D0F8980140B9FFE747F67840C0F602004B
:10C90000432100F067F9FFE70CA800F0C1F908998E
:10C9100001F1340200F06EF9089901F504706B46DC
:10C9200002221A6047F6CB42C0F602024FF4C073EF
:10C9300000F0B6F908994CF67D50C0F6000040F6BC
:10C94000340200F0E6F908994CF6CD70C0F600000C
:10C95000C82200F0DEF9249828B080BD80B56F466B
:10C9600084B0039002910398019002994FF0FF3038
:10C9700015F0A2FA01460198016004B080BD80B5AF
:10C980006F4684B0039002910398019002980428A6
:10C9900008D3FFE7029947F6F740C0F602000422E9
:10C9A00017F07AFE0198029901EB810100EBC100BA
:10C9B00004B080BD80B56F4684B0039002910398A7
:10C9C00001900298042808D3FFE7029947F6F74040
:10C9D000C0F60200042217F05FFE0198029900EBF6
:10C9E000810004B080BD80B56F4684B00390029191
:10C9F000039801900298042808D3FFE7029947F6AC
:10CA0000F740C0F60200042217F046FE0198029992
:10CA100001EB410100EB810004B080BD80B56F46A1
:10CA20008AB00490099008910792002007F80D0C35
:10CA3000012007F80D0C17F80D0CC00760B3FFE7D5
:10CA4000089817F0EAFE0290079817F0E6FE0146F4
:10CA500002980844059005980390089817F0DFFEA7
:10CA600001460398884216D9FFE705980190079878
:10CA700017F0D5FE0146019888420CD8FFE70798C9
:10CA8000089A002117F0CCFF01F04EF901460498F6
:10CA900017F09EFE0BE0FFE70898079918F00EF8D4
:10CAA00001F042F90146049817F092FEFFE70AB040
:10CAB00080BD80B56F4688B00790069105920798B3
:10CAC000029017F001FE01460298059A17F0FEFF4A
:10CAD000069830B9FFE747F60C60C0F6020017F081
:10CAE000CFFD0698019001F0BAF80199024602982C
:10CAF000114404910699049A01F0BAF8029808B01A
:10CB000080BD80B56F468CB002900B900A910A9858
:10CB1000C00F07F8090C17F8090CC00720B1FFE790
:10CB20000A984042019002E00A980190FFE70198BC
:10CB3000089008980A2100F0F3FE01460298079138
:10CB4000002107F8151C17F03CFE029817F8092C75
:10CB5000079902F0010211448DF80C20079A049203
:10CB6000089A0592039A049BDDF814C0EE46CEF8AD
:10CB700000C000F015FF012007F8150C17F8150C80
:10CB800020B9FFE7029817F042FEFFE70CB080BD26
:10CB900080B56F4684B0039002910398019002988B
:10CBA000042808D3FFE7029947F6F740C0F60200D1
:10CBB000042217F071FD0198029900EB810004B086
:10CBC00080BD80B56F4682B00190019814F056FF89
:10CBD00002B080BD80B56F4682B001900091FFE742
:10CBE000FFE70199009A47F6F450C0F60200F4F707
:10CBF000BEFBF6E780B56F468EB00D900C910B92A0
:10CC000009A801F096F80B98FEF76BFD08900898BC
:10CC10000990FFE70B98FEF76FFD079009A807A999
:10CC200001F08EF890B3FFE70C20FFF7CAFF0690E3
:10CC30000C98069988600D980699486009A802909A
:10CC400001F093F8014602984968069A116042F291
:10CC5000CC61C2F2000109680431049101F085F849
:10CC6000006803900AA801F0A2F80399034604980B
:10CC7000069AEC46CCF80020012201F07CF8FFE790
:10CC800009A8002101F09BF80590C3E70EB080BD14
:10CC900081B000904DF6F720C0F6000001B070475B
:10CCA00080B56F468EB08446B868CDF830C00B9121
:10CCB0000A92099307F8150C0C9804900DA803909C
:10CCC00001F0A9F8082014F0D9FE01460398079155
:10CCD00001F0A1F801460B9A05A801F0A4F8DDF8CF
:10CCE00010E007990598069A4A600860079B0A9920
:10CCF000BDF8242017F8150CEC46CCF804E0CCF86D
:10CD000000004DF63D60C0F6000015F08FFD0EB03E
:10CD100080BD80B56F4688B00790069105920820C7
:10CD200014F0ACFE04900799069A02A801F07BF873
:10CD300004990298039A4A6008601420F4F7ECFA08
:10CD40000190019900204881059801990881019975
:10CD50004DF63D60C0F600004860049801990860F7
:10CD600001990120087340F2D070C2F200000068FF
:10CD7000019901F022FA019808B080BDF0B503AF27
:10CD80002DE9000FB9B03890389800F58560119002
:10CD900000F0A6FD9FED8B1A20EE010ABDEEC00A41
:10CDA00010EE100A109000F0A1FD109B11989FED5D
:10CDB000861A20EE010ABDEEC00A10EE101A47F6E0
:10CDC000DD4CC0F6020C6A46C2F818C0136102239B
:10CDD000D3604FF0500CC2F808C04FF00A0CC2F8F4
:10CDE00004C01360516147F6DA41C0F60201012226
:10CDF000002314930FF099F9389800F585612CA859
:10CE0000129000F079FD129920A82D2219F0C2FC91
:10CE100020982199229A239BDDF890C0259C269D7D
:10CE2000279EDDF8A080DDF8A490DDF8A8A0DDF84D
:10CE3000ACB0EE46CDF84CE0CEF81CB0CEF818A061
:10CE4000CEF81490CEF81080CEF80C60CEF80850D2
:10CE5000CEF80440CEF800C00CF063FD14981F908B
:10CE60001E90389890F8400101461591042821D869
:10CE70001599DFE801F01E1E030C15000020C4F216
:10CE800058201F900020C4F2CC201E9016E00020F5
:10CE9000C4F22E301F900020C4F25E301E900DE0D0
:10CEA0000020C4F2E4201F900020C4F222301E9023
:10CEB00004E0FFE700201F901E90FFE79DED1F0A92
:10CEC000B5EE400AF1EE10FA78D0FFE79DED1E0AAC
:10CED000B5EE400AF1EE10FA70D0FFE7389800F294
:10CEE00064400D9000F0FCFC9DED1F1A9FED352A6B
:10CEF0008DED092A20EE020A30EE010ABDEEC00ACD
:10CF000010EE100A0C9000F0F1FC9FED2F1A8DED41
:10CF10000A1A20EE010AB1EE001A30EE010ABDEE47
:10CF2000C00A10EE100A0B9000F0DAFC9DED092A01
:10CF30009DED1E1A20EE020A30EE010ABDEEC00A77
:10CF400010EE100A0E9000F0D1FC9DED0A1A0B9B1A
:10CF50000C9A0D98DDF838E020EE010ABAEE0C1AB2
:10CF600030EE010ABDEEC00A10EE101AEC46CCF805
:10CF700010E0CCF80C30CCF808200122CCF80420CA
:10CF80000223CCF80030CCF8141047F6F441C0F678
:10CF900002010EF007FC389800F264411AA80F90C5
:10CFA00000F0B4FC0F9916A80F2219F0F3FB1698A5
:10CFB0001799189A199B0CF03AFCFFE739B0BDE8B5
:10CFC000000FF0BD9A99593F3333333F80B56F4618
:10CFD0009AB01990002018901790199890F8400175
:10CFE00001460E9102281AD3FFE70E98022804D0BA
:10CFF000FFE70E98032809D012E00020C4F2582061
:10D0000018900020C4F2CC2017900DE00020C4F24C
:10D010002E3018900020C4F25E30179004E0FFE735
:10D02000002018901790FFE79DED180AB5EE400A12
:10D03000F1EE10FA76D0FFE79DED170AB5EE400A43
:10D04000F1EE10FA6ED0FFE7199800F264400B90F1
:10D0500000F046FC9DED181A9FED332A8DED072A4E
:10D0600020EE020A30EE010ABDEEC00A10EE100AF0
:10D070000A9000F03BFC9FED2D1A8DED081A20EE72
:10D08000010AB1EE001A30EE010ABDEEC00A10EE40
:10D09000100A099000F024FC9DED072A9DED171A57
:10D0A00020EE020A30EE010ABDEEC00A10EE100AB0
:10D0B0000C9000F01BFC9DED081ADDF824C00A9BC3
:10D0C0000B98DDF830E020EE010ABAEE0C1A30EED3
:10D0D000010ABDEEC00A10EE101A6A46C2F810E04E
:10D0E000C2F80CC0936001235360022313605161A6
:10D0F00047F6F441C0F602011A460EF053FB1998A8
:10D1000000F2644113A80D9000F000FC0D990FA8E7
:10D110000F2219F03FFB0F981099119A129B0CF0F7
:10D1200086FBFFE71AB080BD9A99593F3333333FEE
:10D1300080B56F4684B00390039801900020029060
:10D14000FFE70199029891F8851188421DD2FFE707
:10D15000019800F5BA700090029900F018F8006884
:10D160000168496888470098029900F010F8006843
:10D1700000F016F80198029900EB810080ED670A33
:10D18000FFE7029801300290DBE704B080BD82B077
:10D19000019000910198009900EB810002B0704766
:10D1A00083B001900198009090F83400C00740B11E
:10D1B000FFE7009890ED090AB1EE400A8DED020AF2
:10D1C00003E00098406A0290FFE79DED020A03B079
:10D1D000704700000000000080B56F4698B01790BF
:10D1E00017980D90F7F795FD0A460D99C1F82C2177
:10D1F000C1F82801D1F82031D1F82421D1F8280133
:10D20000D1F82C11C01A9141F3F774FE01460D9824
:10D2100000EE101A9FEDDF1A80EE010A80ED460A3B
:10D22000D0F82811D0F82C21C0F82421C0F8201102
:10D2300090ED4D0A00F0D4F901460D9800EE101A59
:10D24000B8EE400A80ED450A90F8400101460E9183
:10D2500004284AD80E99DFE801F0140314140A00D8
:10D260000D990020C1F88801C1F88C013EE00D99AC
:10D27000D1F81C04C1F88801D1F82004C1F88C0150
:10D2800034E00D98D0F8180216909DED160A17F0AC
:10D29000B1FC8DED150A9DED160A17F0F1FC0D9805
:10D2A0008DED140A9DED150A00F21C419DED141A36
:10D2B00091ED002A91ED013A21EE031A20EE020AC7
:10D2C00030EE410A80ED620A9DED140A9DED151ABB
:10D2D00091ED002A91ED013A21EE031A20EE020AA7
:10D2E00030EE010A80ED630A00E0FFE70D9890F848
:10D2F000400101460C9104282FD80C99DFE801F079
:10D300000303091803000D99D1F82404C1F8900112
:10D310002BE00D9901F5DE7091ED461AD1ED860AEC
:10D320009FEDAE0A0DF020FE0D9880ED640A1CE022
:10D330000D9890ED650A8DED0B0A9FEDA70AF7EEAB
:10D34000000A00F06FF90D98B0EE401A9DED0B0A3F
:10D3500020EE010A80ED640A07E047F67840C0F647
:10D360000200EC21FFF736FC2FE10D9A02F5C270A6
:10D3700002F5C471D2F898210DF0FEFB0D9890F8DB
:10D38000400101460A91002800F0F980FFE70A9861
:10D390000138032800F21081FFE70D980021139156
:10D3A00090F8300101281AD1FFE70D9890ED4E0A50
:10D3B000B3EE0E1AB4EE410AF1EE10FA04DDFFE707
:10D3C0004FF07E50139009E00D9890ED4E0AB3EEA9
:10D3D0000E1A80EE010A8DED130AFFE703E04FF00D
:10D3E0007E501390FFE713A89FED7C0AF7EE000A2A
:10D3F0000FF02FF90D99D1F83401D1F850110491A3
:10D40000F3F730F941EC100B9FED711B53EC112B2E
:10D4100051EC100B09910890F3F77CF9024604983F
:10D4200005920A46059942EC101B8DED060BF3F7A9
:10D4300019F99DED061B41EC100B51EC110B53EC4F
:10D44000102BF3F767F9089A099B41EC100B51EC8C
:10D45000100BF2F7A9FF41EC100B51EC100BF3F796
:10D4600031FC129000201190FFE70D99119891F86E
:10D470008511884233D2FFE70D9800F5B2701199FB
:10D4800000F002F901460D9809680291D0F8982140
:10D49000119902EB810292ED000A90ED451A20EEFF
:10D4A000010A8DED030A00F5BA70FFF770FE0068FF
:10D4B000FFF776FE02980D99F0EE400A9DED030A03
:10D4C00091ED461A0CF025FC0D98119900EB8100A6
:10D4D00080ED6B0AFFE7119801301190C5E700203D
:10D4E0001090FFE70D99109891F88511884245D268
:10D4F000FFE70D9890F86001C007E8B1FFE70D98CD
:10D500009DED120A00F5D671019100F5CE7290F8EA
:10D51000853100F0C2F80D9800F5BA701099FFF748
:10D5200036FE01990068109A01EB820191ED000A24
:10D530000168096888471CE00D9890ED4D0A00F5D8
:10D54000D671009100F5CE7290F8853100F0A5F803
:10D550000D9800F5BA701099FFF719FE0099006850
:10D56000109A01EB820191ED000A01680968884771
:10D57000FFE7FFE7109801301090B3E725E00020A7
:10D580000F90FFE70D990F9891F88511884212D2FC
:10D5900002E000BF002474490D9800F5BA700F999D
:10D5A000FFF7F5FD0068016889688847FFE70F9875
:10D5B00001300F90E6E708E047F67840C0F6020039
:10D5C00040F22B11FFF706FBFFE718B080BD00BF4C
:10D5D000666666666666EE3FCDCC4C3F0000000096
:10D5E00080B56F4684B002908DED010A02980090DC
:10D5F000D0F8100168B1FFE70098D0F810019DED58
:10D60000010A8047BDEEC00A10EE100A27F8020C8E
:10D6100004E041F2883027F8020CFFE737F8020CEB
:10D6200004B080BD80B56F4684B003908DED020AD2
:10D63000CDED010A0399D1F82801D1F82C11F3F7A7
:10D6400059FC00EE100A9FED0E1A20EE010A17F0A9
:10D6500017FB9FED0C1A20EE010A17F003FB9DED5E
:10D66000021A30EE010A8DED000A9DED020ADDED91
:10D67000010A68460EF0EDFF9DED000A04B080BD82
:10D680000AD7233BCDCC4C3E82B00190009101984B
:10D69000009900EB810002B0704780B56F4690B0F2
:10D6A0000E908DED0D0A0C910B920A930E9802903C
:10D6B0009DED0D0AB5EE400AF1EE10FA04D5FFE734
:10D6C000002007F8010C91E0002009900490FFE78A
:10D6D00004980A99884254D2FFE7029890ED000A14
:10D6E0008DED000A0C98049900EB810090ED000A82
:10D6F00017F0B8FAB0EE401A9DED000A20EE010ACC
:10D700008DED010A0B98049900EB810090ED000A61
:10D7100017F0A8FA02989DED011AB0EE403A0B9A64
:10D72000049902EB810292ED004A90ED012A90EDFE
:10D73000020A22EE042A22EE042A21EE031A31EE16
:10D74000021A0C9800EB810090ED002A20EE020AEC
:10D7500020EE020A30EE010A05A800EB810181EDFE
:10D76000000A049900EB810090ED001A9DED090A72
:10D7700030EE010A8DED090AFFE7049801300490AC
:10D78000A6E7029890ED031A9DED090A30EE010A12
:10D790008DED090A9DED090A9DED0D1AB4EE410AC1
:10D7A000F1EE10FA1EDDFFE700200390FFE703987B
:10D7B0000A99884215D2FFE79DED0D0A9DED091AE1
:10D7C00080EE011A0C98039900EB810090ED000A9D
:10D7D00020EE010A80ED000AFFE703980130039074
:10D7E000E5E7FFE7012007F8010CFFE717F8010C58
:10D7F00010B080BD80B56F4684B0039007F8051C5B
:10D800000399009117F8050C91F84011884201D155
:10D81000FFE742E017F8050C032820D1FFE7009846
:10D8200090F8400103281AD0FFE70098D0F82801AB
:10D8300018F0F2FC18F01EFD0146009801EBD172C1
:10D8400022F001028A1A0121002A18BF4FF0FF318D
:10D8500000EE101AB8EEC00A80ED650AFFE700205E
:10D860000190FFE70099019891F8851188420ED246
:10D87000FFE7009800F5B2700199FFF705FF006817
:10D880000CF070FAFFE7019801300190EAE7009987
:10D8900017F8050C81F84001FFE704B080BD81B0A6
:10D8A0000090009991F8610291F8622240EA02200A
:10D8B00000EE100AB8EE400A81ED4D0AB1F86C0294
:10D8C00000EE100AB8EE400A81ED4E0AD1F8680267
:10D8D000C1F83C0191F81C0281F8300101B0704799
:10D8E0009FED010A704700BF0000F0449FED010A60
:10D8F000704700BF0000874480B56F4682B0019139
:10D9000001992D2218F046FF02B080BD80B56F4608
:10D9100082B0019101990F2218F03CFF02B080BD46
:10D9200087B0059004910120039004984043029031
:10D930000298049948430190019804994843009043
:10D94000FFE705980499884203D2FFE70398069001
:10D9500023E005980299884204D2FFE7039801303A
:10D9600006901AE005980199884204D2FFE70398CF
:10D970000230069011E005980099884204D2FFE732
:10D9800003980330069008E000990598B0FBF1F089
:10D990000590039804300390D3E7069807B07047CA
:10D9A00080B56F468AB0D7F808C0CDF824C0089378
:10D9B00007920690059106980090059916F070FF61
:10D9C000009816F07FFE0146009804910290002016
:10D9D000039007A800F011F80499059A00F012F8D6
:10D9E00001900198039003980599884200D9FFE7B8
:10D9F00002A800F01DF80AB080BD81B00090009828
:10DA000001B0704780B56F4684B0039002910192D7
:10DA1000039A02992D2008700298117801F00101F3
:10DA200008445168926800F010F8019804B080BD75
:10DA300080B56F4682B001900199009108684968ED
:10DA400016F046FE009802B080BD80B56F46BAB0B1
:10DA500039903891379247F62B51C0F60201A7F161
:10DA6000D500C92218F096FE389801380390FFE7D8
:10DA70003798642825D3FFE7379B48F21F51C5F23A
:10DA8000EB11A3FB01204009642200FB123040008F
:10DA900002903798A0FB0110400937900299A7F136
:10DAA000D50001444978399A039BD1540299405CCE
:10DAB000399A0399114401F8010C03980238039034
:10DAC000D6E737980A280FD3FFE737984000019030
:10DAD0000199A7F1D50001444978399A517001990B
:10DAE000405C3999087004E03798303039990870F3
:10DAF000FFE73AB080BD80B56F4682B007F8010CF1
:10DB0000009117F8011C009A00F002F802B080BDE5
:10DB100080B56F4684B0039007F8051C0192019808
:10DB200000F505704FF0FF3100F027F817F8050CED
:10DB300001460091032818D80099DFE801F0020798
:10DB40000C1101980021FFF755FE0FE0019802210A
:10DB5000FFF750FE0AE001980321FFF74BFE05E0B6
:10DB600001980421FFF746FE00E0FFE7019800F569
:10DB7000057000F042F804B080BD80B56F4688B0F3
:10DB80000590049105980190EFF3058007900798A0
:10DB900060B9FFE701980068049914F0C3FC0138EC
:10DBA000B0FA80F0400907F8050C22E00198002146
:10DBB0000391006803AA14F09DFD0138B0FA80F0CB
:10DBC00040090290039860B1FFE74EF60451CEF28F
:10DBD00000014FF080500860BFF34F8FBFF36F8F8D
:10DBE000FFE702980138B0FA80F0400907F8050C09
:10DBF000FFE717F8050C08B080BD80B56F4684B00C
:10DC0000029002980090EFF3058003900398B8B15A
:10DC1000FFE7009800210191006801A914F03EFB84
:10DC2000019860B1FFE74EF60451CEF200014FF0CB
:10DC300080500860BFF34F8FBFF36F8FFFE707E09F
:10DC400000980068002319461A4614F051F9FFE7BE
:10DC500004B080BD81B00090009801B0704780B5DD
:10DC60006F4682B001900198F2F742FB02B080BD8E
:10DC700080B56F468EB0069005910492069801908B
:10DC800005990498099108900999089809AA0D9294
:10DC90000C910B900B980C99401A03900398102844
:10DCA0000ED3FFE7019803A9002216F01DFD0146DF
:10DCB000019816F005FD0198039916F007FD02E0A2
:10DCC00001980A90FFE7019902A8009000F012F86D
:10DCD000019816F0F7FC0599049A16F06DFD01986D
:10DCE00000210291039916F0F3FC009800F00AF865
:10DCF0000EB080BD82B00190009101980099016042
:10DD000002B0704780B56F4684B0029002980190CF
:10DD10000390006828B1FFE70198006816F002FD43
:10DD2000FFE7039804B080BD81B00090009801B077
:10DD3000704781B0009000980021016001B07047E9
:10DD400080B56F4684B0039002910398FDF70FFEF3
:10DD5000006801900298FDF70AFE014601980968E3
:10DD6000401A18BF012004B080BD81B00090009817
:10DD7000006801B0704780B56F4686B0D7F808C01C
:10DD80000590049107F8092C0293059800680499FE
:10DD900017F8092C029BD7F808C0EE46CEF800C051
:10DDA000F3F7D6FF002818BF012006B080BD81B070
:10DDB00000904DF6E350C0F6000001B0704780B50A
:10DDC0006F4684B002900191029A106800F1080138
:10DDD0001160009003A86946FDF7CEFD039804B0DA
:10DDE00080BD80B56F4682B0019000910199009A84
:10DDF00000F002F802B080BD80B56F4684B0039099
:10DE0000029101920198009000994A680878896807
:10DE1000904704B080BD81B000904DF65560C0F6CB
:10DE2000000001B0704783B0029001910092029807
:10DE3000019901600099416003B0704780B56F4659
:10DE400082B001900198009000980168406888476E
:10DE500002B080BD80B56F4682B00190019900F09C
:10DE600002F802B080BD80B56F468CB00B900A916D
:10DE700047F63E61C0F6020109A84FF0FF32049256
:10DE800000F065F8049A47F64661C0F6020108A85A
:10DE900000F07BF8049A47F65261C0F6020107A829
:10DEA00000F091F8049A47F65E61C0F6020106A8F8
:10DEB00000F0A7F8F6F72BFF0590FFE70A9800F2AD
:10DEC0001C40009000F0DFF80099024608A800F01E
:10DED000B6F80A9800F50770019000F0D4F801999F
:10DEE000024609A800F0D9F80A9800F506700290D9
:10DEF00000F0C9F80299024607A800F0F2F80A9863
:10DF000000F5A270039000F0BEF80399024606A83F
:10DF100000F00BF90A98FFF7C2FC0A9800F50570AB
:10DF20004FF0FF31FFF729FE0A98FFF701F90A9831
:10DF3000FFF752F90A9800F50570FFF75EFE0A98A0
:10DF400000F50470022105AAF3F725FEB6E780B5B7
:10DF50006F4686B004900391029204980090059059
:10DF600003980299F4F706FD0190019830B1FFE79C
:10DF70000198F4F7C1FA0099086003E000990020C5
:10DF80000860FFE7059806B080BD80B56F4686B093
:10DF900004900391029204980090059003980299CE
:10DFA000F4F7E8FC0190019830B1FFE70198F4F72D
:10DFB000A3FA0099086003E0009900200860FFE7D9
:10DFC000059806B080BD80B56F4686B00490039179
:10DFD000029204980090059003980299F4F7CAFC05
:10DFE0000190019830B1FFE70198F4F785FA0099A4
:10DFF000086003E0009900200860FFE7059806B07C
:10E0000080BD80B56F4686B004900391029204985B
:10E010000090059003980299F4F7ACFC01900198E8
:10E0200030B1FFE70198F4F767FA0099086003E060
:10E03000009900200860FFE7059806B080BD80B514
:10E040006F4686B00490039107F80D2C0498019058
:10E0500000F08FF878B1FFE701980068039917F88E
:10E060000D2C02F00102F4F756FAB0FA80F04009E4
:10E0700007F8010C03E0002007F8010CFFE717F890
:10E08000010C06B080BD81B0EFF3058000900098D0
:10E09000002818BF012001B0704780B56F4686B0D8
:10E0A0000490039107F80D2C0498019000F06AF891
:10E0B00078B1FFE701980068039917F80D2C02F07A
:10E0C0000102F4F728FAB0FA80F0400907F8010CD1
:10E0D00003E0002007F8010CFFE717F8010C06B079
:10E0E00080BD80B56F4686B00490039107F80D2C73
:10E0F0000498019000F04FF878B1FFE701980068AC
:10E10000039917F80D2C02F00102F4F704FAB0FAA3
:10E1100080F0400907F8010C03E0002007F8010C2B
:10E12000FFE717F8010C06B080BD80B56F4686B0DA
:10E130000490039107F80D2C0498019000F034F836
:10E1400078B1FFE701980068039917F80D2C02F0E9
:10E150000102F4F7E0F9B0FA80F0400907F8010C89
:10E1600003E0002007F8010CFFE717F8010C06B0E8
:10E1700080BD81B0009000980068002818BF012081
:10E1800001B0704781B0009000980068002818BF67
:10E19000012001B0704781B000900098006800280D
:10E1A00018BF012001B0704781B00090009800684E
:10E1B000002818BF012001B0704780B56F4684B0B9
:10E1C000039002910398009004300190F3F7F1FC62
:10E1D000009902981030F4F738FA0198F3F7F8FC38
:10E1E000012004B080BD80B56F468AB009900891C7
:10E1F0008DED070A099803900021019141600160AB
:10E20000C1608160016114300899FDF7C0F903987D
:10E21000019980F80C1100F5887000F06FF80398F0
:10E2200000F58E70089914310BF04EFE039901F53C
:10E2300098703C319DED070A0BF0AEFD039901F596
:10E240000E7084319DED070A0BF0A6FD039901F5D0
:10E250005070CC3147F66762C0F6020209F07EFECC
:10E26000039901F56E70D83147F67262C0F602026A
:10E2700009F074FE039800F586600290F3F767F8E2
:10E28000039800F234400121FEF768FB0398019ADD
:10E2900000F5876047F65261C0F6020100F039F8D8
:10E2A000039800F28C4000F05EF806A800F0BCF87D
:10E2B000039901F5807200F069F8029803996B46A2
:10E2C00002221A6047F67F62C0F602024FF4007322
:10E2D00000F0B2F803994EF21550C0F600004FF46A
:10E2E000FA6200F0E2F803994EF65110C0F6000011
:10E2F0003C2200F0DAF803980AB080BD80B56F4682
:10E3000082B001900198009000F02DF8009802B0C2
:10E3100080BD80B56F4686B00490039107F80D2C40
:10E3200004980190059017F80D0CC00760B9FFE73D
:10E33000039A47F6AE61C0F6020100200423F3F70A
:10E340005BFD019908600BE0039A47F6AD61C0F6EA
:10E35000020100200423F3F74FFD01990860FFE755
:10E36000059806B080BD80B56F4682B001900198D7
:10E37000009000F0B9FE0098043000F0B5FE00985F
:10E38000083000F0B1FE009802B080BD80B56F4645
:10E390008EB00D900C910B9209A8FFF7CAFC0B9858
:10E3A000FDF79FF9089008980990FFE70B98FDF793
:10E3B000A3F9079009A807A9FFF7C2FC90B3FFE7EC
:10E3C0000C20FEF7FEFB06900C98069988600D98CD
:10E3D0000699486009A80290FFF7C7FC0146029819
:10E3E0004968069A116042F2CC61C2F200010968E4
:10E3F00004310491FFF7B9FC006803900AA800F00B
:10E40000DDFE039903460498069AEC46CCF80020FA
:10E410000122FFF7B0FCFFE709A80021FFF7CFFCBE
:10E420000590C3E70EB080BD81B000904FF2F700B9
:10E43000C0F6000001B0704780B56F468EB08446CC
:10E44000B868CDF830C00B910A92099307F8150C03
:10E450000C9804900DA8039000F0D2FE082013F051
:10E460000DFB01460398079100F0CAFE01460B9A86
:10E4700005A800F0CDFEDDF810E007990598069A92
:10E480004A600860079B0A99BDF8242017F8150C0C
:10E49000EC46CCF804E0CCF800004FF22720C0F6A0
:10E4A000000014F0C3F90EB080BD80B56F4688B08F
:10E4B000079006910592082013F0E0FA049007995E
:10E4C000069A02A800F0A4FE04990298039A4A60F2
:10E4D00008601420F2F720FF019001990020488184
:10E4E00005980199088101994FF22720C0F6000094
:10E4F000486004980199086001990120087340F26E
:10E50000D070C2F2000000680199FFF756FE019832
:10E5100008B080BDF0B503AF2DE9000FD9B0589019
:10E52000589800F588602190FFF7DAF99FED531AAB
:10E5300020EE010ABDEEC00A10EE100A2090FFF78F
:10E54000D5F9209B21989FED4E1A20EE010ABDEED1
:10E55000C00A10EE101A47F6906CC0F6020C6A461C
:10E56000C2F818C013610223D3604FF0500CC2F8F8
:10E5700008C04FF00A0CC2F804C01360516147F69E
:10E580008D61C0F602010122002324930DF0CDFD20
:10E59000589800F588614CA82290FFF7ADF92299B0
:10E5A00040A82D2218F0F6F840984199429A439BD2
:10E5B000DDF810C1459C469D479EDDF82081DDF8C1
:10E5C0002491DDF828A1DDF82CB1EE46CDF88CE0E1
:10E5D000CEF81CB0CEF818A0CEF81490CEF810806B
:10E5E000CEF80C60CEF80850CEF80440CEF800C04B
:10E5F0000BF097F924983F903E90589890F80C01B2
:10E600000146259120B1FFE72598012809D020E097
:10E610000020C4F258203F900020C4F2CC203E904D
:10E620001BE0589890F8B00448B9FFE70020C4F206
:10E63000E4203F900020C4F222303E9008E0002009
:10E64000C4F22E303F900020C4F25E303E90FFE7CF
:10E6500003E000203F903E90FFE79DED3F0AB5EEBE
:10E66000400AF1EE10FA7DD0FFE79DED3E0AB5EECF
:10E67000400AF1EE10FA75D004E000BF9A99593FB4
:10E680007B142E3F589800F26D401D90FFF728F93B
:10E690009DED3F1A9FEDA82A8DED192A20EE020A62
:10E6A00030EE010ABDEEC00A10EE100A1C90FFF712
:10E6B0001DF99FEDA21A8DED1A1A20EE010AB1EE96
:10E6C000001A30EE010ABDEEC00A10EE100A1B90CF
:10E6D000FFF706F99DED192A9DED3E1A20EE020A7C
:10E6E00030EE010ABDEEC00A10EE100A1E90FFF7D0
:10E6F000FDF89DED1A1ADDF86CC01C9A1D98DDF826
:10E7000078E020EE010ABAEE0C1A30EE010ABDEEF6
:10E71000C00A10EE101A6B46C3F810E0C3F80CC024
:10E720009A6001225A604FF0020CC3F800C0596190
:10E7300047F6A761C0F6020104230DF033F858989C
:10E7400000F26D413AA81F90FFF7E0F81F9936A834
:10E750000F2218F01FF836983799389A399B0BF02A
:10E7600066F8FFE7589800F27C400B90FFF7B8F886
:10E770009FED731A8DED0E1A20EE010ABDEEC00A50
:10E7800010EE100A0A90FFF7B1F89FED6E1A8DEDAA
:10E79000111A20EE010ABDEEC00A10EE100A09900F
:10E7A000FFF79EF89DED0E1A20EE010ABDEEC00A9D
:10E7B00010EE100A0C90FFF799F8DDF824C00A9BC0
:10E7C0000B989DED111ADDF830E020EE010A9FED67
:10E7D0005E1A30EE010ABDEEC00A10EE101A6A464B
:10E7E000C2F810E0C2F80CC0936003235360022308
:10E7F00012931360516147F6D961C0F602010122FC
:10E80000149200230CF0AEFD589800F27C4132A81F
:10E810000D9000F05FFC0D992EA80F22189217F0B2
:10E82000B9FF2E982F99309A319B0BF000F8589829
:10E8300000F27C401390FFF753F89DED0E1A20EE86
:10E84000010ABDEEC00A10EE100A1590FFF74EF84F
:10E850009DED111A20EE010ABDEEC00A10EE104A1D
:10E86000FFF73EF88DED0F0A589800F23C4090ED0E
:10E87000000A16F005FA9DED0E2AB0EE401A9DED45
:10E880000F0A9FED323A8DED103A21EE031A20EE79
:10E89000020A30EE410ABDEEC00A10EE105AFFF730
:10E8A00025F88DED160A589800F23C4090ED000ACC
:10E8B00016F0A0F99DED103A9DED112ADDF848C043
:10E8C0001398149ADDF854E0B0EE401A9DED160A44
:10E8D00021EE031A20EE020A30EE010ABDEEC00A54
:10E8E00010EE101A6B461D61DC60C3F808E04FF0B3
:10E8F0000C0EC3F804E0C3F800C0596147F6AA61E2
:10E90000C0F6020104230CF02DFD589800F27C4162
:10E910002AA8179000F0DEFB1799189A26A817F07E
:10E9200039FF26982799289A299B0AF080FF59B029
:10E93000BDE8000FF0BD00BF9A99593F7B142E3FF0
:10E94000CDCCCC3ECDCC4C3E000048420000304205
:10E9500080B56F46ACB02B9000202A9029902B9860
:10E9600090F80C010146189120B1FFE71898012892
:10E9700009D020E00020C4F258202A900020C4F2E0
:10E98000CC2029901BE02B9890F8B00448B9FFE701
:10E990000020C4F2E4202A900020C4F22230299002
:10E9A00008E00020C4F22E302A900020C4F25E302D
:10E9B0002990FFE703E000202A902990FFE79DEDD2
:10E9C0002A0AB5EE400AF1EE10FA76D0FFE79DED87
:10E9D000290AB5EE400AF1EE10FA6ED0FFE72B9847
:10E9E00000F26D401590FEF77BFF9DED2A1A9FED1A
:10E9F000762A8DED112A20EE020A30EE010ABDEED4
:10EA0000C00A10EE100A1490FEF770FF9FED6F1A07
:10EA10008DED121A20EE010AB1EE001A30EE010A55
:10EA2000BDEEC00A10EE100A1390FEF759FF9DEDDF
:10EA3000112A9DED291A20EE020A30EE010ABDEEE0
:10EA4000C00A10EE100A1690FEF750FF9DED121A44
:10EA5000DDF84CC0149A1598DDF858E020EE010A54
:10EA6000BAEE0C1A30EE010ABDEEC00A10EE101A12
:10EA70006B46C3F810E0C3F80CC09A6001225A60DC
:10EA800002221A60596147F6A761C0F60201042309
:10EA90000CF088FE2B9800F26D4125A81790FEF728
:10EAA00035FF179921A80F2217F074FE219822999B
:10EAB000239A249B0AF0BBFEFFE72B9800F27C40D0
:10EAC0000D90FEF70DFF9FED421A8DED071A20EE17
:10EAD000010ABDEEC00A10EE100A0C90FEF706FF08
:10EAE0009FED3C1A8DED0A1A20EE010ABDEEC00A18
:10EAF00010EE100A0B90FEF7F3FE8DED080A2B982E
:10EB000000F23C4090ED000A16F0BAF89DED072A9D
:10EB1000B0EE401A9DED080A9FED2F3A8DED093AAF
:10EB200021EE031A20EE020A30EE410ABDEEC00AC1
:10EB300010EE100A0E90FEF7D9FE8DED0F0A2B98FD
:10EB400000F23C4090ED000A16F054F89DED093AB1
:10EB50009DED0A2ADDF82CC00C9A0D98DDF838E0FE
:10EB6000B0EE401A9DED0F0A21EE031A20EE020AC4
:10EB700030EE010ABDEEC00A10EE101A6B46C3F863
:10EB800010E0C3F80CC09A600C225A6002221A608E
:10EB9000596147F6AA61C0F6020104230CF0E2FBBA
:10EBA0002B9800F27C411DA8109000F093FA109968
:10EBB00019A80F2217F0EEFD19981A991B9A1C9BA1
:10EBC0000AF035FE2CB080BD9A99593F7B142E3F38
:10EBD000CDCCCC3ECDCC4C3E0000304280B56F4613
:10EBE00086B005900598039000F56E7009F055FB0E
:10EBF000039800F55070019009F04FFB019904A8AB
:10EC0000029000F00CF802980399E43100F024F827
:10EC1000039800F23C4080ED000A06B080BD80B54C
:10EC20006F4684B00090039002910298019090F892
:10EC30003400C00730B1FFE700980199203100F09F
:10EC4000A7FA05E0009801992031FCF7D7FEFFE70D
:10EC500004B080BD0000000080B56F4684B0039012
:10EC60000291039890ED000A029890ED001A30EEA0
:10EC7000410A8DED010AFFE70198F1F7F3FC41EC41
:10EC8000100B9FED191B53EC112B51EC100BF1F7EE
:10EC9000C7FF48B1FFE79DED010A9FED181A30EE5E
:10ECA000010A8DED010AE7E7FFE70198F1F7DAFCC9
:10ECB00041EC100B9FED0E1B53EC112B51EC100B84
:10ECC000F1F79AFF48B1FFE79DED010A9FED0A1A9F
:10ECD00030EE010A8DED010AE7E79DED010A04B06F
:10ECE00080BD00BF00BF00BF182D4454FB21094068
:10ECF000182D4454FB2109C0DB0FC940DB0FC9C0EC
:10ED000080B56F46AEB02D902D981690F6F701F8AD
:10ED10000A461699CA6088600B684A688868C9689C
:10ED2000C01A9141F2F7E6F80146169800EE101A63
:10ED30009FEDB81A80EE010A80ED040A8168C2686E
:10ED40004260016000212C912B9190F8B0040128C1
:10ED50001AD1FFE7169800F2A44191ED000A90ED58
:10ED6000041A20EE010A9FEDAC1A20EE010A8DED87
:10ED70002B0A91ED010A90ED042A20EE020A20EE02
:10ED8000010A8DED2C0A1EE0169800F2A4412AA873
:10ED90001490FCF7FBF91498169901F58871FFF7A8
:10EDA0005BFF16988DED2B0A00F5956129A815904B
:10EDB000FCF7ECF91598169901F58A71FFF74CFFED
:10EDC0008DED2C0AFFE71698F83000F027F9169819
:10EDD0008DED130AFC3000F021F9B0EE401A9DEDE4
:10EDE000130AB4EE410AF1EE10FA40D0FFE716988C
:10EDF00000F1F8010E9100F55071109127A80F90C5
:10EE0000FFF70DFF0E980F99FFF726FF1099169840
:10EE10008DED280AFC30119025A81290FFF7FFFE17
:10EE200011981299FFF718FF16998DED260A01F532
:10EE3000887001F28C41FFF70FFF8DED240A9DEDE4
:10EE4000280A9DED241A30EE410A8DED230A9DED2E
:10EE5000260A9DED241A30EE410A8DED220A9DED21
:10EE6000220ADDED230A2BA80DF0F3FBFFE716982D
:10EE700000F5887121A82BAA00F0D7F81698F03079
:10EE800000F0CCF816988DED0D0AF43000F0C6F8BD
:10EE9000B0EE401A9DED0D0AB4EE410AF1EE10FA03
:10EEA00040D0FFE7169800F1F001089100F56E716F
:10EEB0000A911FA80990FFF7B2FE08980999FFF779
:10EEC000CBFE0A9916988DED200AF4300B901DA800
:10EED0000C90FFF7A4FE0B980C99FFF7BDFE169956
:10EEE0008DED1E0A01F58A7001F59261FFF7B4FEFF
:10EEF0008DED1C0A9DED200A9DED1C1A30EE410A95
:10EF00008DED1B0A9DED1E0A9DED1C1A30EE410A87
:10EF10008DED1A0A9DED1A0ADDED1B0A2CA80DF0E5
:10EF200098FBFFE7169800F58A7119A82CAA00F043
:10EF30007CF8169800211891179190F80C01014661
:10EF4000079120B1FFE7079801280BD05FE01698E2
:10EF500000F5507009F028FB169800F56E7009F066
:10EF600023FB54E0169800F59871009100F5887025
:10EF700000F054F816988DED020A00F593610391A4
:10EF800091ED020A8DED010A00F28C4000F046F886
:10EF90000098DDED010A1699B0EE401A9DED020AC7
:10EFA000D1ED041A0AF02CFF16988DED180A00F521
:10EFB0000E71049100F58A7000F030F803991698EC
:10EFC0008DED060A91ED000A8DED050A00F59260BF
:10EFD00000F024F80498DDED050A1699B0EE401A09
:10EFE0009DED060AD1ED041A0AF00AFF16988DED80
:10EFF000170A00F550709DED180A09F0F1F91698FE
:10F0000000F56E709DED170A09F0EAF9FFE72EB0E2
:10F0100080BD00BF00247449E4CB164181B000904C
:10F02000009890ED000A01B0704780B56F4686B039
:10F03000019005900491039204980290039991ED38
:10F04000000A90ED001A30EE010AFCF7BBF90198B6
:10F05000029981ED000AFCF7D1FC06B080BD80B5B5
:10F060006F4684B0039007F8051C0399019117F8C7
:10F07000050C91F80C11884201D1FFE728E00198B6
:10F0800000F50E700AF0FCFE019800F598700AF089
:10F09000F7FE019901F5887001F28C410C2217F0FE
:10F0A0007EFB019890F80C0160B9FFE717F8050C9A
:10F0B000012806D1FFE70199D1F88C04C1F81001AD
:10F0C000FFE7FFE7019917F8050C81F80C01FFE74E
:10F0D00004B080BD80B56F4682B0019101990F22C6
:10F0E00017F058FB02B080BD81B00090009800215D
:10F0F000016001B0704780B56F4682B007F8010C1F
:10F10000009117F8011C009A00F002F802B080BDCF
:10F1100080B56F4684B0039007F8051C01920198F2
:10F1200000F234404FF0FF31FEF727FD17F8050CD1
:10F1300001460091022808D3FFE7009802280AD070
:10F14000FFE7009803280AD00DE0019817F8051C86
:10F15000FFF785FF07E0012000F00CF803E0002036
:10F1600000F008F8FFE7019800F23440FEF745FD93
:10F1700004B080BD81B08DF803009DF8030042F219
:10F18000CC61C2F200010968487001B0704700000C
:10F1900080B56F4684B003900291029991ED001AF8
:10F1A0009FED050A30EE410A8DED010A01A9FBF73A
:10F1B000EDFF04B080BD00BFDB0FC94081B00090FF
:10F1C0004FF2CD10C0F6000001B0704780B56F4619
:10F1D00082B0019000910199009A00F002F802B00B
:10F1E00080BD80B56F4684B0039002910192019872
:10F1F000009000994A6808788968904704B080BDFB
:10F2000081B000904FF23F20C0F6000001B070477F
:10F2100083B00290019100920298019901600099D7
:10F22000416003B0704780B56F4682B0019001988D
:10F230000090009801684068884702B080BD80B5A2
:10F240006F4682B00190019900F002F802B080BDD3
:10F2500080B56F468CB00B900A9147F6B061C0F64E
:10F26000020109A84FF0FF32059200F05DF8059AFF
:10F2700047F6B961C0F6020108A8FEF786FE059AB6
:10F2800047F6C261C0F6020107A800F06BF8F5F777
:10F290003EFD0690FFE70A9800F28C40009000F0D7
:10F2A000A3F80099024609A800F07AF80A9800F538
:10F2B0009360019000F098F80199024608A8FEF7C3
:10F2C000BEFE0A9800F2A440029000F08DF8029968
:10F2D000024607A800F092F80A9800F234404FF076
:10F2E000FF31FEF74AFC0A98FFF778FC0A98FFF70F
:10F2F00007FD0A9800F23440FEF77FFC0A9800F5FB
:10F300008761049100F23C40039000F06DF803998E
:10F310000246049800F096F80A9800F586600221EB
:10F3200006AAF2F738FCB6E780B56F4686B00490BF
:10F330000391029204980090059003980299F3F7C4
:10F3400019FB0190019830B1FFE70198F3F7D4F869
:10F350000099086003E0009900200860FFE7059825
:10F3600006B080BD80B56F4686B0049003910292CE
:10F3700004980090059003980299F3F7FBFA019026
:10F38000019830B1FFE70198F3F7B6F800990860EB
:10F3900003E0009900200860FFE7059806B080BDF3
:10F3A00080B56F4686B00490039107F80D2C049841
:10F3B000019000F060F878B1FFE7019800680399C8
:10F3C00017F80D2C02F00102F3F7A5F8B0FA80F05F
:10F3D000400907F8010C03E0002007F8010CFFE7E3
:10F3E00017F8010C06B080BD81B0EFF305800090E6
:10F3F0000098002818BF012001B0704780B56F4603
:10F4000086B00490039107F80D2C0498019000F049
:10F410003BF878B1FFE701980068039917F80D2CC5
:10F4200002F00102F3F777F8B0FA80F0400907F82C
:10F43000010C03E0002007F8010CFFE717F8010CAE
:10F4400006B080BD80B56F4684B00390029107F886
:10F45000092C03980068029917F8092C02F00102A0
:10F460006B461A6004220123F3F707F8B0FA80F024
:10F47000400904B080BD81B0009000980068002869
:10F4800018BF012001B0704781B00090009800685B
:10F49000002818BF012001B0704780B56F46B0B09A
:10F4A0002E902D918DED2C0A2E980C902F900021EE
:10F4B0000E91C1608160416101618161C161203053
:10F4C0002D99FCF784F80C9801210D9180F83C11DE
:10F4D00000F5A07000F0EFF80C9800F5B67000F0A1
:10F4E000F1F80C9800F5EE70F1F731FF0C980D99DA
:10F4F00000F5F070FDF732FA0E982B90FFE72B988D
:10F5000000284FD1FFE74FF48470F1F705FF079013
:10F510002D9820302B9900F0E6F8014607989DEDD4
:10F520002C0A0AF039FC0C9800F5CA702B9900F0EF
:10F53000F4F80146079808607820F1F7EDFE0146DF
:10F540000C98099100F580702B9900F0FEF8089056
:10F550002B991FA80B9000F026F90B9A47F6CD6166
:10F56000C0F6020125A80A9000F009F90A9815F0E2
:10F57000ABFA08990246099808F0F0FC0C9800F5DF
:10F58000D2702B9900F035F9099902460A9811605A
:10F5900015F03DF90B9815F03AF9FFE72B9801307B
:10F5A0002B90ACE700201E90FFE71E9802284ED853
:10F5B000FFE79420F1F7B0FE02902D9868301E9975
:10F5C00000F02FF9014602989DED2C0A0AF07EFB0F
:10F5D0000C9800F5CC701E9900F03EF90146029897
:10F5E00008607820F1F798FE01460C98049100F528
:10F5F00086701E9900F049F903901E9912A8069092
:10F6000000F0D1F8069A47F6DB61C0F6020118A8AF
:10F61000059000F0B4F8059815F056FA03990246E3
:10F62000049808F09BFC0C9800F5D4701E9900F02B
:10F6300047F9049902460598116015F0E8F8069814
:10F6400015F0E5F8FFE71E9801301E90ADE711A810
:10F6500000F09DF90C9901F5987200F04AF901202B
:10F6600001900DF04DFB0C99019891ED0C0A0DF0F5
:10F6700057FB0C9901F5EE706B4602221A6047F6B3
:10F68000E962C0F602024FF4C07300F088F90C99E9
:10F690004FF67D20C0F6000040F6980200F0B8F961
:10F6A0000C9940F28910C0F60100642200F0B0F914
:10F6B0002F9830B080BD81B0009000980021C160CB
:10F6C00001B0704781B00090009800210170417036
:10F6D000416001724FF07E52C26080F8241080F8C1
:10F6E000251001B0704780B56F4684B00390029139
:10F6F00003980190029840B1FFE7029947F6F7405E
:10F70000C0F60200012214F0C7FF0198029901EB34
:10F71000C10100EBC10004B080BD80B56F4684B06C
:10F720000390029103980190029840B1FFE702997B
:10F7300047F6F740C0F60200012214F0ADFF019831
:10F74000029900EB810004B080BD80B56F4684B0A3
:10F750000390029103980190029840B1FFE702994B
:10F7600047F6F740C0F60200012214F095FF019819
:10F77000029901EB410100EB810004B080BD80B52E
:10F780006F4684B000900390029101920198029A12
:10F79000002115F04FF9FEF7C7FA0146009815F061
:10F7A00017F804B080BD80B56F4686B00090059014
:10F7B000049104980A21FEF7B3F8014600980391DA
:10F7C000002107F80D1C14F0FCFF00980399049A1F
:10F7D0000192019A01F0C7FC012007F80D0C17F8FF
:10F7E0000D0C20B9FFE7009815F011F8FFE706B0FF
:10F7F00080BD80B56F4684B003900291039801905C
:10F80000029840B1FFE7029947F6F740C0F60200C0
:10F81000012214F041FF0198029900EB810004B02D
:10F8200080BD80B56F4684B003900291039801902B
:10F830000298032808D3FFE7029947F6F740C0F67D
:10F840000200032214F028FF0198029901EB8101C4
:10F8500000EBC10004B080BD80B56F4684B003905A
:10F860000291039801900298032808D3FFE70299B8
:10F8700047F6F740C0F60200032214F00DFF01988E
:10F88000029900EB810004B080BD80B56F4684B062
:10F8900003900291039801900298032808D3FFE790
:10F8A000029947F6F740C0F60200032214F0F4FE76
:10F8B0000198029901EB410100EB810004B080BD89
:10F8C00080B56F4684B0039002910398019002982E
:10F8D000032808D3FFE7029947F6F740C0F6020075
:10F8E000032214F0D9FE0198029900EB810004B0C4
:10F8F00080BD80B56F468EB00D900C910B9209A81B
:10F90000FEF717FA0B98FBF7ECFE089008980990A1
:10F91000FFE70B98FBF7F0FE079009A807A9FEF791
:10F920000FFA90B3FFE70C20FDF74BF906900C9807
:10F93000069988600D980699486009A80290FEF71C
:10F9400014FA014602984968069A116042F2CC61A5
:10F95000C2F20001096804310491FEF706FA00685A
:10F9600003900AA801F0B7FC039903460498069A8D
:10F97000EC46CCF800200122FEF7FDF9FFE709A8CC
:10F980000021FEF71CFA0590C3E70EB080BD81B0E0
:10F99000009041F2F910C0F6010001B0704780B547
:10F9A0006F468EB08446B868CDF830C00B910A928D
:10F9B000099307F8150C0C9804900DA8039001F01A
:10F9C000ACFC082012F05AF801460398079101F0A8
:10F9D000A4FC01460B9A05A801F0A7FCDDF810E095
:10F9E00007990598069A4A600860079B0A99BDF82E
:10F9F000242017F8150CEC46CCF804E0CCF80000F5
:10FA000041F24130C0F6010012F010FF0EB080BD8F
:10FA100080B56F4688B0079006910592082012F0D5
:10FA20002DF804900799069A02A801F07EFC04992B
:10FA30000298039A4A6008601420F1F76DFC019067
:10FA4000019900204881059801990881019941F2A6
:10FA50004130C0F60100486004980199086001999E
:10FA60000120087340F2D070C2F2000000680199D2
:10FA7000FEF7A3FB019808B080BD0000F0B503AF0E
:10FA80002DE9000FADF5157D9490949800F2E330C8
:10FA90002E90FDF725FF9FEDE11A8DED331A20EE34
:10FAA000010ABDEEC00A10EE100A2D90FDF71EFFF0
:10FAB0002D9B2E989FEDDA1A20EE010ABDEEC00AAA
:10FAC00010EE101A47F6FC6CC0F6020C6A46C2F83B
:10FAD00018C0136102233693D360502595600A2421
:10FAE00054601360516147F6F961C0F602010122CA
:10FAF000359200233A930CF018FB949800F2E3310E
:10FB000088A82F90FDF7F8FE2F997CA82D22389217
:10FB100016F040FE7C9831907D9830907E9A7F9BC5
:10FB2000DDF800C2819EDDF80882DDF80C92DDF878
:10FB300010A2DDF814B2DDF818E287986946329118
:10FB4000C86130993298C0F818E03198DDF8C8E003
:10FB5000CEF814B0CEF810A0CEF80C90CEF80880F5
:10FB6000CEF80460CEF800C009F0DBFE949800F2F5
:10FB7000E3303490FDF7B4FE9DED331A20EE010A18
:10FB8000BDEEC00A10EE106AFDF7B0FE3498359A4B
:10FB90003A9BDDF8D8E09FEDA31A20EE010ABDEEF6
:10FBA000C00A10EE101A47F61678C0F60208EC46A6
:10FBB000CCF81880CCF81060CCF80CE0CCF80850E9
:10FBC000CCF80440CCF800E0CCF8141047F61371E0
:10FBD000C0F602010CF0A9FA949800F2E33170A883
:10FBE0003790FDF789FE3799389A64A816F0D2FD50
:10FBF00064986599669A679BDDF8A0C1699C6A9DC7
:10FC00006B9EDDF8B081DDF8B491DDF8B8A1DDF8C8
:10FC1000BCB1EE46CDF8E4E0CEF81CB0CEF818A0AA
:10FC2000CEF81490CEF81080CEF80C60CEF80850C4
:10FC3000CEF80440CEF800C009F073FE3A98639005
:10FC40006290949890F8910101463B9140B1FFE792
:10FC50003B9801280DD0FFE73B98022812D01AE00C
:10FC60000020C4F2582063900020C4F2CC2062909F
:10FC700015E00020C4F2E42063900020C4F222309A
:10FC800062900CE00020C4F22E3063900020C4F299
:10FC90005E30629003E0002063906290FFE79DED8C
:10FCA000630AB5EE400AF1EE10FA78D0FFE79DED59
:10FCB000620AB5EE400AF1EE10FA70D0FFE79498B0
:10FCC00000F582602A90FDF70BFE9DED631A9FED13
:10FCD000532A8DED262A20EE020A30EE010ABDEEEF
:10FCE000C00A10EE100A2990FDF700FE9FED4C1A95
:10FCF0008DED271A20EE010AB1EE001A30EE010A4E
:10FD0000BDEEC00A10EE100A2890FDF7E9FD9DED4A
:10FD1000262A9DED621A20EE020A30EE010ABDEE9F
:10FD2000C00A10EE100A2B90FDF7E0FD9DED271A9A
:10FD3000DDF8A0C0299A2A98DDF8ACE020EE010A8F
:10FD4000BAEE0C1A30EE010ABDEEC00A10EE101A1F
:10FD50006B46C3F810E0C3F80CC09A6001225A60E9
:10FD60004FF0020CC3F800C0596147F62D71C0F680
:10FD7000020105230BF016FD949800F582615EA840
:10FD80002C90FDF7C3FD2C995AA80F2216F002FD06
:10FD90005A985B995C9A5D9B09F049FDFFE794983E
:10FDA00090F890010146259140B1FFE72598012880
:10FDB0000DD0FFE72598022812D01AE00020C4F2E7
:10FDC000582063900020C4F2CC20629015E00020FF
:10FDD000C4F2E42063900020C4F2223062900CE070
:10FDE0000020C4F22E3063900020C4F25E30629096
:10FDF00003E0002063906290FFE79DED630AB5EE9B
:10FE0000400AF1EE10FA00F07F80FFE79DED620AF4
:10FE1000B5EE400AF1EE10FA76D005E09A99593F16
:10FE2000C3F5283F0AD7233F949800F582602290BB
:10FE3000FDF756FD9DED631A9FEDCC2A8DED1E2A30
:10FE400020EE020A30EE010ABDEEC00A10EE100AE2
:10FE50002190FDF74BFD9FEDC61A8DED1F1A20EE88
:10FE6000010AB1EE001A30EE010ABDEEC00A10EE32
:10FE7000100A2090FDF734FD9DED1E2A9DED621ABB
:10FE800020EE020A30EE010ABDEEC00A10EE100AA2
:10FE90002390FDF72BFD9DED1F1ADDF880C0219A00
:10FEA0002298DDF88CE020EE010ABAEE0C1A30EE52
:10FEB000010ABDEEC00A10EE101A6B46C3F810E03E
:10FEC000C3F80CC09A6001225A604FF0020CC3F8CC
:10FED00000C0596147F63071C0F6020105230BF0EE
:10FEE00061FC949800F5826156A82490FDF70EFD00
:10FEF000249952A80F2216F04DFC52985399549A07
:10FF0000559B09F094FCFFE7949800F21F4114916F
:10FF100000F5D47000210F9100F0B6FC0068FDF7E9
:10FF20003FF90F998DED0E0A949800F5A07001F03D
:10FF300081F89DED0E0A0F9990ED001A80EE010AEE
:10FF40009FED8C1A8DED111A20EE010ABDEEC00A4C
:10FF500010EE100A1390949800F5D47000F094FC01
:10FF60000068FDF71DF90F998DED100A949800F5C2
:10FF7000A07001F05FF89DED100A9DED111A90ED53
:10FF8000002A80EE020A20EE010ABDEEC00A10EE41
:10FF9000100AC0F5B4701590FDF7A2FC9FED761A1B
:10FFA00020EE010ABDEEC00A10EE100A1290FDF715
:10FFB0009DFC129BDDF84CC01498DDF854E09FEDD9
:10FFC0006F1A20EE010ABDEEC00A10EE101A6A4642
:10FFD00016923224D461946113610523D3601FFA11
:10FFE0008EFEC2F808E0C2F804C04FF0020CC2F85E
:10FFF00000C0516147F63371C0F6020101220BF0D7
:020000040801F1
:10000000F8FD949800F21F414EA8179001F0A1F856
:1000100017994AA80F2216F0BDFB4A984B994C9AA3
:100020004D9B09F004FC949800F11C0147A818901E
:10003000FBF7ACF8189948A81990FFF7A9F8199898
:10004000FEF7ECFF9FED4E1A8DED1C1A80EE010AB3
:100050009FED4C1A8DED1D1A20EE010ABDEEC00A6F
:1000600010EE100AADF82601949800F11C0144A886
:100070001A90FBF78BF81A9945A81B90FFF788F8A0
:100080001B98FEF7CBFF9DED1C2A9DED1D1A80EEFF
:10009000020A20EE010AB3EE0E1A30EE010ABDEE9E
:1000A000C00A10EE100AADF81A01BDF81A01B0F539
:1000B000B47F07DDFFE7BDF81A01A0F5B470ADF815
:1000C0001A01FFE7949800F21F400B90BDF826013B
:1000D0000A90BDF81A010C90FDF702FC9FED261A5C
:1000E00020EE010ABDEEC00A10EE100A0990FDF7DD
:1000F000FDFB099BDDF828C00B98DDF830E09FED93
:100100001F1A20EE010ABDEEC00A10EE101A6A4650
:100110002824D461946113610523D360C2F808E0F8
:10012000C2F804C04FF0020CC2F800C0516147F69B
:100130003671C0F6020101220BF05BFD949800F2CB
:100140001F4140A80D9001F004F80D993CA80F2222
:1001500016F020FB3C983D993E9A3F9B09F067FBC7
:100160000DF5157DBDE8000FF0BD00BF9A99593F10
:100170000AD7233F000034439A99193FCDCCCC3D98
:10018000DB0FC9400000B443B0B502AFD8B0579000
:10019000002056905590579890F8910101462D9166
:1001A00040B1FFE72D9801280DD0FFE72D980228D8
:1001B00012D01AE00020C4F2582056900020C4F259
:1001C000CC20559015E00020C4F2E4205690002089
:1001D000C4F2223055900CE00020C4F22E3056902C
:1001E0000020C4F25E30559003E0002056905590F8
:1001F000FFE79DED560AB5EE400AF1EE10FA76D013
:10020000FFE79DED550AB5EE400AF1EE10FA6ED00B
:10021000FFE7579800F582602A90FDF761FB9DED9E
:10022000561A9FEDD52A8DED262A20EE020A30EED1
:10023000010ABDEEC00A10EE100A2990FDF756FB28
:100240009FEDCE1A8DED271A20EE010AB1EE001AAD
:1002500030EE010ABDEEC00A10EE100A2890FDF73C
:100260003FFB9DED262A9DED551A20EE020A30EE49
:10027000010ABDEEC00A10EE100A2B90FDF736FB06
:100280009DED271ADDF8A0C0299A2A98DDF8ACE088
:1002900020EE010ABAEE0C1A30EE010ABDEEC00AD9
:1002A00010EE101A6B46C3F810E0C3F80CC09A6049
:1002B00001225A6002221A60596147F62D71C0F678
:1002C000020105230BF06EFA579800F5826151A8E0
:1002D0002C90FDF71BFB2C994DA80F2216F05AFA13
:1002E0004D984E994F9A509B09F0A1FAFFE7579805
:1002F00090F890010146259140B1FFE7259801282B
:100300000DD0FFE72598022812D01AE00020C4F291
:10031000582056900020C4F2CC20559015E00020C3
:10032000C4F2E42056900020C4F2223055900CE034
:100330000020C4F22E3056900020C4F25E3055905A
:1003400003E0002056905590FFE79DED560AB5EE6C
:10035000400AF1EE10FA76D0FFE79DED550AB5EEB2
:10036000400AF1EE10FA6ED0FFE7579800F5826070
:100370002290FDF7B5FA9DED561A9FED7F2A8DED7F
:100380001E2A20EE020A30EE010ABDEEC00A10EE6F
:10039000100A2190FDF7AAFA9FED791A8DED1F1A28
:1003A00020EE010AB1EE001A30EE010ABDEEC00ADD
:1003B00010EE100A2090FDF793FA9DED1E2A9DED98
:1003C000551A20EE020A30EE010ABDEEC00A10EE08
:1003D000100A2390FDF78AFA9DED1F1ADDF880C000
:1003E000219A2298DDF88CE020EE010ABAEE0C1A70
:1003F00030EE010ABDEEC00A10EE101A6B46C3F8CB
:1004000010E0C3F80CC09A6001225A6002221A6000
:10041000596147F63071C0F6020105230BF0C2F9AD
:10042000579800F5826149A82490FDF76FFA249946
:1004300045A80F2216F0AEF945984699479A489B71
:1004400009F0F5F9FFE7579800F5D47000211991EC
:1004500000F01AFA0068FCF7A3FE19998DED1A0A4C
:10046000579800F5A07000F0E5FD9DED1A0A90ED9B
:10047000001A80EE010A9FEDC11A8DED1D1A20EEC3
:10048000010ABDEEC00A10EE100AC0F1B40027F850
:10049000560C579800F5D47001211B9100F0F4F927
:1004A0000068FCF77DFE1B998DED1C0A579800F53E
:1004B000A07000F0BFFD9DED1C0A9DED1D1A90ED92
:1004C000002A80EE020A20EE010ABDEEC00A10EEFC
:1004D000100AB430ADF81001022007F8590C37F8B3
:1004E000560CB0F5B47F04DDFFE7002027F8560C6A
:1004F000FFE7BDF81001B0F5B47F05DDFFE74FF46D
:10050000B470ADF81001FFE7579800F5A070002116
:1005100000F090FD90ED000AB5EE400AF1EE10FA01
:100520000BD1FFE7022007F8590C4FF4877027F82A
:10053000560C5A20ADF8100131E037F8560C092856
:100540000ADCFFE7BDF81001B0F5AF7F04DDFFE77F
:10055000022007F8590C21E037F8560C1D2811DC51
:10056000FFE7BDF81001B0F5A57F0BDDFFE7032025
:1005700007F8590C11E000BF9A99593FC3F5283F7D
:100580000AD7233F4FF4877027F8560C5A20ADF84E
:100590001001032007F8590CFFE7FFE7FFE7579822
:1005A00000F21F400F9017F8590C0E9037F8560CB8
:1005B0001090BDF81041FDF793F99FED711A20EEF0
:1005C000010ABDEEC00A10EE100A0D90FDF78EF97B
:1005D0000D9BDDF838C00F98DDF840E09FED691AFB
:1005E00020EE010ABDEEC00A10EE101A6A46119202
:1005F0003225D561956113610523D3609460C2F8FB
:1006000004E0C2F800C0516147F63371C0F6020140
:1006100002220BF0EEFA579800F21F4140A8129008
:1006200000F097FD12993CA80F2216F0B3F83C9801
:100630003D993E9A3F9B09F0FAF8579800F11C014A
:1006400039A81390FAF7A2FD13993AA81490FEF76F
:100650009FFD1498FEF7E2FC9FED4B1A8DED171AE3
:1006600080EE010A9FED491A8DED181A20EE010A5D
:10067000BDEEC00A10EE100A27F87A0C579800F168
:100680001C0136A81590FAF781FD159937A8169028
:10069000FEF77EFD1698FEF7C1FC9DED172A9DED35
:1006A000181A80EE020A20EE010AB3EE0E1A30EE9E
:1006B000010ABDEEC00A10EE100A27F8860C37F8C2
:1006C000860CB0F5B47F07DDFFE737F8860CA0F5A0
:1006D000B47027F8860CFFE7579800F21F400A9085
:1006E00037F87A0C099037F8860C0B90FDF7F8F87C
:1006F0009FED231A20EE010ABDEEC00A10EE100A8B
:100700000890FDF7F3F8089B099A0A98DDF82CE0A9
:100710009FED1C1A20EE010ABDEEC00A10EE101A61
:10072000EC462824CCF81C40CCF81840CCF810300B
:100730000523CCF80C30CCF808E0CCF804200222D9
:10074000CCF80020CCF8141047F63671C0F6020140
:100750000BF04FFA579800F21F4132A80C9000F0AE
:10076000F8FC0C992EA80F2216F014F82E982F9949
:10077000309A319B09F05BF858B0B0BD00003443AB
:100780009A99193FCDCCCC3DDB0FC9400000B44352
:1007900080B56F468EB00D900D98049000F5D27024
:1007A0000021069100F067F801680BA80590FEF79C
:1007B00036FA0598FEF732FC06988DED0C0A0A9081
:1007C000FFE70A98022821D8FFE7049800F5D470C3
:1007D00002900A9900F058F8006801684968884753
:1007E00002980A9900F050F80068FCF7D9FC0498C8
:1007F0008DED030A0A9900F050F89DED030A80ED93
:10080000000AFFE70A9801300A90DAE70020099011
:10081000FFE7099878B9FFE7049800F5D2700999C5
:1008200000F029F80068016849688847FFE70998DF
:1008300001300990EDE7049800F5D270002100F036
:100840001AF8016807A80190FEF7E9F901980CA9C8
:1008500000F02EF804988DED080A9DED081A90ED31
:10086000070A90ED092A81EE021A30EE010A80EDA6
:10087000070A0EB080BD82B00190009101980099E6
:1008800000EB810002B0704782B0019000910198A6
:10089000009900EB810002B0704782B00190009196
:1008A0000198009900EB810002B070470000000041
:1008B00080B56F4686B00590049105980190049824
:1008C00090ED000AFAF77EFD01988DED030A90ED98
:1008D000000A9DED031A30EE410A8DED020AFFE792
:1008E0000298EFF7BFFE41EC100B9FED191B53EC84
:1008F000112B51EC100BF0F793F948B1FFE79DED88
:10090000020A9FED181A30EE010A8DED020AE7E7A0
:10091000FFE70298EFF7A6FE41EC100B9FED0E1BD0
:1009200053EC112B51EC100BF0F766F948B1FFE7CF
:100930009DED020A9FED0A1A30EE010A8DED020AC2
:10094000E7E79DED020A06B080BD00BF00BF00BF13
:10095000182D4454FB210940182D4454FB2109C093
:10096000DB0FC940DB0FC9C080B56F46A2B0219034
:1009700021981490F4F7CDF90A4614994A61086158
:100980008B68CA6808694969C01A9141F0F7B2FAE0
:100990000146149800EE101A9FEDD61A80EE010A57
:1009A00080ED060A01694269C260816000F008FAC0
:1009B00014980021209190F890010146159140B1C2
:1009C000FFE71598012807D0FFE71598032806D000
:1009D00008E00120209008E00520209005E000209C
:1009E000209002E001202090FFE7149890F89001F9
:1009F00001461391022808D3FFE7139802285FD01D
:100A0000FFE7139803287DD1FFE7149890F86C1145
:100A10000020C907129039B1FFE7149890F87401CB
:100A200080F001001290FFE71498129901F0010183
:100A300080F87C1190F86C1101F0010180F87411BC
:100A400090F87C01C00700B3FFE71498D0F8840148
:100A5000D8B9FFE7149920981F90D1F86801D1F810
:100A60008011401A1E901F981E99884203D2FFE7FA
:100A70001F98119002E01E981190FFE714991198A9
:100A80001D901D98C1F88401FFE71499D1F88001E9
:100A9000D1F8841188420DD3FFE714994FF0FF304D
:100AA000C1F888010020C1F88001C1F8840181F8F3
:100AB0006C0104E01499C86BC1F88801FFE722E0DB
:100AC000149800F035FA8DED1C0A9DED1C0AB5EE68
:100AD000400AF1EE10FA04D1FFE74FF0FF3010901A
:100AE0000BE09DED1C1A9FEDB30A80EE010ABCEEEF
:100AF000C00A10EE100A1090FFE714991098C1F880
:100B0000880100E0FFE7149890F8910101460F91E9
:100B1000022804D3FFE70F98022809D009E01499AE
:100B20000020C1F88C014FF0FF30C1F88801FFE7C9
:100B3000FFE7149890ED630AD0ED0A0A90F83400AC
:100B4000B0FA80F040090BF0E5FD14988DED0A0A2B
:100B500000F5A0700D9000210C9100F06BFA9DED56
:100B60000A0A0C9902460D9882ED000A00F062FA1A
:100B700001460D9891ED000AB1EE400A8DED0B0A89
:100B8000012100F057FA9DED0B0A0C9902460D98D1
:100B900082ED000A00F04EFA01460D9809680E91A8
:100BA000022100F047FA01460E980860F4F7AFF80A
:100BB0001499D1F87021D1F88811801A88421FD376
:100BC000FFE71499D1F84C01C1F8780191ED082A9A
:100BD00091ED530A9FED781A81EE021A30EE010A68
:100BE00081ED530AD1F880010130C1F88001F4F79A
:100BF0008EF81499C1F87001002081F86D01FFE7AB
:100C0000149890F891010146099128B1FFE70998DD
:100C1000013802282FD3CBE000201B90FFE71B9860
:100C200078B9FFE7149800F5D2701B99FFF723FEFF
:100C30000068016889688847FFE71B9801301B90AE
:100C4000EDE700201A90FFE71A9802280FD8FFE777
:100C5000149800F5D4701A99FFF716FE0068016821
:100C600089688847FFE71A9801301A90ECE701205D
:100C70000CF096F89CE000201990FFE719980028E6
:100C80003ADCFFE7149800F5CA70199900F0DBF917
:100C9000014614980968069190ED530A8DED070AF4
:100CA00000F5D27008901999FFF7E5FD0068FCF790
:100CB00077FA14990698B0EE401A9DED070A9FED59
:100CC0003F2AC1EE020AD1ED061A91ED071A09F08A
:100CD00097F808988DED180A1999FFF7CCFD006870
:100CE0009DED180A016809688847FFE719980130E7
:100CF0001990C3E70024744900201790FFE7179864
:100D0000022839D8FFE7149800F5CC70179900F045
:100D1000A3F9014614980968039100F5A07017998A
:100D200000F088F90146149891ED000A8DED040A4F
:100D300000F5D47005901799FFF7A6FD0068FCF741
:100D40002FFA14990398F0EE400A9DED040A91EDF4
:100D5000061A08F0DEFF05988DED160A1799FFF7C1
:100D600093FD00689DED160A016809688847FFE752
:100D7000179801301790C2E7149890F83C0158B9C1
:100D8000FFE7012002900BF0BBFF1499029891ED50
:100D90000B0A0BF0C5FF0AE0012001900BF0B0FF39
:100DA0001499019891ED0C0A0BF0BAFFFFE7FFE7E9
:100DB00022B080BD00007A44DB0FC9C000F8FF45B7
:100DC00080B56F4682B001900198009090F8B40110
:100DD000012840F0A280FFE7009890F83400012835
:100DE0002FD1FFE7009991F8C30191F8C42140EA9F
:100DF000022000EE100AB8EE400A81ED540A91F884
:100E0000CD0191F8CE2140EA022000EE100AB8EEA2
:100E1000400A81ED560A4FF08340C1F85C0191F819
:100E2000CB0191F8CC2140EA022000EE100AB8EE86
:100E3000400A81ED580A0020C4F2C820C1F86401BC
:100E400035E0009890F8340080BBFFE7009991F8F6
:100E5000BF0191F8C02140EA022000EE100AB8EE6E
:100E6000400A81ED540A91F8CD0191F8CE2140EA73
:100E7000022000EE100AB8EE400A81ED560A00206A
:100E8000C4F2F010C1F85C0191F8CB0191F8CC21CB
:100E900040EA022000EE100AB8EE400A81ED580A3E
:100EA0000020C4F22010C1F86401FFE7FFE70098BA
:100EB00090ED540A90ED551AB4EE410AF1EE10FA95
:100EC0000ED1FFE70098D0F8680148B1FFE700981D
:100ED00090ED540AB5EE400AF1EE10FA17D1FFE793
:100EE000009890ED542A90ED560A90ED591A30EE84
:100EF000420A80EE010A14F079FB0099BCEEC00AA8
:100F000081ED5A0AD1F85001C1F85401FFE7009968
:100F1000D1F85C01C1F88C0107E000990A20C1F802
:100F20006801886BC1F88C01FFE702B080BD00004A
:100F300084B00290029890ED540A90ED561A80EE1B
:100F4000010A8DED010A90ED580A90ED591A80EED4
:100F5000010A8DED000A90F83400012803D1FFE763
:100F60000098039057E09DED010A9FED2D1AB4EE15
:100F7000410AF1EE10FA04DDFFE74FF07C500390D8
:100F800049E09DED010A9FED271AB4EE410AF1EE0A
:100F900010FA04DDFFE74FF07E5003903BE09DED3B
:100FA000010A9FED211AB4EE410AF1EE10FA07DDB5
:100FB000FFE79DED000A30EE000A8DED030A2AE0FE
:100FC0009DED010A9FED191AB4EE410AF1EE10FAF7
:100FD00009DDFFE79DED000AB0EE081A20EE010AD8
:100FE0008DED030A17E09DED010A9FED111AB4EE95
:100FF000410AF1EE10FA09DDFFE79DED000AB1EEBE
:10100000001A20EE010A8DED030A04E00020C4F26C
:10101000A0000390FFE79DED030A04B0704700BFF6
:101020006666663FCDCC4C3F9A99193FCDCC4C3E7D
:10103000CDCCCC3D82B0019000910198009900EB9D
:10104000810002B0704782B0019000910198009930
:1010500000EB810002B0704782B0019000910198CE
:10106000009900EB810002B0704783B002908DF8C8
:101070000710029900919DF8070091F8901188429D
:1010800001D1FFE705E000999DF8070081F8900184
:10109000FFE703B0704780B56F4684B0039007F850
:1010A000051C0399009117F8050C91F891118842DD
:1010B00001D1FFE727E00099002081F86C01019041
:1010C000FFE7019802280ED8FFE7009800F5CC70E2
:1010D0000199FFF7C1FF006808F044FEFFE701989F
:1010E00001300190EDE717F8050C022805D1FFE764
:1010F00000990020C1F88401FFE7009917F8050C5A
:1011000081F89101FFE704B080BD80B56F4682B0E1
:1011100001900199009101F2B51001F50B711022B7
:1011200015F03DFB009901F2C51001F21F210D22BF
:1011300015F035FB009901F5E97001F25121072204
:1011400015F02DFB009991F8E40181F8B40102B08B
:1011500080BD80B56F4682B0019101990F2215F0D4
:1011600019FB02B080BD80B56F4688B0079206902B
:10117000059106980090059913F092FB009813F0E2
:10118000A1FA01460098049102900020039007A85C
:1011900000F011F80499059A00F012F801900198F6
:1011A000039003980599884200D9FFE702A800F050
:1011B00016F808B080BD81B00090009801B070476B
:1011C00080B56F4684B0039002910192039A029811
:1011D00001991268FCF739FC019804B080BD80B514
:1011E0006F4682B00190019900910868496813F038
:1011F0006FFA009802B080BD80B56F4682B007F8E4
:10120000010C009117F8011C009A00F003F802B0DD
:1012100080BD000080B56F4684B0039007F8051CC0
:101220000192019800F5F0704FF0FF31FCF7A5FC3A
:1012300017F8050C01460091092844D80099DFE809
:1012400001F0050A0F1420252A33383D01980021AA
:10125000FFF721FF38E001980121FFF71CFF33E081
:1012600001980221FFF717FF2EE0019890F89101F5
:10127000022805D1FFE70199012081F86C01FFE701
:1012800022E001980021FFF7F0FE1DE00198022105
:10129000FFF7EBFE18E0019890F89011013101F092
:1012A0000101FFF7E2FE0FE001980321FFF7DDFEE9
:1012B0000AE00199002081F83C0105E00199012034
:1012C00081F83C0100E0FFE7019800F5F070FCF7C1
:1012D00094FC04B080BD81B0009041F2E720C0F6DC
:1012E000010001B0704780B56F4682B00190009157
:1012F0000199009A00F002F802B080BD80B56F46F7
:1013000084B00390029101920198009000994A687C
:1013100008788968904704B080BD81B0009041F2A0
:101320005930C0F6010001B0704783B002900191BE
:1013300000920298019901600099416003B07047E2
:1013400080B56F4682B001900198009000980168C6
:101350004068884702B080BD80B56F4682B001907A
:10136000019900F002F802B080BD80B56F4686B0EA
:101370000590049147F63E61C0F6020103A84FF0C4
:10138000FF32FCF7E4FDF3F7C2FC0290FFE704989C
:1013900000F5F270019000F022F80199024603A8CE
:1013A000FCF77BFE0498FFF7B0FE049800F5F070A0
:1013B0004FF0FF31FCF7E1FB0498FFF7E9F90498DF
:1013C000FFF7D2FA049800F5F070FCF716FC0498C9
:1013D00000F5EE70022102AAF0F7DDFBD7E781B03D
:1013E000EFF3058000900098002818BF012001B09D
:1013F000704780B56F4688B0079007980490002129
:10140000039141600160C16081600161143002900C
:10141000EFF79DFF0498039A183047F63971C0F62C
:10142000020100F05CF80498039A1C3047F6B061A2
:10143000C0F6020100F07DF8049803990162416250
:101440008162C1623030FDF74FFE04983430FDF701
:101450004BFE04983830FDF747FE04980399C163AA
:10146000016441648164C16401655430019000F0FD
:101470001AFA0499024601986B461A6041F28752A3
:10148000C0F6010247F64273C0F6020300F010FAFC
:10149000049803997C30FBF761FA04980399803033
:1014A000FBF75CFA049803998430FBF757FA02982B
:1014B000039A04990023CBF680730B624A628A6216
:1014C000CA626B4603221A6047F64772C0F60202F0
:1014D0004FF4807300F00FFA049808B080BD80B517
:1014E0006F4686B00490039107F80D2C0498019084
:1014F000059017F80D0CC00760B9FFE7039A47F68F
:10150000AE61C0F6020100201023F0F775FC0199CE
:1015100008600BE0039A47F6AD61C0F602010020B7
:101520001023F0F769FC01990860FFE7059806B001
:1015300080BD80B56F4686B00490039107F80D2CEE
:1015400004980190059017F80D0CC00760B9FFE7EB
:10155000039A47F6AE61C0F6020100200C23F0F7B3
:101560004BFC019908600BE0039A47F6AD61C0F6A9
:10157000020100200C23F0F73FFC01990860FFE70F
:10158000059806B080BD80B56F46DAB04D904C919D
:101590004B924C98012807D1FFE747F65370C0F6ED
:1015A0000200EFF7E4FE7BE14C98042840F07781DD
:1015B000FFE74B98406847F6E301C0F60201EEF7FB
:1015C0001FFE002840F0C280FFE74B98816843AAC5
:1015D00024924E924E98599044A82390FBF769FAB2
:1015E0002398002126910A22279200F0BDF9014696
:1015F0002398259113F00BF9249852905298FCF7F8
:1016000029FB25984A904B98C1683BAA29924F9292
:101610004F9858903CA82890FBF74BFA28982699A9
:10162000279A00F0A1F9014628982A9113F0EFF8C3
:10163000299853905398FCF70DFB2A9842904298B2
:10164000B0F57A7F04DDFFE74FF47A704290FFE750
:101650004298012803DCFFE702204290FFE7FFE702
:101660004A98429988423DDDFFE74D98343000F0BA
:1016700095F910EE100AEEF7F5FF41EC100B8DED29
:10168000200B4D98383000F089F910EE100AEEF773
:10169000E9FF41EC100B8DED1E0B4D98303000F042
:1016A0007DF910EE100AEEF7DDFF9DED1E2B9DED8E
:1016B000200B41EC110B684680ED002B80ED021BE6
:1016C00053EC102B47F69970C0F60200EFF74FFE6F
:1016D0004298F0F751F9F1F741FF42994A98401AC0
:1016E0004A90BDE74D98343000F058F910EE100ADA
:1016F000EEF7B8FF41EC100B8DED1C0B4D98383018
:1017000000F04CF910EE100AEEF7ACFF41EC100BB4
:101710008DED1A0B4D98303000F040F910EE100AA4
:10172000EEF7A0FF9DED1A2B9DED1C0B41EC110B6C
:10173000684680ED002B80ED021B53EC102B47F622
:10174000B170C0F60200EFF712FEA7E04B984068B8
:1017500047F6CB71C0F60201EEF752FD002840F0CB
:101760009C80FFE74B98816833AA1392509250985F
:10177000579034A81290FBF79CF91298002115910C
:101780000A22169200F0F0F801461298149113F014
:101790003EF8139854905498FCF75CFA14983A90D9
:1017A0004B98C1682BAA18925192519856902CA828
:1017B0001790FBF77EF917981599169A00F0D4F850
:1017C00001461798199113F022F8189855905598DA
:1017D000FCF740FA199832903298B0F57A7F04DD20
:1017E000FFE74FF47A703290FFE73298012803DC6C
:1017F000FFE702203290FFE7FFE73A9832998842EC
:101800004ADDFFE74D99086A4A6A06928A6A089299
:10181000C96A0A91EEF726FF0246069807920A4621
:10182000079942EC101B8DED100BEEF71BFF0246E3
:10183000089809920A46099942EC101B8DED0E0B8F
:10184000EEF710FF02460A980B920A460B9942ECFB
:10185000101B8DED0C0BEEF705FF9DED0C2B9DED98
:101860000E1B9DED100B41EC130B684680ED043B05
:1018700080ED022B80ED001B53EC102B47F6D67049
:10188000C0F60200EFF773FD3298F0F775F8329961
:101890003A98401A3A90B0E7FFE7FFE7FFE7FFE723
:1018A00000205AB080BD80B56F46F2F7DEF880BDEB
:1018B00080B56F4688B0D7F808C0079006910592AA
:1018C00004930798039020300599069A00F0ECFCE9
:1018D000039804996A4600235360136042F2BF22C2
:1018E000C0F60102F1F7CDF90398B968F1F7D6F91E
:1018F000039808B080BD80B56F468EB08446B86846
:10190000CDF830C00B910A92099307F8150C0C988A
:1019100004900DA8039000F0F6FC082010F0AEF83B
:1019200001460398079100F0EEFC01460B9A05A8CA
:1019300000F0F1FCDDF810E007990598069A4A607E
:101940000860079B0A99BDF8242017F8150CEC468F
:10195000CCF804E0CCF8000042F22D30C0F60100D3
:1019600010F064FF0EB080BD80B56F4684B0039068
:1019700002910192039813F0A7F80246029B019886
:101980006946086046F23150C0F6020047F6E3713E
:10199000C0F6020100F009FC04B080BD81B00090E7
:1019A000009890ED000A01B070470000F0B503AF59
:1019B0002DE9000F8DB00C900C980590F3F7A9F964
:1019C0000A460599CA6088600B684A688868C968D1
:1019D000C01A9141EFF78EFA0146059800EE101AF1
:1019E0009FED541A80EE010A80ED040A8168C268F6
:1019F00042600160C16B0B91016C0A91416C0991CD
:101A0000816C0891C16C0791016D06919DED083ABA
:101A10009DED074A90ED090A90ED0A2A90ED0B1A08
:101A200022EE042A20EE430A30EE420A9DED062AF9
:101A300021EE021A30EE410AB6EE001A20EE010A3B
:101A400042F20041C2F2000181ED000A9DED084A18
:101A50009DED065A90ED080A90ED0A3A90ED0B2A9A
:101A600023EE053A20EE040A30EE030A9DED073A14
:101A700022EE032A30EE420A20EE010A42F204412D
:101A8000C2F2000181ED000A9DED074A9DED065A64
:101A900090ED082A90ED093A90ED0B0A23EE053AF5
:101AA00022EE042A32EE432A9DED083A20EE030A84
:101AB00030EE020A20EE010A42F20841C2F20001B1
:101AC00081ED000A9DED064A9DED075A90ED080A4A
:101AD00090ED093A90ED0A2A23EE053A20EE040A29
:101AE00030EE030A9DED083A22EE032A30EE420A58
:101AF00020EE010A42F20C40C2F2000080ED000A22
:101B00009DED0B0AB5EE400AF1EE10FA14D1FFE795
:101B10009DED0A0AB5EE400AF1EE10FA0CD1FFE78E
:101B20009DED090AB5EE400AF1EE10FA00F0FE81D3
:101B300002E000BF00247449DDF814809DED0B0A1B
:101B40009DED0A1A21EE011A20EE000A30EE011A6C
:101B50009DED090A20EE000A30EE010A0AF023FD8D
:101B600042F21040C2F20000009080ED000A90EDB9
:101B7000001A9DED0B0A20EE010A8DED0B0A90ED87
:101B8000001A9DED0A0A20EE010A8DED0A0A90ED79
:101B9000001A9DED090A20EE010A8DED090A98ED63
:101BA000080A30EE000A42F2144AC2F2000A8AED34
:101BB000000A98ED090A30EE000A42F2184EC2F20D
:101BC000000E8EED000A98ED0A0A30EE000A42F28D
:101BD0001C40C2F2000080ED000A98ED0B0A30EEC6
:101BE000000A42F22046C2F2000686ED000A98ED95
:101BF000080AB1EE003A20EE030A42F22444C2F28F
:101C0000000484ED000A98ED090A20EE030A42F26E
:101C10002843C2F2000383ED000A98ED0A0A20EE81
:101C2000030A42F22C49C2F2000989ED000A98ED3C
:101C3000090AB2EE001A20EE010A42F23042C2F264
:101C4000000282ED000A98ED0A0A20EE010A42F233
:101C50003441C2F2000181ED000A98ED080A20EE3D
:101C6000000A42F2384BC2F2000B8BED000A98EDED
:101C7000090A20EE000A42F23C45C2F2000585ED59
